:020000040800F2
:1000000000500020CD0F00087D100008C536000804
:100010007D1000087D1000087D1000080000000021
:100020000000000000000000000000007D1000083B
:100030007D100008000000007D1000084544000805
:100040007D1000087D1000087D1000087D1000085C
:100050007D1000087D1000087D1000087D1000084C
:100060007D1000087D1000087D1000087D1000083C
:100070007D1000087D100008252100087D10000873
:100080007D1000087D1000087D1000087D1000081C
:100090007D1000087D1000087D1000087D1000080C
:1000A0007D1000087D1000087D1000087D100008FC
:1000B000A51200087D1000087D100008F119000845
:1000C000D91B0008F5190008D51B00087D10000891
:1000D0007D10000859210008952100087D100008B6
:1000E0007D1000087D1000087D1000080000000051
:1000F0000000000000000000000000000000000000
:0C01000000000000000000005FF808F1A3
:1001100010B5054C237833B9044810B10448AFF347
:1001200000800121217010BDD405002000000000D6
:10013000A402010808B5064B1BB106480649AFF3F7
:1001400000800648016811B1054A02B1904708BD18
:1001500000000000A4020108D8050020D4050020FA
:100160000000000081F0004102E000BF83F0004386
:1001700030B54FEA41044FEA430594EA050F08BF42
:1001800090EA020F1FBF54EA000C55EA020C7FEA06
:10019000645C7FEA655C00F0E2804FEA5454D4EB83
:1001A0005555B8BF6D420CDD2C4480EA020281EA4D
:1001B000030382EA000083EA010180EA020281EA85
:1001C0000303362D88BF30BD11F0004F4FEA0131D7
:1001D0004FF4801C4CEA113102D0404261EB4101E6
:1001E00013F0004F4FEA03334CEA133302D052426C
:1001F00063EB430394EA050F00F0A780A4F1010428
:10020000D5F1200E0DDB02FA0EFC22FA05F2801861
:1002100041F1000103FA0EF2801843FA05F3594147
:100220000EE0A5F120050EF1200E012A03FA0EFCC6
:1002300028BF4CF0020C43FA05F3C01851EBE371F0
:1002400001F0004507D54FF0000EDCF1000C7EEB0D
:1002500000006EEB0101B1F5801F1BD3B1F5001F4B
:100260000CD349085FEA30004FEA3C0C04F101046A
:100270004FEA445212F5800F80F09A80BCF1004F93
:1002800008BF5FEA500C50F1000041EB045141EA15
:10029000050130BD5FEA4C0C404141EB010111F416
:1002A000801FA4F10104E9D191F0000F04BF0146C1
:1002B0000020B1FA81F308BF2033A3F10B03B3F19F
:1002C00020020CDA0C3208DD02F1140CC2F10C022F
:1002D00001FA0CF021FA02F10CE002F11402D8BF8D
:1002E000C2F1200C01FA02F120FA0CFCDCBF41EA59
:1002F0000C019040E41AA2BF01EB0451294330BD28
:100300006FEA04041F3C1CDA0C340EDC04F1140404
:10031000C4F1200220FA04F001FA02F340EA0300DB
:1003200021FA04F345EA030130BDC4F10C04C4F121
:10033000200220FA02F001FA04F340EA0300294601
:1003400030BD21FA04F0294630BD94F0000F83F44B
:10035000801306BF81F480110134013D4EE77FEA2E
:10036000645C18BF7FEA655C29D094EA050F08BF7A
:1003700090EA020F05D054EA000C04BF194610465B
:1003800030BD91EA030F1EBF0021002030BD5FEA9F
:10039000545C05D14000494128BF41F0004130BDC7
:1003A00014F580043CBF01F5801130BD01F000451B
:1003B00045F0FE4141F470014FF0000030BD7FEA8E
:1003C000645C1ABF194610467FEA655C1CBF0B4689
:1003D000024650EA013406BF52EA033591EA030FA0
:1003E00041F4002130BD00BF90F0000F04BF002198
:1003F000704730B54FF4806404F132044FF00005CB
:100400004FF0000150E700BF90F0000F04BF002143
:10041000704730B54FF4806404F1320410F00045A9
:1004200048BF40424FF000013EE700BF42004FEAA4
:10043000E2014FEA31014FEA02701FBF12F07F4321
:1004400093F07F4F81F06051704792F0000F14BF1E
:1004500093F07F4F704730B54FF4607401F0004562
:1004600021F0004120E700BF50EA010208BF7047B9
:1004700030B54FF000050AE050EA010208BF7047AE
:1004800030B511F0004502D5404261EB41014FF417
:10049000806404F132045FEA915C3FF4DCAE4FF01B
:1004A00003025FEADC0C18BF03325FEADC0C18BF02
:1004B000033202EBDC02C2F1200300FA03FC20FA53
:1004C00002F001FA03FE40EA0E0021FA02F11444A0
:1004D000C1E600BF70B54FF0FF0C4CF4E06C1CEAB5
:1004E00011541DBF1CEA135594EA0C0F95EA0C0F2A
:1004F00000F0DEF82C4481EA030621EA4C5123EA9D
:100500004C5350EA013518BF52EA033541F48011CB
:1005100043F4801338D0A0FB02CE4FF00005E1FB7E
:1005200002E506F00042E0FB03E54FF00006E1FBC8
:1005300003569CF0000F18BF4EF0010EA4F1FF040B
:10054000B6F5007F64F5407404D25FEA4E0E6D414B
:1005500046EB060642EAC62141EA55514FEAC5205C
:1005600040EA5E504FEACE2EB4F1FD0C88BFBCF5D8
:10057000E06F1ED8BEF1004F08BF5FEA500E50F189
:10058000000041EB045170BD06F0004646EA01014F
:1005900040EA020081EA0301B4EB5C04C2BFD4EB81
:1005A0000C0541EA045170BD41F480114FF0000E7A
:1005B000013C00F3AB8014F1360FDEBF002001F0E8
:1005C000004170BDC4F10004203C35DA0C341BDC62
:1005D00004F11404C4F1200500FA05F320FA04F034
:1005E00001FA05F240EA020001F0004221F0004168
:1005F00010EBD37021FA04F642EB06015EEA430EDB
:1006000008BF20EAD37070BDC4F10C04C4F120050A
:1006100000FA04F320FA05F001FA04F240EA0200BD
:1006200001F0004110EBD37041F100015EEA430E8E
:1006300008BF20EAD37070BDC4F1200500FA05F2AE
:100640004EEA020E20FA04F301FA05F243EA02032D
:1006500021FA04F001F0004121FA04F220EA02003C
:1006600000EBD3705EEA430E08BF20EAD37070BD82
:1006700094F0000F0FD101F00046400041EB010162
:1006800011F4801F08BF013CF7D041EA060195F044
:10069000000F18BF704703F00046520043EB0303FE
:1006A00013F4801F08BF013DF7D043EA06037047EB
:1006B00094EA0C0F0CEA135518BF95EA0C0F0CD0F6
:1006C00050EA410618BF52EA4306D1D181EA03013C
:1006D00001F000414FF0000070BD50EA410606BF36
:1006E0001046194652EA430619D094EA0C0F02D17B
:1006F00050EA013613D195EA0C0F05D152EA0336C0
:100700001CBF104619460AD181EA030101F00041DD
:1007100041F0FE4141F470014FF0000070BD41F026
:10072000FE4141F4780170BD70B54FF0FF0C4CF400
:10073000E06C1CEA11541DBF1CEA135594EA0C0F1F
:1007400095EA0C0F00F0A7F8A4EB050481EA030E6C
:1007500052EA03354FEA013100F088804FEA033353
:100760004FF0805545EA131343EA12634FEA022221
:1007700045EA111545EA10654FEA00260EF00041E2
:100780009D4208BF964244F1FD0404F5407402D234
:100790005B084FEA3202B61A65EB03055B084FEAC5
:1007A00032024FF480104FF4002CB6EB020E75EBC2
:1007B000030E22BFB61A754640EA0C005B084FEAEA
:1007C0003202B6EB020E75EB030E22BFB61A754667
:1007D00040EA5C005B084FEA3202B6EB020E75EBB2
:1007E000030E22BFB61A754640EA9C005B084FEA2A
:1007F0003202B6EB020E75EB030E22BFB61A754637
:1008000040EADC0055EA060E18D04FEA051545EA25
:1008100016754FEA06164FEAC30343EA52734FEACE
:10082000C2025FEA1C1CC0D111F4801F0BD141EA47
:1008300000014FF000004FF0004CB6E711F4801FAC
:1008400004BF01430020B4F1FD0C88BFBCF5E06F8C
:100850003FF6AFAEB5EB030C04BFB6EB020C5FEA9C
:10086000500C50F1000041EB045170BD0EF0004EF1
:100870004EEA113114EB5C04C2BFD4EB0C0541EA23
:10088000045170BD41F480114FF0000E013C90E620
:1008900045EA060E8DE60CEA135594EA0C0F08BFE4
:1008A00095EA0C0F3FF43BAF94EA0C0F0AD150EAE3
:1008B00001347FF434AF95EA0C0F7FF425AF104676
:1008C00019462CE795EA0C0F06D152EA03353FF49E
:1008D000FDAE1046194622E750EA410618BF52EA1B
:1008E00043067FF4C5AE50EA41047FF40DAF52EAEF
:1008F00043057FF4EBAE12E74FEA4102B2F1E04369
:1009000024BFB3F5001CDCF1FE5C0DD901F0004CF6
:100910004FEAC0024CEA5070B2F1004F40EB830046
:1009200008BF20F00100704711F0804F21D113F172
:100930003872BCBF01F00040704741F480114FEAAB
:100940005252C2F11802C2F1200C10FA0CF320FA34
:1009500002F018BF40F001004FEAC1234FEAD32351
:1009600003FA0CFC40EA0C0023FA02F34FEA4303BB
:10097000CCE77FEA625307D150EA01331EBF4FF044
:10098000FE4040F44000704701F0004040F0FE405F
:1009900040F40000704700BF80F0004002E000BF5C
:1009A00081F0004142001FBF5FEA410392EA030F5A
:1009B0007FEA226C7FEA236C6AD04FEA1262D2EBA4
:1009C0001363C1BFD218414048404140B8BF5B42A9
:1009D000192B88BF704710F0004F40F4000020F042
:1009E0007F4018BF404211F0004F41F4000121F058
:1009F0007F4118BF494292EA030F3FD0A2F10102A2
:100A000041FA03FC10EB0C00C3F1200301FA03F1DF
:100A100000F0004302D5494260EB4000B0F5000F02
:100A200013D3B0F1807F06D340084FEA310102F1C1
:100A30000102FE2A51D2B1F1004F40EBC25008BF73
:100A400020F0010040EA03007047490040EB00003D
:100A500010F4000FA2F10102EDD1B0FA80FCACF16C
:100A6000080CB2EB0C0200FA0CF0AABF00EBC2506B
:100A700052421843BCBFD0401843704792F0000F59
:100A800081F4000106BF80F400000132013BB5E7AC
:100A90004FEA41037FEA226C18BF7FEA236C21D022
:100AA00092EA030F04D092F0000F08BF0846704787
:100AB00090EA010F1CBF0020704712F07F4F04D155
:100AC000400028BF40F00040704712F100723CBF68
:100AD00000F50000704700F0004343F0FE4040F492
:100AE000000070477FEA226216BF08467FEA236350
:100AF0000146420206BF5FEA412390EA010F40F43B
:100B0000800070474FF0000304E000BF10F0004386
:100B100048BF40425FEA000C08BF704743F096436D
:100B200001464FF000001CE050EA010208BF704788
:100B30004FF000030AE000BF50EA010208BF70470F
:100B400011F0004302D5404261EB41015FEA010C24
:100B500002BF84460146002043F0B64308BFA3F11C
:100B60008053A3F50003BCFA8CF2083AA3EBC253FE
:100B700010DB01FA02FC634400FA02FCC2F120021D
:100B8000BCF1004F20FA02F243EB020008BF20F054
:100B90000100704702F1200201FA02FCC2F12002BA
:100BA00050EA4C0021FA02F243EB020008BF20EAAF
:100BB000DC7070474FF0FF0C1CEAD0521EBF1CEADD
:100BC000D15392EA0C0F93EA0C0F6FD01A4480EACB
:100BD000010C400218BF5FEA41211ED04FF00063B4
:100BE00043EA501043EA5111A0FB01310CF00040E0
:100BF000B1F5000F3EBF490041EAD3715B0040EA06
:100C0000010062F17F02FD2A1DD8B3F1004F40EBD5
:100C1000C25008BF20F00100704790F0000F0CF0A8
:100C2000004C08BF49024CEA502040EA51207F3A6C
:100C3000C2BFD2F1FF0340EAC250704740F4000047
:100C40004FF00003013A5DDC12F1190FDCBF00F038
:100C500000407047C2F10002410021FA02F1C2F1E6
:100C6000200200FA02FC5FEA310040F1000053EA82
:100C70004C0308BF20EADC70704792F0000F00F0D0
:100C8000004C02BF400010F4000F013AF9D040EAD6
:100C90000C0093F0000F01F0004C02BF490011F46A
:100CA000000F013BF9D041EA0C018FE70CEAD15368
:100CB00092EA0C0F18BF93EA0C0F0AD030F0004CE8
:100CC00018BF31F0004CD8D180EA010000F000409C
:100CD000704790F0000F17BF90F0004F084691F05A
:100CE000000F91F0004F14D092EA0C0F01D1420294
:100CF0000FD193EA0C0F03D14B0218BF084608D15D
:100D000080EA010000F0004040F0FE4040F40000A6
:100D1000704740F0FE4040F4400070474FF0FF0C39
:100D20001CEAD0521EBF1CEAD15392EA0C0F93EA80
:100D30000C0F69D0A2EB030280EA010C49024FEAD2
:100D4000402037D04FF0805343EA111143EA10138B
:100D50000CF000408B4238BF5B0042F17D024FF443
:100D6000000C8B4224BF5B1A40EA0C00B3EB510F1E
:100D700024BFA3EB510340EA5C00B3EB910F24BF07
:100D8000A3EB910340EA9C00B3EBD10F24BFA3EB8C
:100D9000D10340EADC001B0118BF5FEA1C1CE0D154
:100DA000FD2A3FF650AF8B4240EBC25008BF20F007
:100DB000010070470CF0004C4CEA50207F32C2BF5B
:100DC000D2F1FF0340EAC250704740F400004FF0F8
:100DD0000003013A37E792F0000F00F0004C02BF29
:100DE000400010F4000F013AF9D040EA0C0093F0F3
:100DF000000F01F0004C02BF490011F4000F013B4D
:100E0000F9D041EA0C0195E70CEAD15392EA0C0FB4
:100E100008D142027FF47DAF93EA0C0F7FF470AFEC
:100E2000084676E793EA0C0F04D14B023FF44CAF2F
:100E300008466EE730F0004C18BF31F0004CCAD1C4
:100E400030F000427FF45CAF31F000437FF43CAF00
:100E50005FE700BF4FF0FF3C06E000BF4FF0010C22
:100E600002E000BF4FF0010C4DF804CD4FEA400204
:100E70004FEA41037FEA226C18BF7FEA236C11D04E
:100E800001B052EA530C18BF90EA010F58BFB2EB01
:100E9000030088BFC81738BF6FEAE17018BF40F081
:100EA000010070477FEA226C02D15FEA402C05D135
:100EB0007FEA236CE4D15FEA412CE1D05DF8040BBA
:100EC000704700BF844608466146FFE70FB5FFF74D
:100ED000C9FF002848BF10F1000F0FBD4DF808ED05
:100EE000FFF7F4FF0CBF012000205DF808FB00BFF6
:100EF0004DF808EDFFF7EAFF34BF012000205DF850
:100F000008FB00BF4DF808EDFFF7E0FF94BF01209C
:100F100000205DF808FB00BF4DF808EDFFF7D2FF99
:100F200094BF012000205DF808FB00BF4DF808EDDC
:100F3000FFF7C8FF34BF012000205DF808FB00BFA9
:100F40004FEA4002B2F1FE4F0FD34FF09E03B3EBD6
:100F500012620DD94FEA002343F0004310F0004F16
:100F600023FA02F018BF404270474FF0000070476C
:100F700012F1610F01D1420205D110F0004008BF0B
:100F80006FF0004070474FF00000704742000ED2F3
:100F9000B2F1FE4F0BD34FF09E03B3EB126209D4B4
:100FA0004FEA002343F0004323FA02F070474FF06A
:100FB0000000704712F1610F01D1420202D14FF0DF
:100FC000FF3070474FF00000704700BF1D481E49BA
:100FD000026800608A4200F01F80002100F004B81F
:100FE0001A4B5B584350043119481A4B42189A4225
:100FF000FFF4F6AF184A00F003B8002342F8043BB0
:10100000164B9A42FFF4F9AF08F0B4FC0BF046FD22
:1010100002F02CFAFFF7FEBF114E12483060124862
:10102000016821F070610160410201600F4C1820DD
:1010300020600F490F4808600F48D0F800D0406882
:1010400000470000F04F0020EFBEADDEC8020108EF
:1010500000000020D4050020D405002054170020F3
:10106000181002400900000004000140140C014067
:10107000000C01404434434400F0FF1FFFF7FEBF63
:10108000034BDA880280198941805B89838070472D
:10109000F0050020054B1A88510001805A88510044
:1010A00041809B885A008280704700BFF005002075
:1010B00070470000074B084A0360426007480B6016
:1010C000074A4FF07E534860CB604FF4BC711180EB
:1010D000704700BFB110000881100008951000088B
:1010E0004200002038B504460D46002D14DD0520D1
:1010F00003F0DBF9204608F049FE204608F04BFEDD
:101100000028FAD1204608F04AFE204608F04CFE9E
:101110000028FAD1013DE8E738BD000070B53E4D2A
:1011200090B0284609F04AFC3C4880213C4B069090
:101130000A9120204FF40051002409264FF48072B8
:1011400005930D904FF480630E91284605A90C93EA
:101150000B92079409940F94089609F0A7FC28466F
:10116000012109F0D0FC009403942E4C01254FF48A
:1011700060222046694602928DF804508DF8055091
:101180008DF8106008F0CCFD20460A212A46032382
:1011900008F017FE20460B210222032308F011FE5F
:1011A000032220460C21134608F00BFE20460D2199
:1011B0000422032308F005FE20460E210522032306
:1011C00008F0FFFD20460F210323062208F0F9FD59
:1011D000204605210722032308F0F3FD20460621BF
:1011E0000822032308F0EDFD3246032320460721A1
:1011F00008F0E7FD2046294608F0BFFD20462946B5
:1012000008F0B2FD20460221FFF76CFF2046294678
:1012100008F0CEFD10B070BD08000240F0050020BF
:101220004C24014000240140002070472DE9F0418A
:101230000F88002347FA03F2D2072DD58A7803F0EE
:101240000705DC08AD0012F0100F18BF91F803C0BD
:1012500002F00F0618BF46EA0C064FF00F0C0CFA0E
:1012600005FC06FA05F550F82480282A28EA0C0C1B
:1012700045EA0C0540F8245006D1012202FA03F297
:10128000C46824EA020206E0482A05D1012202FAD3
:1012900003F2C4682243C2600133102BCAD1BDE8F7
:1012A000F08100005E4B2DE9F0411C78002C58D0F5
:1012B00002214FF0804009F0F0F8012808D1594C84
:1012C000594B21884FF08040198009F0D9F82080CF
:1012D00002214FF0804009F0EBF852485249028851
:1012E0000B889A4201D9D21A01E0D843121893B25E
:1012F000B3F57A6F4D4A03D900231370BDE8F0812E
:10130000A3F2EF2188B240F2DA5188421ED8127857
:10131000072A1BD84648032A00EBC201CB80454967
:1013200009D840F2D930834205D9012303FA02F2E9
:10133000087802430A7009780F2907D13E483D4BCF
:10134000016800221A700A685368984737483A4B78
:1013500001784A1C0270186801680A689047BDE865
:10136000F0812546354850F8347000EBC402B7F1DF
:10137000804F9688B2F806804DD13846414609F034
:101380008CF8012847D13846414609F091F80C2ED7
:101390001CD8DFE806F0071B1B1B0C1B1B1B111BBB
:1013A0001B1B16004FF0804009F06AF80DE04FF06B
:1013B000804009F068F808E04FF0804009F066F8D6
:1013C00003E04FF0804009F064F80546184AE00059
:1013D00012F83410131839B90120194902F83400F1
:1013E00002225D804A8011E05F889D80BD4201D964
:1013F000EF1B01E0F9436F18DF80002717540E4AF6
:1014000010680368196888470D494F804FF0804085
:101410000E8008F099FF0134082CA3D1BDE8F081BB
:101420004D060020520600204E06002054060020E3
:101430000C0600204C060020C810002000000020F0
:10144000020600202DE9F04300248FB00A2706464B
:101450000D463A46214604A801940BF017FC21469C
:1014600010220AA80BF012FC844B854A1D608548A7
:101470007578337840F2DC510570D180D181D1820A
:10148000D183D184D185D186D187002B00F094807F
:1014900007A821463A460BF0F9FB03942820002DBB
:1014A00042D0012502A98DF80B004FF002087648C2
:1014B000ADF808508DF80A8008F07AFB1C2203A8CA
:1014C0008DF80C208DF80D408DF80E508DF80F50D2
:1014D00008F0CEFC07A808F0B7FE4FF6FF704723D0
:1014E000ADF8200007A94FF08040ADF81C30ADF8F2
:1014F0001E4008F061FD65494FF080404C80CC8073
:101500000C810C808D80624C08F01EFF4FF08040F3
:1015100041462A4608F0BBFE4FF08040294608F0BD
:101520009CFEA946277047E002221F248DF80B007D
:1015300002A955488DF80A20ADF8084008F038FB9C
:1015400001241C2103A88DF80C108DF80D508DF886
:101550000E408DF80F4008F08BFC07A808F074FED1
:101560004FF6FF704723ADF8200007A94FF08040E9
:10157000ADF81C30ADF81E5008F01EFD434A5580F2
:101580009480D5801581434C404963199888088020
:101590002859083508F0D8FE202DF4D14FF08040AE
:1015A0001E21012208F073FE01214FF0804008F057
:1015B00054FE374904250D7018254FF47071ADF8AD
:1015C00004108DF8075001A9022533488DF8065004
:1015D00008F0EEFA04A808F037FE33892F484722B6
:1015E00090FBF3F4611EADF814102D4804A9ADF87A
:1015F000102008F0E1FC4FF47A704FF480717022F3
:1016000000230124ADF82E00ADF8341024480AA9B7
:10161000ADF82820ADF82C30ADF82A40ADF83050A8
:1016200008F014FD0AA91E4808F054FD0AA91C4838
:1016300008F094FD0AA91A4808F0D2FD08211848BC
:1016400008F02EFE0821164808F032FE0821144842
:1016500008F038FE0821124808F03CFE21461048E8
:1016600008F0FBFD21460E4808F003FE0C48082157
:1016700008F016FE0FB0BDE8F08300BFC8100020D0
:101680000C0600204D060020000801400206002044
:101690005006002000000020000C014040420F00D6
:1016A00000080040044B1A78824203D9034B53F8D8
:1016B00020000180704700BF500600209CDC00081D
:1016C00070470000024B03EBC000C088704700BFAA
:1016D0000C0600202DE9F84F9C4C2068838A9BB2B1
:1016E00013F0010239D0018821F400631A04110CAF
:1016F0000180012109F040F9954A964B11780020AC
:101700001870D9B1944803781BB9944A1178FF290D
:1017100014D10123037092480278022A06D18B4922
:101720000B68188882B242F4006119808D4B87489B
:1017300019780068012209F039F92FE18948834BB3
:1017400001780022186809F031F9844A1178FF29DC
:1017500000F02481FF207F4BDEE003F00201C9B2DC
:1017600000293DD0BFF35F8F7D4D2E78012E354689
:1017700016D177490B789BB177490B7883B1114625
:1017800009F0FAF8BFF35F8F20683146038B09F048
:10179000E7F8754A206816704FF480613246FBE026
:1017A000038BBFF35F8F6E490A78022A09D1684B19
:1017B0001A7832B1684B1A781AB1002109F0DCF8B6
:1017C000E5E00978032907D1614B1A7822B1624913
:1017D0000B78002B40F0DD804FF480610122DBE0CC
:1017E00003F00406F6B2002E71D0594BDFF8788171
:1017F0001A78012688F80060574B002A4DD01A78D5
:10180000002A4AD0564D2F78524D022F574F29D9D2
:1018100009F0B2F8206895F80090D7F800A009F018
:10182000C2F84FFA89FB0AF80B0009EB06003146B3
:101830002870206809F094F8206888F800603F68F4
:1018400095F8008009F0AFF84FFA88F907F8090019
:10185000B04420684FF48061324685F8008009F07A
:1018600097F82BE0314609F07BF820682E78D7F8FE
:10187000008009F098F84FFA86F9731C08F80900FF
:10188000D9B220684FFA81F83F68297009F08BF8C7
:10189000033607F808002E7010E01B78012113B9F9
:1018A000334A13782BB109F05BF82A480278511CAF
:1018B00003E009F049F8284801210170234A116822
:1018C0000B8803F4807082B2002AF9D166E003F03D
:1018D00040010F461F4D09B3244B2F78D3F80080E9
:1018E00009F061F84FFA87F908F80900781CC1B2CD
:1018F00029701B4D4FB22A780337BA4205D12068B0
:101900004FF48061324609F043F8124B28781A7878
:1019100051B2884242D1501C18703FE01B063DD5A1
:101920002B785EB2721C27D0124901330A682B70E3
:10193000915D09F036F80A4895F900200178914246
:101940002CD120684FF480613A4625E068060020DB
:1019500067060020660600206C060020590600205D
:101960005A0600206E060020650600206006002052
:10197000580600205C060020154A2970117809F0ED
:1019800010F81448017811B9134B1A7832B913487A
:1019900000684FF48061002208F0FAFF0E4A104BF5
:1019A000117893F900004A1C90420ED10D4B0E495C
:1019B000187800220A7028B1084908684FF440716D
:1019C00008F0E6FF094B00221A70BDE8F88F00BF4F
:1019D00059060020670600205A06002068060020ED
:1019E00066060020650600206C0600206D060020BB
:1019F000FFF770BEFFF76EBEF0B5484C89B04FF4EC
:101A000040651C2307460226204602A9ADF808506F
:101A10008DF80A308DF80B60FFF708FC4048142160
:101A200007608DF80E10204603A9ADF80C508DF814
:101A30000F60FFF7FBFB25610825384CA2685205B3
:101A400003D40A2002F026FDF7E74FF480660A204F
:101A5000666102F01FFD6F1E0A20266102F01AFD6A
:101A600017F0FF05E9D14FF4006767610A2002F023
:101A700011FD66610A2002F00DFD26610A2002F0C8
:101A800009FD022027611C218DF80F002046244CFF
:101A90004FF440638DF80E1003A9ADF80C30FFF73A
:101AA000C5FB206808F0B2FE04A808F033FF2068E8
:101AB0002A464FF4407108F06BFF1A484FF48043F8
:101AC0004BF6FF72049001212068ADF81C30ADF890
:101AD0001620ADF8145008F02BFF04A9206808F078
:101AE000AFFE4FF4A06008F0B9F92221012201A84D
:101AF0008DF804108DF805508DF806508DF80720EC
:101B000008F0B6F9212301A82E468DF804308DF88F
:101B1000055008F0ADF909B0F0BD00BF000C014060
:101B200068060020801A0600274B37B51868818A9E
:101B30008AB20192019B13F4706F02D0234A0121F3
:101B40001170019B13F4E06F31D04FF480610022DB
:101B5000038B08F01DFF0198810528D41A4D2868D1
:101B6000018801F4007293B20BBB048804F4807105
:101B70008CB29CB1028802F4807399B20029F9D129
:101B8000012108F0EDFE10480068028802F400739D
:101B900099B20029F9D1FFF72FFF08E0012108F0E1
:101BA000DFFE28684FF44071224608F0F1FE064837
:101BB0000268938A23F470610804030C0449938239
:101BC00000220A703EBD00BF6806002064060020A7
:101BD0006D060020FFF7A8BFFFF7A6BF014B1888CE
:101BE00080B2704756060020F8B5134B05469B8916
:101BF0000E461446ECB116B116F8017B00E0FF2743
:101C00000D48022108F086F80028F9D00A48394624
:101C100008F07BF80848012108F07CF80028F9D08A
:101C2000054808F074F8C0B20DB105F8010B013C8D
:101C3000E0E70120F8BD00BF003800402DE9F04783
:101C4000012188B04FF4804008F0B4FD374C0121E9
:101C50004FF4804008F0C6FD03214FF420401823C4
:101C6000ADF800008DF80310204669468DF802306B
:101C70004FF00408FFF7DAFA2D4E4FF48042204669
:101C80006946ADF800204FF480554FF0100A8DF8EA
:101C90000280FFF7CBFA69462046ADF800508DF878
:101CA00002A0FFF7C3FA304607F0D2FF07214FF436
:101CB000007000230222ADF81600ADF81C104FF0A2
:101CC0000109304603A94FF48277ADF80C30ADF826
:101CD0001030ADF81A30ADF81220ADF80E70ADF836
:101CE00014901F46ADF818A007F0E4FF30464946AF
:101CF00007F0FFFF9F238DF804308DF805708DF8F5
:101D000006708DF807700DEB08014246656102A868
:101D1000FFF76AFF25619DF80900B0F1EF014A4223
:101D200052EB010008B0BDE8F08700BF000C014095
:101D3000003800407047036B13B15A68006C01E033
:101D4000026AC069101A18BF01207047436B13B1B3
:101D500090F844007047826A406A111A4B4253EB74
:101D60000100704730B50446007985B000230D4668
:101D70000091C107ADF80430ADF80630ADF8083079
:101D8000ADF80C30ADF80A3002D50422ADF80A20C7
:101D9000820705D5BDF80A1041F00803ADF80A30F6
:101DA000206D694608F088FBA56005B030BD026B68
:101DB000034610B5406942B11A6CD9688C1A013AD1
:101DC00018BF1146005D196410BD196ADA68405CDD
:101DD0000131B1FBF2F402FB1411196210BD0000D5
:101DE000F0B51D465F4B91B098420F46164604D1A0
:101DF0001046294600F0F0F807E05B49884240F0C1
:101E0000AC801046294600F03DF9044605F0040276
:101E100000202571A66001962062E061A0626062E8
:101E2000E762ADF8080002F0FF0632B14FF4005748
:101E3000ADF80A704FF4806601E0ADF80A60002347
:101E4000ADF80C6015F00106ADF8103002D1ADF818
:101E50000E6002E00421ADF80E1005F0020505F059
:101E6000FF072DB1BDF80E0040F00802ADF80E20BE
:101E700001A9206D08F020FB05A808F037FEE36CEF
:101E800000254FF48051802005930E910F95099500
:101E90000B950A900C953EB3206BD0B16369E66850
:101EA000202206930D920896079508F087FD206B77
:101EB00005A908F0FBFD206B012108F024FE206D30
:101EC0004021012208F076FB206B08F031FE2064EF
:101ED0000AE0206D40F2255108F075FB206D40F2BC
:101EE0002551012208F04CFB05A808F0FFFD4FF436
:101EF0008055A16C0E958026002505910F950995BA
:101F00000B950A960C951FB3606BD8B1226910230C
:101F1000079308920D9508F051FD606B05A908F034
:101F2000C5FD0122606B022108F0F8FD606B2946B7
:101F300008F0FCFD606B314645600122206D08F021
:101F400039FB05E0206D40F22771012208F018FBF3
:101F5000206D012108F008FB00E00024204611B0AC
:101F6000F0BD00BF0038014000440040836A816931
:101F7000426BC918D160416A994203D9CB1A5360A8
:101F8000816204E00169CB1A536000228262002161
:101F900080F84410406B012108F0B5BD10B5426ACD
:101FA0008469A154416A02690131B1FBF2F402FB78
:101FB0001411426B416232B11368DB070BD4BDE8E8
:101FC0001040FFF7D3BF006D40F227710122BDE83A
:101FD000104008F0D5BA10BD234B13B5234A9860C2
:101FE00023481A6058614FF4807222480C462249F7
:101FF000DA601A61214A9961011D18659964D964F2
:102000001A630121143A4FF480405A6308F0C6FB6A
:10201000022318214FF40070A2078DF80330ADF8A9
:1020200000008DF8021003D515486946FFF7FEF849
:1020300048234FF480628DF80230E307ADF80020AA
:1020400003D50F486946FFF7F1F80E2001218DF8FE
:10205000040001A88DF805108DF806108DF8071002
:1020600007F006FF00481CBD30090020BCDC00085A
:102070002F08002000380140AF0600205800024021
:1020800000080140214B224A13B598600C4680207D
:1020900040211A60D86019611E4A1F491F485A61C1
:1020A00098610A1D19654FF4003001219A64DA64C1
:1020B00008F080FB042002231821ADF80000A007DF
:1020C0008DF803308DF8021003D515486946FFF7E7
:1020D000ADF808224823E107ADF800208DF8023062
:1020E00003D50F486946FFF7A1F8262001218DF896
:1020F0000400022201A88DF805108DF806208DF845
:10210000071007F0B5FE01481CBD00BF8409002080
:10211000BCDC0008AF070020004400406F06002030
:102120000008014010B50B4C4FF4005008F004FDBE
:102130000021606B08F0E7FC626AA36A9A4204D04F
:102140002046BDE81040FFF711BF012084F844008D
:1021500010BD00BF300900200D4B186D028802F041
:1021600080018AB29AB19A6A596A8A420AD09969F8
:10217000895C013281801969B2FBF1F001FB102208
:102180009A62704740F22771002208F0F9B970474F
:10219000300900201C4B10B51A6D1488A4B204F04D
:1021A000200188B290B1D96A19B1938898B2884752
:1021B0000CE09288D9695869D2B24254D869DA6879
:1021C000411CB1FBF2F002FB1011D96104F0800454
:1021D000A4B2C4B10C4B9A6A586A82420BD0986977
:1021E000196D805C013288801969B2FBF1F001FB46
:1021F00010229A6210BD186D40F227710022BDE8CE
:10220000104008F0BDB910BD84090020014B1868CA
:1022100002F0EEB8441700200149002000F0ACBEE7
:102220000D22000810B5FEF771FC0A49FEF7C2FC4A
:102230000949FEF773FD094B044618680078FEF75C
:1022400065FC01462046FEF7B5FCFEF79FFE80B216
:1022500010BD00BF3333534000F07F45EC09002030
:1022600038B50D4C00202578FEF7DEFF0B4A05F04F
:10227000070322F813000135002325701846D15AB0
:1022800002334018102B80B2F9D1C008FFF7CAFF03
:10229000034A107038BD00BFD8090020DA090020B9
:1022A000CC100020074B084A19781088884207D3C1
:1022B000064B1A68907888428CBF00200120704736
:1022C00000207047CC100020CE100020EC09002028
:1022D00038B5114B2024186000250020FEF7A4FF1C
:1022E0002D180A2002F0E1F8013CF6D1C5F34F1099
:1022F000FFF798FF084901230A6851786418A04243
:1023000002D30133062BF9D104489278037053436A
:1023100003490B8038BD00BFEC09002040000020BD
:10232000CE1000202DE9F04F0446008885B048B952
:10233000B4F9023043B9B4F90420D2F1010138BF35
:10234000002102E0002100E0014611F0010377D1F5
:102350003D4D00B22B7000F03FFD0646B4F902007F
:1023600000F03AFD0546B4F9040000F035FD0446DE
:10237000304608F0EBFB0746304608F05BFC804631
:10238000284608F0E3FB0646284608F053FC0546BD
:10239000204608F0DBFB8246204608F04BFC39461D
:1023A00081465046FEF706FC394683464846FEF70E
:1023B00001FC514601904046FEF7FCFB4946029065
:1023C0004046FEF7F7FB314603905046FEF7F2FB1E
:1023D0001E4C4946206006F10040FEF7EBFB294603
:1023E0006060A5600298FEF7E5FB01460198FEF7E4
:1023F000D9FA2946E0600398FEF7DCFB014658460F
:10240000FEF7CEFA3146206108F10040FEF7D2FB1C
:10241000294660615846FEF7CDFB01460398FEF75A
:10242000BFFA2946A0610198FEF7C4FB0146029855
:10243000FEF7B8FA3946E0613046FEF7BBFB206292
:1024400005B0BDE8F08F00BF41000020F00900207A
:102450002DE9F8434D4B0C460168013A196080881C
:102460009880072A30D8DFE802F004080F14191EFC
:102470002226188820805A8803E0598821801A88EB
:10248000524262809A881EE01988484220805A8809
:10249000F6E75988484220801A88F2E719884842AE
:1024A000208058880CE05A882280188808E0198813
:1024B00021805A8803E05988484220801A88504277
:1024C00060809B885A42A280314B1A78002A5AD1E8
:1024D000B4F90000FEF71AFB8046B4F90200FEF7DB
:1024E00015FB0746B4F90400FEF710FB294D06461C
:1024F00029684046FEF75EFBE96881463846FEF7EC
:1025000059FB01464846FEF74DFAA9698146304617
:10251000FEF750FB01464846FEF744FA08F04AFB36
:10252000696820804046FEF745FB296981463846A8
:10253000FEF740FB01464846FEF734FAE96981465A
:102540003046FEF737FB01464846FEF72BFA08F007
:1025500031FBA96860804046FEF72CFB6969804624
:102560003846FEF727FB01464046FEF71BFA296A6C
:1025700007463046FEF71EFB01463846FEF712FAC4
:1025800008F018FBA080BDE8F88300BF140A002003
:1025900041000020F009002070B5124D06462B784E
:1025A000114C9BB101F070FF2268B318984218D308
:1025B0000021297001F068FF20600C4802780AB100
:1025C000531E03700A480121017070BD01F05CFFC9
:1025D00021683231884204D30120287001F054FF71
:1025E000206070BD1C0A0020240A00201E0A002062
:1025F0001D0A002037B58DF805101F498DF80730EA
:102600000B788DF8040002A88DF80620C21812F885
:10261000044C0D46443CE0B20A2828D81749022B46
:1026200031F8104003D814B12046FFF7B5FF2B78DE
:10263000022B0BD9124D2D6801F026FF021B95428B
:1026400004D20D490F4B0020087018700E48027814
:102650000146012A00D074B9074B1878022801D826
:10266000421C1A7000230B7008490B7003E03224DF
:10267000022BD9D9DBE73EBD1A0A0020D4DC0008C2
:10268000240A00201E0A00201D0A00201C0A002027
:10269000014B1860704700BFC810002070B53D4B5B
:1026A00004465A7B3C4802B1012202704FF400708C
:1026B00000F094F9002828D0384E394B316858780A
:1026C0000D68003018BF0120AA68904748B13368F0
:1026D000344D1868012102692970904708B1022120
:1026E00029702E4D2B681868C268904728B12C4974
:1026F0004B7813B92B4A0220107029680B6898692F
:10270000804710B1274900220A70202004F04AFCBB
:1027100060B12048244B827A0AB9C17A21B120489D
:10272000C27A0AB9012100E0002119701D4B187806
:10273000022802D14C204E211DE0012807D14D2155
:1027400053204C220B46BDE87040FFF753BF164A9A
:102750001178012903D1532001464E2206E00E4B89
:102760001878012804D15320014602464D23EAE798
:1027700024B153204D210A464423E4E70B4A117843
:1027800021B13220BDE87040FFF706BF084B1C7036
:1027900070BD00BFC41600201B0A0020C810002016
:1027A000B31600201F0A0020200A00201E0A002065
:1027B0001C0A0020014B1870704700BF1E0A002041
:1027C0000E4B1A78402A16D15888B0F5697F12D17D
:1027D0001979BE290FD193F8A1230020EF2A0CD13B
:1027E00013F8011B064A48409342F9D1D0F1010089
:1027F00038BF0020704700207047704700F801087C
:10280000A4FB01087FB51B4D1B4C284604F000FCBF
:102810002146284604F016FC1F3D04F1240001F077
:1028200039FD2E4604F15C0004F060FF16F8C20B7F
:1028300002F0ECF8304603F01FFB681C03F0DAFBF3
:1028400005F1B80000F0C0FD04F1280001F01CFD06
:1028500004F1490304F1380005F1C001009301902F
:10286000029105F17800A11D224605F1BE0302F098
:102870005DFD7FBD97140020A011002010B5FFF76B
:102880009FFF10B90A2001F0B3FE0E4C0E492046FE
:102890004FF469720AF04CF994F8A033022B02D974
:1028A000002084F8A00394F8A013D02202FB014377
:1028B000064803F598710AF03BF9BDE81040FFF7B0
:1028C000A1BF00BFD010002000F80108781400203C
:1028D00008B5FFF7D3FF0F2014210122BDE80840FF
:1028E00007F028B808B5054BD02202FB0030044998
:1028F00000F598700AF01CF908BD00BFD010002048
:1029000078140020224A38B5402313704FF46970C0
:102910000023BE21EF245080117182F8A14382F878
:10292000A2331D461A4A985C0133B3F5697F85EAE4
:102930000005F7D182F8A25307F04EFE04250024CB
:10294000691E11F0FF0516D0342007F059FE11481A
:1029500007F0ACFE0F4C04280BD10F4A2046A158BB
:1029600007F07AFE0D4B04349C42F4D1042804464F
:1029700001D00446E4E707F03BFE042C02D1FFF748
:102980001FFF20B90A20BDE8384001F031BE38BD34
:10299000D010002000F80108D018FE17A4FB010891
:1029A000C82314211E22038001238170C270037189
:1029B00064214FF496722823C180028143817047BD
:1029C00008B5054B93F8A003FFF78CFFFFF79AFFBC
:1029D000BDE80840FFF77CBFD0100020034B99688A
:1029E00008420CBF00200120704700BFD01000201B
:1029F000024B9A6810439860704700BFD0100020C7
:102A00002DE9F347AF4AB04D10685168AF4C6B46A3
:102A100003C34FF46972002128460AF037F9D02227
:102A2000002120460AF032F94020032128700220BC
:102A30006971FFF7DDFFFA22A5F8F2202A236E2242
:102A4000A5F8EE304FF4FA7085F804212B2340F2FC
:102A50004C42A5F8F60085F80531212002F54873AF
:102A6000202185F80601A5F8163140F27E404FF48A
:102A70007A7300274FF001094FF4167685F8F410A9
:102A8000A5F8142140F2DC5100F52F72A5F8D00012
:102A900003F5CB70A5F81211A5F8F060A5F8D220C7
:102AA00085F8A073A5F8FA70A5F8F870A5F8FC7081
:102AB00085F8E27085F8E37085F8E470A5F8E670B3
:102AC000A5F8E870A5F8EA7085F8ED7085F8EC9047
:102AD00085F8077185F82C7185F82D7185F82E71B0
:102AE00085F8107185F8187185F8197185F81A91B3
:102AF000A5F8D430A5F8D6006C30A5F8D8004FF46E
:102B0000C870A5F8DE004FF41650322340F2B452DC
:102B1000C5F8240140F6AC50A5F8DA20A5F8DC3061
:102B20001A46A5F8E030A8814FF4E1331E20C5F81D
:102B30002031E07252232073552085F82A31E0704D
:102B400017230B204FF028086375A37560712D23A0
:102B500014204FF0080E22716373A0714FF00E0A1B
:102B600085F81C7185F81D7185F8287185F8297123
:102B7000AF7385F81B71277084F8018084F8028098
:102B8000E775A7732776E773677684F810E06074BB
:102B900050204FF0640C4FF0780E84F807A0E076D8
:102BA0004FF00A0A5A20A376207284F81CC084F8D9
:102BB0000AE02375E077412304F12A0084F812A08B
:102BC00084F8098084F81E9084F82030E18484F829
:102BD000212084F8237084F8247084F8257084F808
:102BE000227001F0FFFE0421394B84F82E10394881
:102BF0003949152284F83420A063E36321643748FF
:102C000005F58471278584F82F8084F8308084F856
:102C1000449004F001FB4FF44872C8204FF49663CF
:102C200040F2D9313E4684F8707084F8717084F8AF
:102C3000728084F8739084F87670A4F8742084F815
:102C4000B8A084F8B900A4F8BA30A4F8BC104FF4C6
:102C50007F724FF4FA601DF80710A4F87820A0F5F1
:102C6000FA73FF220137A4F87A00A4F87C3084F8C4
:102C70007E1084F87F200834082FE8D113480124FF
:102C800080F8BE4080F8BF4080F8C040C230FFF7F7
:102C900087FE00200C4B0021C2181030C0281161A3
:102CA000F8D100240E48D02220180849D03409F069
:102CB0003FFFB4F51C7FF5D102B0BDE8F047FFF748
:102CC00021BE00BF84DC0008D01000207814002052
:102CD000F6287C3F9A99193F3D0A773FEADC0008C5
:102CE0000012002008B5FFF76BFD18B9BDE80840D9
:102CF000FFF786BE08BD0000024B9A6822EA00007A
:102D000098607047D0100020014B9868704700BF52
:102D1000D0100020044B986800F04101B1F141024D
:102D2000534253EB02007047D0100020884203DB6F
:102D30008242B4BF11460146084670470023036132
:102D400070472DE9F041066904460136012E0D4613
:102D5000066105D10023616021608360BDE8F081D8
:102D6000D0F8008008464146FDF71AFE0746304677
:102D7000FDF7CCFE01463846FDF7D0FF0146404640
:102D8000FDF710FE0646606031462846FDF708FE56
:102D900001463846FDF70EFFA168FDF703FE2660E9
:102DA000E060A060BDE8F08110B50446006901282C
:102DB00007DD0138FDF7AAFE0146E068FDF7AEFF2A
:102DC00010BD002010BD08B5FFF7EEFFBDE80840BC
:102DD00007F0BEBF0000000008B5FDF715FB04A317
:102DE000D3E90023FDF776FBFDF786FD08BD00BFA4
:102DF000399D52A246DF913F2DE9F041069C0646DF
:102E00000F46002B0CBF4FF020084FF03008204633
:102E100010F8013B0BB9154603E0002AFBDD013A2F
:102E2000F6E7002D04DD30464146B847013DF8E79E
:102E300014F8011B11B13046B847F9E7BDE8F0813D
:102E40002DE9F04389B006460F4603921C46039ACB
:102E5000134613F8011B0393002900F08A802529EB
:102E600001D0304683E0002004905578911C302D2D
:102E7000039105D19578033203924FF0010800E0E9
:102E80008046A5F13003D8B2092806D8284603A900
:102E90000A2204AB00F020F905466C2D05D10399F8
:102EA000012211F8015B039100E00022642D2FD074
:102EB00010D8582D3AD006D8002D5AD0252DC6D17D
:102EC0003046294653E0632DC1D130462178251D77
:102ED000B8474AE0752D0DD0782D27D0732DB6D187
:102EE000251D2468304600943946049A0023FFF7D4
:102EF00083FF3AE0251D20680A2122B1002205AB9C
:102F000000F074F802E005AB00F0A0F82C4623E0D6
:102F100005AD04F104092068294612B100F08BF8D0
:102F200001E000F0B8F84C46009517E004F1040900
:102F30002068102142B1B5F15804634253EB0402FA
:102F400005AB00F053F806E0B5F158035A425A4178
:102F500005AB00F07BF84C4605A80090304639469A
:102F6000049A4346FFF748FF71E72C466FE7B847DE
:102F70006DE709B0BDE8F083024B196002490860B3
:102F8000704700BF280A00202C0A00200FB407B5A4
:102F9000094904AB0868094953F8042B09680193EF
:102FA000FFF74EFF064B186801F041FA0028F9D0F0
:102FB000BDE80E4004B070472C0A0020280A00200B
:102FC0004417002070B50646B6FBF2F408461546D5
:102FD00014B12046FFF7F6FF05FB1464024B195DA0
:102FE00000F8011B70BD00BFF3DC0008F0B5012440
:102FF000B0FBF4F58D4201D34C43F9E70026C4B190
:10300000B0FBF4F504FB1500B4FBF1F41EB9002D80
:1030100001DC002CF4D1092DEFB204DD002A0CBF35
:103020005725372500E03025ED1903F8015B0136FF
:10303000E5E71C70F0BD00280B4603DA2D22404264
:1030400003F8012B0A210022FFF7D0BFF0B50124BD
:10305000B0FBF4F58D4201D34C43F9E70026C4B12F
:10306000B0FBF4F504FB1500B4FBF1F41EB9002D20
:1030700001DC002CF4D1092DEFB204DD002A0CBFD5
:103080005725372500E03025ED1903F8015B01369F
:10309000E5E71C70F0BD00280B4603DA2D22404204
:1030A00003F8012B0A210022FFF7D0BFA0F1300363
:1030B000DAB2092A01D818467047A0F16101052942
:1030C00001D857387047A0F14103052B01D8373894
:1030D00070474FF0FF3070472DE9F8430D68044604
:1030E0000F469046994600262046FFF7DFFF00284E
:1030F00006DB404504DC08FB060615F8014BF3E748
:103100003D602046C9F80060BDE8F883931E222B7D
:1031100088BF0A22031E10B50C4603DA2D2001F8E1
:10312000010B5842FFF74EFF00210170204610BDF1
:1031300030B587B005460C4603A800210C2209F0E3
:10314000A5FD28460021FDF7F1FE20B128462949BA
:10315000FDF728FC03E028462649FDF721FC264917
:10316000FDF728FDFDF7ECFE054685EAE570A0EBCE
:10317000E5700A226946FFF7C9FF002D01DB202315
:1031800000E02D2368468DF80C3009F017FF012868
:1031900007D130228DF80D208DF80E208DF80F20EC
:1031A0000CE0022805D130218DF80D108DF80E109D
:1031B00004E0032802D130208DF80D00694603A8F1
:1031C00009F0FAFD03A809F0F9FEC51EEDB22A4682
:1031D00003A9204609F090FF0023635520460749C4
:1031E00009F0EAFD03A92046491909F0E5FD20464A
:1031F00007B030BD6F12033A00007A44B0E6000811
:103200002DE9F041027803460130202AFAD0092A3C
:10321000F8D02D2A02D10346414D04E02B2A08BFE5
:1032200003464FF07E551E460024334616F8010B28
:10323000A0F13007F9B209290DD83A492046FDF727
:10324000B9FC04463846FDF761FC01462046FDF70F
:10325000A9FB0446E9E72E2817D1324F334616F86A
:10326000010B3038C2B2092A0FD8FDF74FFC39469E
:10327000FDF754FD01462046FDF794FB294904461D
:103280003846FDF797FC0746E8E71878652801D02F
:10329000452839D15E782D2E02D19F1C012605E0EC
:1032A0002B2E01D05F1C00E09F1C00267B1E0027F8
:1032B00013F8012F303AD1B2092903D80A2000FBB4
:1032C0000727F5E7B7F59A7F28BF4FF49A77B846F6
:1032D0004FF07E51B8F1070F07D908461249FDF7A4
:1032E00069FCA8F108080146F4E707F0070737B1C1
:1032F00008460C49FDF75EFC013F0146F7E72EB199
:103300002046FDF70BFD04E04FF07E512046FDF70F
:1033100051FC01462846FDF74DFCBDE8F08100BF99
:10332000000080BF0000204120BCBE4C014B0022A9
:103330009A807047300A0020034BB3F90400D0F1A3
:10334000010038BF00207047300A00200649074BB3
:103350000A68B3F90400137805214B439842D4BF9F
:1033600000200120704700BF380A0020300A0020EA
:1033700010B50446FFF7EAFF002814BF20460020DE
:1033800000F0010010BD0000074B084A1968B2F9AF
:1033900004004B780A78D118052251438842D4BFE3
:1033A00000200120704700BF380A0020300A0020AA
:1033B000044B9A8811B2142901DD143A00E000226E
:1033C0009A807047300A0020024B002218600248A1
:1033D00082807047380A0020300A0020034B0449DD
:1033E0001860044800220160C28070473C0A002037
:1033F00018DD0008300A002008B501F0EBFA024B96
:1034000000221A7008BD00BFB316002010B5FFF7E8
:103410009DFFE0B1104B5C78201C18BF0120FFF726
:10342000A7FF70B10D480E4B01680E484A8901682C
:103430001A805A809A804A88DA800B4BD888411CBF
:10344000D980FFF7A1FF00B90CB9FFF7D5FF064BF4
:103450009A88501C988010BDB31600203C0A0020AA
:103460000A170020380A0020300A002070B5894C65
:1034700086B0FFF737FCFFF701FAA07B003018BFDA
:10348000012001F01DF8FEF7C7FE94F8073133B1B3
:10349000012B01D0092B02D18DF8003004E000216E
:1034A0008DF8001084F807116846FDF737FE0220FA
:1034B000FFF794FA10B17848FEF70AFF7748FEF755
:1034C00031FF022003F078FD754D724AB5F92830BE
:1034D00002F1E200B2F8EE1092F8ED2000F07CFF6D
:1034E00010B9032001F084F86E4C4FF400464FF4FD
:1034F000805066610A25C4F810086A4C6A4EE36879
:10350000013D83F40041E160F26882F48050F06094
:10351000192000F0CAFF192000F0C7FF15F0FF05C1
:10352000EBD14FF480534FF4004133612161594C8A
:1035300001F0F6FA607904F1100101F057FF04F58B
:10354000907004F05DFC66790E2E01D0082E03D138
:1035500001228DF80A2001E08DF80A504FF48070A6
:10356000FFF73CFA18B90820FFF738FA00E001200D
:1035700000F001008DF80600FFF7CCFB8DF8070086
:103580000120FFF72BFA8DF805000820FFF726FA37
:1035900080F001058DF8045002F04EFB3D4E404B8B
:1035A0008DF8080093F8C010B6F8E000B6F8DE20F9
:1035B000C1F38004ADF80E004FF47A754FF48040EB
:1035C0008DF80940ADF80C20ADF81050FFF706FA61
:1035D00018B1B6F8DA30ADF81030BDF80C10B1F50E
:1035E000FA7F02D90024ADF810402D48B6F8122118
:1035F00096F80761B0F8BC50012EADF81220ADF876
:10360000145004D0092E01D1072600E000262748D7
:103610008DF80B60FFF7E2FE254C2060FFF738F8CD
:1036200001A82168FDF70EFF2048216803F068FD1E
:103630004FF48070FFF7D2F968B10820FFF7CEF998
:1036400048B9144B1B4A93F81D0193F81C11A2F1C1
:10365000C10302F01FFD4FF40060FFF7BFF910B186
:10366000154804F0C1F800F0F5FE1449094A086055
:103670005079052803D14FF4C87000F0F3FC104EC8
:103680004FF47A70012500F00BFE757300F0FCF921
:10369000FCE700BFD0100020D4110020B61100209C
:1036A000781400200008014000100140D8110020CB
:1036B000C81000203A15002044170020640A00209A
:1036C000B316002008B5034BB3F9D40001F0A4FFF2
:1036D000FEE700BFD010002008B500F0E7FD0B4B5F
:1036E00050B19A7842B1597879B901225A70084B91
:1036F00008491888088008BD587830B90220FF2191
:103700000122BDE8084006F015B908BDB316002037
:1037100092150020561500202DE9F04FB54BB64A02
:10372000B3F90600D18C85B088420FDBB0F5FA6F93
:1037300092F8254007DA451A6C43A1F5FA6694FB26
:10374000F6F4643403E0C4F1640400E06424AB4A9A
:10375000A94BB2F8127192F9EC2093F8231000975C
:10376000574293F87050019193F87160B9B293F891
:1037700024300291002103930A469E4FDDF8008019
:1037800031F907C040F2E637C8EB0C0303F2F31E31
:10379000BE4503D8002BB8BF5B4201E04FF4FA737B
:1037A000022ADFF864822CD025B1AB42CCBFC5EB36
:1037B000030300236427DFF878A293FBF7FE6FF082
:1037C000630B3AF81E900BFB0E3B0EF1010E3AF91B
:1037D0001EA00FFA89FECEEB0A0E0EFB0BFE9EFB1F
:1037E000F7FEF14428F80190DDF8048003FB08FEA1
:1037F000834B9EFBF3F3DB199BB2634393FBF7F719
:1038000012E026B1B342CCBFC6EB03030023029FF4
:103810005F43A8F80470039F002BB8BF5B427B4353
:10382000774F93FBF7F76437734B02EB030E9EF869
:103830000190642307FB09F898FBF3F9DFF8F481A2
:1038400002F808909EF80B909EF815E007FB09F827
:1038500007FB0EF798FBF3F9DFF8DC8197FBF3F336
:1038600002F80890DDF80080664FC445D35503DAAE
:10387000654BCF5A7F42CF5201320231032A7FF487
:103880007CAF5E4C4FF4FA62B4F81411FFF74EFAB5
:10389000B4F814614FF47A75801B4543C6F5FA639A
:1038A000B5FBF3F56421594895FBF1F36FF063061E
:1038B00030F8132006FB0355013330F9130013B21F
:1038C000C01A4543524B504C95FBF1F1587A8A1877
:1038D000E280002838D04F4F4F4D3E882988721A19
:1038E00010B2FFF779FA074607F030F90646384676
:1038F00007F0A0F90546B4F90200FDF707F90746FD
:10390000B4F90000FDF702F931468046FDF752F99F
:10391000294681463846FDF74DF901464846FDF7F0
:103920003FF8FDF70DFB314620803846FDF742F9A0
:10393000294606464046FDF73DF901463046FDF76B
:1039400031F8FDF7FDFA60800220FFF747F890B1EB
:10395000324806220378591CCBB20370B3FBF2F055
:1039600002FB103111F0FF0F05D1FEF779FCFEF7D5
:1039700099FC2B4B18702A4A1078003018BF012090
:10398000FEF78CFE00F074FB18B100F08FFC58B904
:1039900004E0022003F006FB0028F6D0214BDA6891
:1039A00082F48051D9600EE0194B997819B11D4A03
:1039B0004FF4805010615B781BB11A484FF480516E
:1039C000416103F0F1FE1848184A01681368C81AEB
:1039D000002835DB0E4B587B80BB9870114B01F5EE
:1039E000F421D86880F48050D86001F5907313609A
:1039F00026E000BF0A17002078140020D010002015
:103A00000CFEFFFF8B150020DA160020E2160020C6
:103A1000B316002092150020561500205B0A0020E6
:103A2000540A002000100140400A00204C0A0020E7
:103A3000FA1600208E1500208815002001219970AB
:103A400004F0EAF90C4A107830B94FF40060FEF740
:103A5000C5FF08B103F0E2FE202003F0A3FA18B17D
:103A60000649086803F084FA054B9A680AB10548CC
:103A7000904705B0BDE8F08F30100020400A0020CC
:103A8000701500204A15002038B50820FEF7A6FF63
:103A900010B1994803F056FB984B994A1B6811687E
:103AA000591A002902DA002800F01B8203F59C4411
:103AB000914820349349146003F056FB4FF4804042
:103AC000FEF78CFF20B1904D2B780BB900F082FFF0
:103AD0008E4A92F81B11B1B18D4CC81C34F91050AC
:103AE0004FF47A720021A5F57A70FFF71FF9FDF700
:103AF0000DF88849FDF712F98749FDF75BF8FDF7E6
:103B000045FA864B18804FF40070FEF767FF20B12E
:103B1000834A116808684469A0477C4D0022B5F8C3
:103B20001401B5F81641134679499B08555E854244
:103B3000C4BF63F07F03DBB2A542B8BF43F04003CC
:103B40000232082AF0D17748774A047805469C4229
:103B500004D11078F92803D8411C00E0002111702D
:103B60004FF480402B70FEF739FF68B1674D684B0A
:103B7000B5F81211B5F8DC20B3F90640881A844272
:103B800002DD8B189C420CDB4FF48040FEF726FFD1
:103B9000D8B95F4C5D49B4F90650B1F8142195428B
:103BA00013DA00F023FF00F029FF6048B0F8463038
:103BB0005BB1554C5E492578002D00F01F820A78D4
:103BC000002A00F01B82FFF787FD574B1C78142C4E
:103BD00040F0CA80564D6C78ECB1544BB3F8465067
:103BE0002DB950490C785F2C01D100F0F3FE474A03
:103BF00092F81801002800F0B7804C4BB3F84650FB
:103C0000002D40F0B18047490C787D2C40F0AC800D
:103C100000F0E0FEA8E0434D2978572911D14FF478
:103C20007A7000F03DFB4FF48070FEF7D7FE08B1CC
:103C300002F08EF9082003F0B5F9E0B93D4B188089
:103C400019E00420FEF7CAFEA8B12A785A2A12D138
:103C50003948037823B104703848012202700AE021
:103C6000374C257885F00101217009B1022000E070
:103C70000320FEF79FFD2B4C25785D2D00F0C581BC
:103C80005B2D00F0C4815E2D00F0C381274BB3F89B
:103C9000465035B923490C786F2C02D1FFF71CFD33
:103CA00015E01A4A1F4B92F8180118B115B91D7882
:103CB0007E2DF3D01978972904D14FF4C87000F005
:103CC000D1F904E0A72902D1194A012494731548B7
:103CD0000378BB2B03D11548818D8D1C04E0B72BD5
:103CE00004D11248838D9D1E858531E0BE2B29D1DC
:103CF0000E4D6A8D941C2AE0D8110020400A002045
:103D0000600A002008170020C4160020D0100020F0
:103D10000A17002000007A4400C07F445415002098
:103D2000C81000205A0A0020500A002078140020F1
:103D3000B316002092150020440A0020530A0020E8
:103D4000510A0020BD2B0FD1744D698D8C1E6C85DE
:103D5000734C94F8A003FEF7C5FDFEF7D3FDFEF704
:103D6000B7FD7048002202700420FEF737FE0028DD
:103D70002CD06D4B1A788AB16C48457875B16C4976
:103D8000674AB1F90640B2F81401844206DD694D74
:103D90002C781CB9684932220A801C70654B587C0B
:103DA00050B1664B1D782DB9654C227812B9624826
:103DB00032210180012008E0614D2C7834B15B4A4A
:103DC000517819B95F4B29700120187000235E4C9F
:103DD0001A4634F8020F40F2135501B2A942CCBF83
:103DE0000025012505FA03F5A0F21550B0F5C77FAF
:103DF0008CBF002001202A435D1C00FA05F002431D
:103E000040F2A4608142D4BF00210121981C01FA34
:103E100000F103330A430C2B92B2DAD100233F495D
:103E2000444C01EB4300B0F846100A420CBF00209E
:103E3000012018550133152BF1D1627822B10220EF
:103E400003F0B0F868B914E04FF40070FEF7C6FD57
:103E500078B13E4C21680868C36898470028EED1C5
:103E600007E0324CE17839B900F0C0FD0120E07084
:103E700002E02E4C0022E2702E4B2C4C987830B190
:103E800021790022E27019B900F0B0FD0120207103
:103E9000284B26491A780AB901200870CA782C4B99
:103EA00012B92249087918B14FF40041596102E072
:103EB0004FF400421A61202003F074F808B102F0B8
:103EC000F9FF1C4B19481A7B02B101221449827276
:103ED0004B79082B01D00E2B45D1144A002050728B
:103EE00041E01C480368042B3DD8DFE803F00305DC
:103EF000080B35000122026001684B1C0360026858
:103F0000511C0160134803685A1C02604FF4807012
:103F1000FEF764FD00B302F0CBF924E07814002032
:103F2000D0100020500A0020510A0020B3160020B3
:103F30000A170020C4160020580A0020520A002048
:103F4000440A0020530A002010170020C810002047
:103F500000080140480A00203648002101604FF463
:103F60000050FEF73BFD00F075FA334B33499A8958
:103F70000860334B1AB11968411A002959DB8418BB
:103F80001C6000F0D1FFFFF7C7FB00F063FA2D4B78
:103F90002A4A19681060441A18602B482B4A90F876
:103FA0007630148053B12A49CC780CB90A792AB1F9
:103FB0002848294BC48819880A19C280202002F099
:103FC000F1FF40B12248C3790BB9017A19B1047BE2
:103FD0000CB102F0E5FE2148214A174B00F11E0109
:103FE0001468B3F8F62000F12903A04701F026FB7E
:103FF00001F0A2FABDE8384001F0FABA487800288A
:104000003FF4E3AD00F0E6FCDFE5012102E0022130
:1040100000E00321CCB20848621E80F8A023FEF71E
:1040200071FCFEF72BFC02202821224605F082FCC1
:104030002CE638BD480A0020D0100020400A00209D
:104040005C0A0020640A002078140020560A002030
:10405000B3160020DA1600208C0B00207914002003
:1040600044000020014B1880704700BF6A0A0020FE
:10407000034B1888D0F1010038BF0020704700BF03
:104080006A0A0020F8B51E4B0022196813461D4C21
:104090002588B5F5C87F1C4D01D10026EE501B4E7A
:1040A000EF5832F906C0184C6744EF50002504332E
:1040B00095538D5202320C2BE9D1124B1A88012AEA
:1040C00018D1236803F1C8024FF4C87392FBF3F2CE
:1040D0000A806268C83292FBF3F24A80A268C83252
:1040E00092FBF3F30A4A12889B1A8B8000F07AFC49
:1040F000FEF766FC034801884A1E0280F8BD00BF37
:10410000641500206A0A0020780A0020AC150020FF
:1041100042000020F8B5354B0446188832280ED1ED
:104120003349344D0A683448168857889388218863
:1041300062882E806F80AB800180428001E0002881
:1041400034D02B4D00222E681346284F2B49388837
:10415000322801D10025CD502948CD58175EED19E0
:10416000CD50002104331152B15202320C2B0D46B6
:10417000EBD11E480188012914D1224B224A02208A
:1041800011701D70FEF716FB1A4A19481188036852
:1041900050889288198058809A80174B19885888BF
:1041A00021806080114B1A88511E198017480378AE
:1041B000DBB10F4900220B681049027008683222F7
:1041C00090FBF2F01880486890FBF2F05880896804
:1041D0000F4891FBF2F201882046521A9A8000F0B3
:1041E00001FCBDE8F840FEF7EBBBF8BD580A002023
:1041F000641500206C0A0020720A0020840A002046
:10420000AC150020520A0020440A0020530A002066
:1042100042000020064B02881988891A19804288BA
:104220005988891A5980808899880A1A9A80704713
:10423000AC1500200F4B10B5596804460E4888474E
:104240000D480E4A01461278FEF702F90C48038821
:1042500013B12046FFF716FF0420FEF7BFFB10B195
:104260002046FFF757FF07490868BDE81040FFF7F1
:10427000D1BF00BF58150020AC150020680A0020EF
:104280006A0A002064150020014B1860704700BFC7
:1042900064150020014B1860704700BFA00A002081
:1042A000014B1880704700BFE00A0020034B1888BC
:1042B000D0F1010038BF0020704700BFE00A0020A5
:1042C0002DE9F8433C4B3D48596888473B483C4AF8
:1042D00001461278FEF7BCF83A480388002B42D01A
:1042E000394C256800242F782646254635490A880A
:1042F000B2F57A7F08D1354B354A00201421E850B9
:1043000001FB0620FEF71AFDDFF8B0802F4B38F9CD
:104310000400E9584FF014090A18EA502C4B09FB25
:104320000639FCF7F3FB01464846FEF70AFD00207C
:1043300024F80800DFF88C802649B8F80020605285
:10434000012A2FD14846FEF73EFD8146DFB13846AF
:10435000FCF7DCFB01464846FCF7E8FD98B14FF45A
:104360007A73A8F80030154B1A4A18881188401A39
:104370001880518858889288401A99885880881ADD
:104380009880BDE8F883114B4FF47A72E858114BCE
:1043900000F5FA7191FBF2F0E0520F210A200122A0
:1043A00005F0C8FA013604350234032E9ED10549C2
:1043B0000A88501E0880D6E770150020941500204A
:1043C000E20A0020E00A0020A00A0020940A00204F
:1043D000A40A0020660B002008B503480349FCF737
:1043E00069FE012008BD00BF58150020701500208F
:1043F00008B503681A68904708BD38B505460C46ED
:1044000014F8011B19B12846FFF7F2FFF8E738BD91
:1044100008B503685968884708BD08B503689968F6
:10442000884708BD08B50368DA68904708BD08B535
:1044300003681969884708BD08B503685A69904739
:1044400008BD7047024B1A68501C1860704700BFC7
:10445000E40A002010B5094A094913688C681068FD
:104460008342F8D1074A106811684FF47A725043BA
:10447000001BB0FBF1F102FB031010BDE40A0020A9
:1044800010E000E0E80A0020014B1868704700BF08
:10449000E40A002038B50446FFF7DCFF0546FFF7C5
:1044A000D9FF401BA042FAD338BD10B504462CB149
:1044B0004FF47A70FFF7EEFF013CF8E710BD000003
:1044C000F0B53E4B8BB0054601AC0FCB84E80F0036
:1044D000284605F0AFFA0121394806F06BF90121B1
:1044E00044F61D2006F05AF901200146354E06F02B
:1044F00049F90AAD06F082F900204FF6FF718DF8F8
:10450000020025F8281D304669462F4FFCF78EFE25
:104510002E486946FCF78AFE69463846FCF786FE57
:104520002B4B5A6842F000705860FFF78AFF4FF437
:1045300080514FF40043274A39613361106826499E
:10454000884206D19DF80A30142B02D110228DF832
:104550000A20211D0198FCF769FE1E481E4B0168C8
:10456000994206D19DF81220142A02D110208DF80C
:10457000120004A90398FCF759FE05A806F0B4F848
:10458000059B1649164AB3FBF1F0164910600868FE
:104590004FF47A73B0FBF3F2511E1348134AF02321
:1045A000416082F823300021072381600360FDF71A
:1045B00045FB6420FFF779FF0BB0F0BD8CDC0008F1
:1045C000070040000008014000100140000C0140BD
:1045D0000000014084010020001BB70040420F0092
:1045E000E80A00208801002010E000E000ED00E073
:1045F00010B540F2DB1460430D4B4FF400424FF412
:1046000080515A61841EC3F810180948C26882F4A8
:104610000043C360D0F80C1881F48052C0F80C2815
:104620002046FFF742FF1920FFF73FFFEDE700BFED
:104630000008014010B1034A034B1A6003480449C3
:10464000C8607047EFBEADDEF04F00200400FA05F1
:1046500000ED00E02DE9F04F89B00793754B074658
:104660000692B3F90000B3F902200028B8BF404217
:10467000002AB8BF524200248242B8BF02460592C7
:104680002546A146A0460494A24626466A49CB7810
:1046900013B90A79002A38D0022E36D0674B654804
:1046A000EA5EDDF818B0295E02EB4100CBF10001B3
:1046B0005A46FEF73BFB6249DDF81CC06B5E3CF9D5
:1046C0000520C01A8318F879FA7E584364214FF008
:1046D000050E90FBF1F06FF0040151430EFB02F266
:1046E0000393FEF723FBDFF878B1039B824654F86F
:1046F0000B00544942F210721818FEF717FB7A7C2F
:1047000044F80B005043011304914B48C3781BB18C
:1047100002790AB9022E2FD14649502035F901807D
:10472000DFF828B100FB08F2BB5DDFF8389135F9FE
:104730000B0092FBF3F154F809300A1AD0184249E1
:104740004FF47A52FEF7F2FA35F90B1049F80400EB
:104750000029B8BF4942B1F5207F02DD002049F8A9
:10476000040059F80420B9197D23887A92FBF3FCE0
:1047700000FB0CFE4FEAAE192F4B1A79B2B1022E94
:1047800014D0DDF814B0DDF810C00BFB08F0CBF549
:10479000FA7303FB0A020BFB09F003FB0C034FF453
:1047A000FA7192FBF1F293FBF1F308E0D97809B1C9
:1047B000022E02D14B46424601E0049B5246234959
:1047C000DFF8A4B0695A16F80BC008B20CFB00FB66
:1047D0006FF04F0C9BFBFCFC94441D4ACDF800C0CD
:1047E00035F902C0A952CCEB00001A4ADFF87CC0B0
:1047F000019054F80C10A0584018019902904018EC
:10480000A15844F80C100199A150134A0434B15C2A
:10481000202201FB00F090FBF2F1581A009B0F4997
:10482000C21801366A520235032E7FF42FAF09B049
:10483000BDE8F08FDA160020B3160020FA0D002034
:10484000800B0020F0D8FFFF80C1FFFF600B00202D
:10485000100B0020180B00208B1500208215002063
:10486000240B0020040B00208E150020F80A0020E5
:104870002DE9F04F002485B0039305468946924602
:1048800006462346474AD17809B91079B8B1022CB7
:1048900017D0454B454F33F9140037F91420CAF1AE
:1048A000000102EB40005246FEF740FA4049039FE8
:1048B00031F9143037F91420C01A83180AE0022C99
:1048C00008D1394A99F80570B2F904101B374F43E3
:1048D000791114E03348C17871B9334F99F8042045
:1048E00037F914101B324A430079111138B16A7C30
:1048F0005A4301EB222102E0EF795F4339112D4F3A
:10490000DFF8C4C037F91400BCF800200F1A295D85
:104910007A437943DFF8B480D0124FEAE11B58F8AC
:104920002420B17A01FB0020234948F824004FF4E9
:1049300000120293CDF804C0FEF7F8F91F4BDDF822
:1049400004C053F8241043F82470791ABCF800709E
:104950004FF6FF723B09B2FBF3F74F43184BDFF8FA
:1049600070C048F824005CF8241053F82480BF116C
:1049700008EB010243F82470337DD11959430BEB46
:104980006030104A00EB21214CF8248022F81410EA
:1049900001340136032C029B7FF474AF05B0BDE8EF
:1049A000F08F00BFB3160020DA160020FA0D0020A9
:1049B000800B0020600B00200000E0FFEC0A0020CC
:1049C0002C0B002082150020560A0020040B00202A
:1049D000380B0020024B5A780AB1002058707047FB
:1049E000B31600200023038043807047024B00224F
:1049F0001A605A60704700BF240B0020024B00224F
:104A00001A605A609A607047040B00200128034B1B
:104A100014BF034A034A1A60704700BF44000020D5
:104A200055460008714800082DE9F84F384E0446F5
:104A30003768384606F08AF80546384606F0FAF830
:104A400076688046304606F081F88346304606F0A8
:104A5000F1F8D4F80490064629464846FCF7AAF82F
:104A6000A768824641463846FCF7A4F801465046FE
:104A7000FBF796FF216882465846FCF79BF84146B3
:104A800004464846FCF796F83146FCF793F8014691
:104A90002046FBF787FF314604463846FCF78AF884
:104AA0002946FCF787F801462046FBF77BFF0146C5
:104AB000504606F04BF91749FCF77CF8FBF7B6FCBB
:104AC00011A3D3E90023FBF72FFE134B044618680C
:104AD0000D46FBF7ABFC02460B4620462946FBF78A
:104AE00047FB00220D4BFBF71FFEFBF705FF06F00F
:104AF00061F881B20A0444BF00F5B47189B208B20A
:104B0000BDE8F88FAFF30080182D4454FB21094015
:104B1000580B00200000E144940B002000002440CA
:104B200010B5194C2088FBF7F1FF1849FCF742F843
:104B300006F040F8164B18802088FBF7E7FF014687
:104B40001448FCF7EBF81449FCF7E8F8134908603F
:104B50001348B0F87400FBF7D9FF01461148FCF781
:104B6000DDF8FBF763FC06A3D3E90023FBF7B2FCF7
:104B7000FBF7C2FE0C4A106010BD00BFAFF300800F
:104B80003B597E90A9E7814042000020C903683F5D
:104B9000540B00200AE81C4100401C46A8150020C8
:104BA0007814002000006144C4150020AFF3008099
:104BB0002DE9F041044600680D460146FBF7FAFF77
:104BC000D4F80480064641464046FBF7F3FF014611
:104BD0003046FBF7E7FEA768064639463846FBF73E
:104BE000E9FF01463046FBF7DDFE06F0B1F8002193
:104BF0000646FCF773F970B920683146FCF78EF869
:104C0000314628606068FCF789F831466860A06822
:104C1000FCF784F8A860BDE8F0812DE9F04F0C683E
:104C2000836889B0D0F800A0D0F8048006462046FA
:104C300003938B4605F08AFF0746204605F0FAFFEE
:104C4000DBF804408146204605F080FF05462046FB
:104C500005F0F0FFDBF8082004461046019205F04D
:104C600075FF8346019805F0E5FF394602905846E6
:104C7000FBF7A0FF394604900298FBF79BFF5946CB
:104C800005904846FBF796FF029906904846FBF7C9
:104C900091FF294607905846FBF78CFF0146504686
:104CA000FBF788FF214683460698FBF783FF014602
:104CB0000598FBF777FE01464046FBF77BFF014670
:104CC0005846FBF76FFE214683460498FBF772FFB8
:104CD00001460798FBF764FE01460398FBF76AFF5D
:104CE00001465846FBF75EFE3060029905F1004030
:104CF000FBF760FF01465046FBF75CFF2146834609
:104D00000798FBF757FF01460498FBF749FE014659
:104D10004046FBF74FFF01465846FBF743FE21464E
:104D200083460598FBF746FF01460698FBF73AFED7
:104D300001460398FBF73EFF01465846FBF732FE5B
:104D4000214670605046FBF735FF2946044609F1BD
:104D50000040FBF72FFF01464046FBF72BFF0146C3
:104D60002046FBF71FFE394604462846FBF722FF84
:104D700001460398FBF71EFF01462046FBF712FE93
:104D8000B06009B0BDE8F08F80EAE073A3EBE07398
:104D90008B4206DB002801DD401A704702D0401824
:104DA00070470020704700002DE9F041524B86B05B
:104DB0001A685B6802F1004203F1004301934F4B14
:104DC0000646B3F900000092FBF7A0FE00F1004098
:104DD000FBF72CFB46A3D3E90023FBF77BFBFBF798
:104DE0008BFD474C0290B4F90000FBF78FFE039057
:104DF000B4F90200FBF78AFE0490B4F90400FBF753
:104E000085FE6946059003A8FFF707FF3D4B93F821
:104E10004430012B16D13C48417869B93B4C4025C0
:104E2000226892FBF5F7D01BFBF770FE0599FBF7A4
:104E3000B9FDFCF785F82060344B4021186890FBE1
:104E4000F1F001E0324B1888FBF760FE014605984F
:104E5000FBF7A6FD05903046FBF754FE2D490746AB
:104E6000FBF7A0FD01463846FBF758FF2A4D0746E1
:104E70002C6805982146FBF793FD01463846FBF761
:104E800099FE01462046FBF78DFD244C28601D4D00
:104E900007460398D4F8008005F08CFE95F8301092
:104EA000FFF772FF08EB000204982260D4F8048038
:104EB00005F080FE95F83010FFF766FF08EB000361
:104EC00038466360D4F8088005F074FE95F82F101A
:104ED000FFF75AFF1249134B0A684044A060186854
:104EE000B6180E60411C196006B0BDE8F08100BF25
:104EF000399D52A246DF913F580B002092150020A9
:104F0000BC15002078140020B3160020980B002058
:104F1000420000203661823C900B00209C1500204E
:104F2000700B0020880B00202DE9F04F87B0FFF7B1
:104F3000C7F9022002F036F8002800F0AD81AE4833
:104F4000FFF778F9FFF786FAAC4C05462768C71BD0
:104F50003846FBF7D7FDAA49C968FBF72BFE834605
:104F6000A848256090F82E8000252C462E46A64A9B
:104F7000105FFBF7CBFD5946FBF71CFE03AB585106
:104F8000B8F1000F27D04046FBF7C0FD01464FF0B7
:104F90007E50FBF7C3FEDFF8B092824651464FF0D9
:104FA0007E50FBF7FDFC55F80910FBF703FE97490F
:104FB0000346085F0193FBF7A9FD5146FBF7FAFD95
:104FC00001460198FBF7EEFC49F80500FBF7B8FF36
:104FD0008F4A105303E08D498D4A605AA0528C4B82
:104FE0000435E15E0234062C01FB0166BFD1894A1B
:104FF0006420138846435B43874803A996FBF3F676
:10500000FFF70BFE082001F0CDFF20B1834803A974
:10501000FFF703FE07E0824803A9FFF7FEFD804883
:105020000146FFF7C5FD493E7E49B4B23B2CB1F8BD
:10503000F00007D97B4E0820B6F8F25001F0B2FF1D
:1050400030BB4FE0FBF75EFD4FF07E518046FBF733
:10505000A9FC01464FF07E50FBF760FE0024064697
:105060006D4D404655F81410FBF7A4FD8146684885
:10507000005FFBF74BFD01464846FBF793FC3146CA
:10508000FBF798FD45F814000234062CE8D1D1E76F
:10509000B6F8F200FBF736FD80462846FBF732FDF6
:1050A0004FF07E51FBF77EFC01464FF07E50FBF740
:1050B00035FE00240646594D404655F81410FBF7BE
:1050C00079FD594A8146105FFBF720FD01464846AD
:1050D000FBF768FC3146FBF76DFD45F81400023420
:1050E000062CE8D1514B4C4DB3F90000FBF70EFDF7
:1050F000AC68014620460126FBF718FF00B90646BA
:105100004B4968684E73214605F020FE494CD5F89E
:1051100008802060286800F1004668680146FBF7B7
:1051200049FD414605464046FBF744FD01462846F9
:10513000FBF738FC05F00CFE0146304605F006FE94
:1051400060602068FBF772F929A3D3E90023FBF71D
:10515000C1F9FBF7D1FB05F02DFD374D28806068C4
:10516000FBF764F922A3D3E90023FBF7B3F9FBF7BC
:10517000C3FB05F01FFD6880082001F013FF2F4CD2
:1051800008B1264800E02648FFF74EFC1D4D208060
:105190003846FFF709FE95F87620002A00F0808057
:1051A0001D4B18689C6801465F68FBF703FD394694
:1051B00006463846FBF7FEFC01463046FBF7F2FB9D
:1051C000214606462046FBF7F5FC01463046FBF734
:1051D000E9FB05F0BDFD01462046FBF79FFD1849A0
:1051E0000446FBF78FFE88B316480021018057E084
:1051F0003B597E90A9E78140A2140020840B002037
:10520000701500207814002094150020AC150020A3
:10521000BC15002042000020C8150020480B0020CB
:1052200048000020D010002068150020540B0020FA
:10523000B3160020580B0020800B00209215002090
:105240008FC2753C8C0B0020740B0020204605F0AB
:105250002DFD274B1968FBF7ADFC05F0ABFCB0F555
:10526000617FA8BF4FF46170FBF7CEF81EA3D3E9AE
:105270000023FBF759FAFBF73FFB05F0DBFC044684
:1052800095F87600FBF742FC2146FBF793FC05F00E
:1052900091FC184B188003E0174B188058809880B9
:1052A000164A5379012B164B07D0164819885A888D
:1052B0009B8801804280838011E01349B3F9042068
:1052C000B1F9000002EB4000032290FBF2F080B243
:1052D0000C4A088019885B8890801180538007B041
:1052E000BDE8F08FAFF30080A2EB0FE5DD1696402E
:1052F000C41500208C0B0020AC150020D01000201D
:1053000094150020600B0020440B0020AFF30080B8
:1053100010B5054C00202188FCF7D2F961880120E6
:10532000BDE81040FCF7CCB95400002010B5094C82
:10533000206009480160094909480A60094A0A4988
:105340001360029B039A03600848049B0A60036091
:1053500010BD00BFEC150020E4150020D81500207A
:10536000D4150020DC150020E8150020E0150020F1
:10537000094B1A6802EBC001CB79FF2B04D01BB19B
:10538000064830F8130004E00728D4BF888840F2AC
:10539000DC5000B2704700BFEC1500200A17002057
:1053A000054B1A6802EBC00090F9063019420CBF99
:1053B00001204FF0FF307047EC15002010B500249D
:1053C0004FF48040FDF70AFB08B1054B00E0054BA8
:1053D0001868054A8188A1520234182CF0D110BDFA
:1053E000E4150020D815002008160020F8B53A4B27
:1053F0003A4E0546187006EBC0000F46384C41780F
:1054000020202160FDF7EAFA08B101222260162D62
:1054100019D1002438590021FBF760FD28B14FF461
:105420008040FDF7DBFA50BB25E02E4A3B191619E8
:105430000FCB86E80F002C48103401784A1CC02C92
:105440000270E7D1EBE716F8357006EBC506264B80
:10545000D6F804E01F70BEF1000FE0D00024BC427B
:10546000DDDA204E200136180EEB00010FC90134A1
:1054700086E80F00F3E7082D1C4B23D124E01A4FD8
:105480003F78012FF7D91A4C00261034BE42F2DAC9
:1054900054F8100C4FF07C51FBF78CFB4FF07C5113
:1054A00044F8100C54F8140CFBF784FB4FF07C51BB
:1054B00044F8140C54F80C0CFBF77CFB013644F850
:1054C0000C0CE2E70E2D01D1012000E00020187441
:1054D000BDE8F840FFF772BF9C0B0020A4DE000877
:1054E000A00B0020A80B00209D0B0020B31600206D
:1054F000B00B0020F0B58C46461C002300224CF86F
:1055000003201033C02BF9D10A4800EBC6014F68C5
:1055100007B9F0BD0024074B13F83620944208DA8F
:1055200020010CEB000539180FC9013485E80F0084
:10553000F1E7F0BDA4DE0008284B10B5186800287C
:105540004AD027490A78531E142B3DD8DFE803F0D0
:105550000B3C3C24403C3C1C3C3C3C3C3C2C3C3C00
:105560003C3C3C242C001F4801684A7832B11E495B
:1055700000204989BDE81040FCF7A2B81B4B5878C1
:105580000028F4D10146F5E7174C0020E188FCF72C
:1055900097F801202189EDE7134C00202189FCF7C1
:1055A0008FF801206189E5E70F4C0020E188FCF7C6
:1055B00087F801202189FCF783F802206189FCF734
:1055C0007FF80320A189D5E72020FDF707FA18B15D
:1055D000BDE81040FFF79CBE10BD00BFA00B00202F
:1055E0009C0B0020DC15002054000020B316002086
:1055F00010B50024064B1878A04208D9054920466A
:1056000031F814100134FCF74DF8E4B2F2E710BDA4
:105610009D0B0020F0150020064B1A780023D9B20C
:10562000914204D2044921F813000133F7E7FFF750
:10563000DFBF00BF9D0B0020F01500202DE9F74FC4
:10564000A34B187803280FD9A249A34CB1F9042021
:105650006FF06305002AB8BF5242A91AB4F90400DA
:105660006432FDF763FBA080994A1678012E1DD89D
:105670009A4E3478651E9A4C142D00F2C981DFE8E9
:1056800015F0A400C701C7017B00B300C701C70123
:105690005A01C701C701C701C701C701D000C7012F
:1056A000C701C701C701C7015F00A1018D488A4B2F
:1056B000884F0168B7F806B0B3F800805F88B3F987
:1056C00004A0894C019100251034B542D0D20FFAC4
:1056D0008BF0FBF71BFA54F8101CFBF76BFA8146B2
:1056E00038B2FBF713FA54F8081CFBF763FA0146CB
:1056F0004846FBF757F981460FFA88F0FBF706FAA0
:1057000054F80C1CFBF756FA01464846FBF74AF9D9
:10571000019A814692F9000041420AFB01F0FBF731
:10572000F5F954F8041CFBF745FA01464846FBF727
:1057300039F9FBF705FC6D4B23F815000135C3E77C
:1057400001210420FFF72CFE634D654C6E887043E9
:1057500087B204202781FFF70BFE38182081012132
:105760000520FFF71DFE2B88584385B20520658173
:10577000FFF7FEFD2B1826E002210420FFF710FEA4
:10578000554C0121A688704387B20420FFF708FE1C
:105790006588534C00FB0572042097B2FFF7E8FDC3
:1057A0003818208102210520FFF7FAFD70430121FE
:1057B00086B20520FFF7F4FD00FB056105208DB2E0
:1057C000FFF7D6FD2B18638122E101210520FFF7A9
:1057D000E7FD414A424E9788784384B20520FFF79F
:1057E000C7FD2018708113E1414900200D68FFF7C3
:1057F000BFFD404F95F90630B7F90260734332267A
:1058000093FBF6F2801820800120FFF7B1FD95F997
:105810000E10B7F90050694391FBF6F3C718678083
:10582000F6E03549354E4A78376812B9B888E081D4
:1058300008E0284C3988B4F906007A88FDF776FA32
:10584000274BD881264D2E4FE989284A3E68118082
:10585000347854B3264D0220FFF78AFD2B68B3F944
:105860001010B3F91220FDF761FA2649264B0A6899
:10587000198854890EB2201A02B2964203DA3E68A1
:105880003278511803E003DD3F683878091A19802F
:105890002D681D4F95F91630B7F900006421434378
:1058A0000F4A93FBF1F6A4199480134D0C4BAF7A79
:1058B00067B1084801880E4AD9801981868817681F
:1058C0005E814488064D9C8103241FE00248F1E775
:1058D0009D0B0020DA160020821500209C0B002072
:1058E00054000020DC150020A80B0020F01500203B
:1058F000EC150020800B0020B3160020D8150020E6
:10590000D4150020E8150020A40B002007EBC403E9
:1059100093F90600B5F906106426414391FBF6F6AB
:10592000EE802046FFF724FD01343218EA8002356C
:10593000072CEBD16CE0A54FA54B78781E6810B909
:10594000B588E58108E0A3497288B1F9060031887D
:10595000FDF7ECF9A04AD0819F4C9C4B9F48E7890A
:105960009E7A0780012103201EB1FFF719FD994D92
:1059700002E0FFF715FD9A4D6E880221704387B251
:105980000320FFF70DFD2D8800FB05710420E18049
:105990000121FFF705FD7043022186B20420FFF7C5
:1059A000FFFC00FB056203202281FFF7E1FC8A4C2B
:1059B000E388C018E0800420FFF7DAFC2789C519C6
:1059C000258125E0864A0324978802212046FFF797
:1059D000E7FC7843012186B22046FFF7E1FC804DC9
:1059E000C4F10603590835F811207B4D00FB026015
:1059F00086B225F814602046FFF7BAFC331825F864
:105A000014300134072CE0D1724F744AF9881180A8
:105A10002020FCF7E3FF002845D00020FFF7A8FC7A
:105A20006D4F054638800120FFF7A2FC6D49788054
:105A30000B7A002B37D06C4A6C4B14686C4A267872
:105A400006F00201CCB2D4B11468B3F9001094F995
:105A50000E2094F906404A43322192FBF1F6B3F945
:105A60000230B2B2664273436FF0310493FBF4F636
:105A70009419651993FBF1F13D80561811E01168F6
:105A8000B3F9026091F906403222664396FBF2F4C4
:105A90002D193D8091F90E10B3F900304B4393FB63
:105AA000F2F6801978800026514F4B4D3B68A85F75
:105AB00003EB860233F92610B2F90220FDF736F91E
:105AC000A8530236102EEFD1474C2168087800F019
:105AD0000407FBB22BB9414A464C168827780123AC
:105AE0001CE0454D2E780E2E0AD0082E08D0434AD1
:105AF00002EBC6046178002914BF0225002500E0EE
:105B0000042500263E4F701907EB4603C0B21989E1
:105B10000136FBF7D5FD042EF4D1DCE7BB4209D2F8
:105B20002E4C36B234F913100133B142A8BF0E46E1
:105B3000B6B2F3E7002427462E490878874272D28E
:105B4000234D31B22B685A88914204DD2348951BBE
:105B5000235AEA1822524FF48040FCF73FFF1F4DB2
:105B6000C0B1284A264B1068B3F906104389184A79
:105B70009942254905DD09681268285F49885288DD
:105B800004E012680B68285F91881A88FDF7CEF848
:105B900028533EE0DFF83880285FD8F8003005EB66
:105BA000040919885A88FDF7C1F8164A1449136880
:105BB0002853B1F90600998988422ADA1020FCF7A7
:105BC0000DFFD8F8002008BB108820E0B316002095
:105BD000D8150020DA16002054000020F01500200F
:105BE00082150020C4160020E0150020800B002044
:105BF000EC1500209D0B00209C0B0020A4DE00086B
:105C00000A170020E8150020E41500209088A9F864
:105C10000000064843781BB905490648625A2252DB
:105C20000137023488E7BDE8FE8F00BFB3160020BD
:105C300008160020F0150020024B1868003018BF2D
:105C400001207047A00B002044F25063984203DD0E
:105C5000A0F50C40A038704703498842BCBF00F54E
:105C60000C40A030704700BFB0B9FFFF10B5FAF785
:105C70004DFF00210446FBF759F908B1204601E029
:105C800004F100400549FBF749F80549FAF792FF8E
:105C900004F05CFF034B186010BD00BF8096184BEA
:105CA00035FA8E3C6400002010B5044C00232070AF
:105CB0002361FEF7E9FB606110BD00BF48160020BC
:105CC000F8B51D4614460E46FAF720FF6968FAF744
:105CD00071FF3146FAF76EFF2168FAF763FE206024
:105CE000FBF72EF9ED68074605F10040FBF728F9B0
:105CF00006462846FBF724F9314602463846FDF7AA
:105D000015F8FAF703FF2060FBF71AF9F8BD000059
:105D1000F8B5101A0C461F46FAF7F8FE0546381B70
:105D2000FAF7F4FE174B079E1968FAF743FF294666
:105D300004462846FAF73EFF214607462046FAF772
:105D400039FF01463846FAF72DFE05F001F80E49F5
:105D5000FAF730FFFBF71AF906990860214605F1BA
:105D6000004004F0F3FF0949FAF724FF0849FAF765
:105D700019FEFBF7E5F80028BCBF00F50C40A03089
:105D80003060F8BD640000202C7D8E3FA00CB34530
:105D900000A00C4610B50446002003460D49CA5C1D
:105DA000A2B12E2A04D1013394B1C91800220A5598
:105DB000084A0A21D25C4843A2F13001092901D8DE
:105DC000303880180E2B02D80133E7E710BD0020D1
:105DD00010BD00BF980E00202DE9F843224B074666
:105DE00048681D68381A0C469146FAF78FFE294616
:105DF000FAF794FF1D4920610A6880469078FAF707
:105E000081FEFAF713FB16A3D3E90023FAF762FB2E
:105E100002460B4600201649FAF786FCFAF76CFD9D
:105E20002946FAF7BFFD01462846FAF777FFA6682C
:105E3000054631464046FAF7B3FD01462846FAF7D3
:105E4000B9FE01463046FAF7ADFDD9F808102061D9
:105E50006760A060FAF7AEFEFBF772F8BDE8F88362
:105E6000182D4454FB211940200E002064160020F8
:105E70000000F03FAFF30080014B1860704700BF97
:105E800064160020F8B52D4B187810B1012850D1B8
:105E90000AE02B4B2B4A58782B4B02EB0011496838
:105EA0005868FEF7BFFA41E0274D6868FEF7BFFA71
:105EB00000283ED0224C2178264601291ED1FEF72B
:105EC000E3FA06466069321A632A35D92169042942
:105ED00012D81C4F686807EB01135968FEF7A2FA45
:105EE000607807EB0017B9686868FEF786FA2269E0
:105EF0006661511C21611CE0022018E022693AB958
:105F00006478104B686803EB04114968FEF78AFA5D
:105F100033690B4C8B2B09D80C4A0B48D15C406879
:105F2000FEF766FA21694B1C236102E00320FFF7AC
:105F3000BBFE034A00205060F8BD00BFF80D0020F2
:105F400048160020C4E300084417002036E3000888
:105F500010B50B4CE37A8BB10A48017804290DD9AE
:105F6000094A0A4B1068516818605960FFF77EFEB5
:105F70000748084B028801211A80217310BD00BF19
:105F8000B3160020A0160020881600206C160020F2
:105F900092150020EA0D0020002370B51C460F4822
:105FA00000211952142060430D4A0E4E0E4D995295
:105FB00000223250595335180C4E6960AA60325095
:105FC00035180B4E01346960AA6002333518022C73
:105FD00032506960AA60E2D170BD00BF3416002063
:105FE000FA0D0020E40C00203A160020940C00204A
:105FF000340E002070B504460079FAF783FD1E497F
:10600000FAF78CFE1D4D1E4E2860A07BFAF77AFD34
:106010001949FAF783FEEE6068606079FAF772FD5D
:106020001849FAF77BFE184D2860E07BFAF76AFD05
:106030001149FAF773FE6860607EFAF763FD134951
:10604000FAF76CFEEE60A860A079FAF75BFD0D49E7
:10605000FAF764FE0E4D2860207CFAF753FD0649DE
:10606000FAF75CFE6860A07EFAF74CFD0749FAF784
:1060700055FEEE60A86070BD0000C842D40D00203F
:106080000000FA4400002041100E002000007A4475
:10609000D40C00202DE9F041134C9846134E144BBC
:1060A0000546002031701A60FFF7FEFD6570FEF7AF
:1060B000EBF9A060307800276760B8420CBF01247C
:1060C00003244046FFF796FF0A49234601EB0515D6
:1060D0006A6839460848FBF783FE084A5060012089
:1060E000BDE8F041FFF7E0BD48160020F80D0020A4
:1060F00064160020C4E30008004400404417002058
:10610000F8B51B4B187803282ED11A494FF480524A
:106110004FF40044A1F500650A612C61164C6068DB
:10612000FEF776F960B1134D4FF480566E616068EA
:106130002768FEF772F901463846FEF759F92E61D5
:106140000D4C2068FEF764F90028E7D00B4D4FF4A2
:10615000004694E881006E61FEF75FF9014638461B
:10616000FEF746F92E61D9E74FF0FF30F8BD00BFCA
:10617000481600200010014044170020000801408C
:10618000F7B50368164C174D23600968164E616019
:106190000068FFF76BFD94E80C001448019600902E
:1061A00095E80300FFF7B4FD6B68114A6168366833
:1061B000C81A1660FAF7AAFC0E4A0F4F1168FAF7D0
:1061C000F9FCFAF7BDFE2968786020680B4A431A8B
:1061D0000B483B60016816600A4BCA881A80FEBDF6
:1061E000F00D0020881600205C0E0020000E00201C
:1061F000EC0D0020640000208C0E00206C0E0020AE
:10620000641600207E0E0020264BF0B51D68024665
:1062100000F1100116781446AB195B78013203F0D7
:106220000403DBB263B18A42F4D10020F0BD13B1A4
:106230000A225343DBB210F8011B30395B18DBB282
:10624000211A0229F3DC0021844209D911B10A2262
:106250005143C9B210F8012B303A8918C9B2F3E79B
:106260002E2E11D10134042000220A2672432678F2
:10627000AF197F7807F00407FFB217B1303A9219CF
:1062800001340138F1D100E00022074C6420614361
:1062900000FB021106240548B1FBF4F200FB0320C9
:1062A000F0BD00BFA401002040420F00809698007E
:1062B0002DE9F04F9A4B8BB05868B8B9994C2178BA
:1062C0004A1E032A00F26185DFE812F0F304F304AA
:1062D0003E0528056068FEF7A0F8934904460B7850
:1062E000012B00F0DF8008D3022B06D08C4C6068B5
:1062F000FEF78EF80028EDD1E0E7242C07D18B4B78
:106300008B4A8C4C0021197011702170C5E02C2C27
:1063100002D02A2C40F08280854D844A2978864B11
:10632000157800205854854AB5B918781570472853
:1063300068D15978502965D19878472840F013855D
:10634000D978472940F00F851B79412B40F00B8508
:106350000120107000F007BD117801293AD1022DFB
:1063600005D11846FFF750FF754908604AE0032D34
:1063700007D11978532945D1714802685342036007
:1063800040E0042D05D11846FFF73EFF6C4B5860E6
:1063900038E0052D07D11B78572B33D168494A685F
:1063A000504248602EE0062D07D119786548302903
:1063B00094BF00210121C17224E0072D04D1FFF711
:1063C000E9FC614A10701DE0092D1BD1FFF7E2FCCA
:1063D0005E4B16E0022915D1072D0CD10120FFF7E5
:1063E000D9FC41F2184250434FF47A71584BB0FB3C
:1063F000F1F0188006E0082D04D10120FFF7CAFC57
:10640000544B1880494B4A49013500202A2C1D70F5
:10641000087039D15048012404703EE00D2C4E4ADA
:1064200001D00A2C26D11478FCB1434C2178647831
:10643000A1F13000C3B2092B84BFA1F13703DBB255
:10644000A4F1300003F00F02C3B21101092B84BF85
:10645000A4F13703DBB2374C03F00F028918207820
:10646000CBB2C21A514251EB02043B4B00201870D0
:106470007CB912E02E490B780E2B03D82E48C45459
:1064800001330B70127842B92A4B1A7854401C70B1
:1064900003E02A4A1078012800D00020C00700F14C
:1064A000338123E72D4B0022197808293FF61EAFD0
:1064B000DFE801F00A05111927607C96A000622828
:1064C00001D1022105E01A70B52C7FF40FAF1C78C2
:1064D000611C19700AE72249224A03261E700870BF
:1064E0001070214B0BE01F4E0421197032781E4BA7
:1064F000A1181878CAB2101818701C4B32701C7092
:10650000F4E605211970174B174E1A783078A11848
:10651000CAB210183070164E1A703480E6E600BF0A
:106520004417002048160020F80D0020D30C00204E
:10653000E40D00206A0E0020980E0020720E00204C
:1065400088160020B3160020A01600203216002066
:106550003E160020680E0020D20C0020300E0020D5
:10656000700E0020E50D0020E60D0020910C0020AB
:10657000E80D00206C4906261E700A786B4BA618A1
:106580001878F2B210181870694B0A70198801EB6C
:106590000424A6B2B6F5007F01D81E8003E00022D5
:1065A0001A80644B1A70002463497FE35E495F4E92
:1065B0000A783078A318DAB2101830705E4E0A707C
:1065C00033885B4AC72B98BF5C49108898BFCC546E
:1065D0005C1CA1B2884231807FF488AE072107E0BD
:1065E000514808261E700378A3423FF47FAE002175
:1065F000504B6EE74D4E1A70337883427FF476AE7F
:106600004F4C207806283BD005D8022813D0032809
:106610007FF46CAE23E0122847D030287FF466AEBA
:10662000464A484C1679454A102E88BF10262670D7
:106630002178002347E0414C434E6368A0682169FC
:106640007360424B4FF47A723060414C91FBF2F62A
:10665000187840492680C87201223F4923E0374913
:106660004A7912F0010004D00E79F41E634253EB14
:10667000040036490870002839D1364AD07236E015
:106680002E4EF47A14F0010104D0B07AC21E5342A7
:1066900053EB02012D4E317009B92E4CE17227489F
:1066A0002E4990F82F200A7021E024482C49866951
:1066B000426942F210742B4B96FBF4F00A8018806A
:1066C00001222949EFE70C328B4210DA12F8046CF0
:1066D000264812F8034C1E54254E26489C5512F8A5
:1066E000014C16781C54244C1E550133EBE71A4913
:1066F0000A78002A3FF4FAAD1B4B1E78002E3FF4B7
:10670000F5AD00240C701C701C4CA068E060FDF717
:10671000BBFEA060202000F04FFC19490A78012A36
:1067200030D100232FE000BFE50D0020E60D002052
:10673000E80D0020300E0020960E00200C0D0020E9
:10674000910C0020A1160020881600207C0E00204D
:1067500032160020B3160020E70D0020A0160020FE
:106760003E160020680E0020710E00202116002029
:106770007616002090160020A21600204816002051
:10678000880E002001237E4C0B70E07A00283FF435
:10679000ADAD7C490A78042A7FF6A8AD677807B9C1
:1067A0002773257B15B90FB1FFF7D2FB764E052174
:1067B0003378764F5C1C94FBF1F001FB1042327091
:1067C000734E97F800C0734D06EB82020023724CA3
:1067D00072491F59DFF810E27148724E5F5097FB03
:1067E000FEF1195006FB0170DFF8009203EB040A7A
:1067F00042F2107490FBF4F71668BCB253F80970BB
:106800001060C6EB07084044052643F8090090FBDA
:10681000F6F00EFB01016448BCF1010F25F8024FB0
:10682000195005D1023CB4F5797F98BFCAF8001021
:1068300004331432082BCAD1FDF726FE5B4D5C4CA5
:106840002A68801AFAF75EF95A49FAF767FA20605F
:10685000FDF71AFE286025684FF07E512846FAF7AA
:1068600047FB08B94FF07E55256006A907AC4A489A
:10687000514B0194009103C80CCBFFF749FA069ADB
:1068800064234E49B2FBF3F00880079A3C4892FB20
:10689000F3F34B4C027B23800AB90A8022804949DA
:1068A0000C78002C36D0424F4FF07E503968FAF702
:1068B00035FA454D384E2B6804463068C01AFAF751
:1068C00025F92146FAF776F9FAF73AFB7268696812
:1068D0003E4D0746501AFAF719F92968FAF76AF98E
:1068E0002146FAF767F9FAF72BFB04B2384802257C
:1068F000B0F902303FB2E21892FBF5F1B0F9002096
:106900008BB2B918334C91FBF5F291B263802180C0
:10691000438001802B4B01201F4C1870184B61687D
:10692000294A20681C7A516010601CB9DA79002A63
:106930003FF4DCAC284E294D294C01960095164FAA
:1069400094E80C00FFF7E4F961687868254E081AAE
:10695000FAF7DCF81D4B1968FAF72CF9FAF7F0FA98
:1069600070600A48226890F900303C68012BC4EB43
:10697000020131603CD0022B7FF4B8AC9FE000BF35
:10698000B3160020A0160020940E0020900C0020CA
:10699000680C0020020E002088160020740E0020D3
:1069A000240E0020806967FFC00C0020C80C002066
:1069B000200E002000007A446C160020681600208B
:1069C00074160020080E0020800E002064000020B5
:1069D000CE0C00202C0E00205C0E0020000E0020AB
:1069E000F00D00208C0E002080969800600E002094
:1069F000002634463546DFF818C3AF4F5CF825B0A3
:106A0000CDF80CC05846FAF781F83968FAF7D2F891
:106A1000FAF796FADFF8DC92A84934F80920DFF893
:106A2000DC82801A83B21FB2635238460497A44FA7
:106A3000FAF76CF83968FAF7BDF8FAF781FA4FF00F
:106A4000140A0AFB058A82B29E4B049819680592C3
:106A50003B4658445246FFF733F90599DFF8B4B284
:106A6000DDF80CC00A1824F80B205CF8250051460C
:106A70003A46FFF7B1F994494FF4FA62FCF756F938
:106A800034F8093034F80B20313399B2622998BFB9
:106A90000020801883B224F80B308C4940F6B832BD
:106AA00018B2FCF743F958F80610894A01352BF85B
:106AB0000400B15002341436022D9CD116E4854FE7
:106AC0002D683E686C08B6F90820A24228BF22460D
:106AD000814C97B2268839B230B2814209DD794BB8
:106AE0007E491868FAF766F8FAF72AFA8719BFB2EA
:106AF00027807B4A7B4E14683168661A3046FFF760
:106B0000A3F80028D8BF404241F293139842CCBF6B
:106B10000020012050B33046F9F7F8FF7249FAF728
:106B200049F804F087F806462846F9F7EBFF0146D6
:106B30003046FAF73FF8FAF703FA6C4A63491080D7
:106B400000B240F6B832FCF7F1F8201848F6A0443D
:106B5000A04203DDA0F50C40A03804E00028BCBF33
:106B600000F50C40A0306249086001E0604D2C60E7
:106B70005F4B1D68C5F50C502830F9F7C7FF5A491F
:106B8000FAF718F8064603F0E1FF0990304604F0E2
:106B900051F8002508902C462E4638B2F9F7B6FF7A
:106BA00008AA52F82610FAF705F880465148DFF88F
:106BB0000C91005FF9F7AAFF01464046F9F7F0FE95
:106BC000FAF7BEF94FF47A7224F809004A4900B284
:106BD000FCF7ACF881B20BB2DFF83C8124F8091065
:106BE00018460493F9F792FFD8F80010F9F7E2FF7E
:106BF000FAF7A6F9DFF8D8A04FF0140B0BFB06ABA1
:106C0000049A30491FFA80FC0968434610465A46E8
:106C1000CDF80CC0FFF754F842460346594639F9FF
:106C200004000493FFF7D8F8049ADDF80C8080186C
:106C300008EB000CDFF8DC801FFA8CF124F8081058
:106C400008B240F6B8322149FCF770F855F80A202E
:106C50002A4B013628F80400EA5002341435022E7B
:106C60009BD11C480368197931B1214A642014680A
:106C7000234A94FBF0F11180224C1B882068984233
:106C80000ED91749174B0A681C68101BFEF7DCFF6A
:106C900042F210710028B8BF404288427FF726AB0D
:106CA000194B1A4A01201C88154910700C80FFF7F7
:106CB0001DBBFFF7E7F868E0D40D0020BC0C0020F6
:106CC000100E0020200E002030F8FFFF48F4FFFFD8
:106CD000340E0020641600207E0E00200000C84202
:106CE0005C0E00206C0E0020D3023739CC0C002043
:106CF000EC0D00202C0E002018FCFFFF940C00204F
:106D000080150020000E0020EA0D0020900C0020CD
:106D10008C0E00203A160020D40C002062686078A7
:106D2000531C411CCAB263600523B2FBF3F003FBA2
:106D300010216170FDF7A8FB154AA06015480023DB
:106D4000C372137001200BE0FDF79EFBA36840F6B1
:106D5000C411C01A884218D9202000F035F9042047
:106D6000FEF7A2FF11E00C498A78522A7FF44AAB61
:106D7000CB784D2B7FF446AB087943287FF442ABA8
:106D8000064A02211170FFF73DBB0BB0BDE8F08F42
:106D9000A0160020B3160020980E0020720E0020CE
:106DA0003D4B2DE9F047B3F90000F9F7AFFE3B4941
:106DB000F9F700FF044603F03DFF0646204603F0C6
:106DC000C5FEDFF8EC900546D9F80000344F90F886
:106DD0000380B8F1000F2BD0324CB7F90210B4F891
:106DE00002A00FFA8AF2881AFEF72EFFC8F10001FE
:106DF0004246FBF79BFFB4F8008000EB0A03B7F9AB
:106E000000000FFA88F7C01B6380FEF71DFFD9F85A
:106E10000010CA785142FBF789FF00EB080297B2D5
:106E20002780B4F90200F9F771FE804638B206E017
:106E3000B7F90200F9F76AFE8046B7F90000F9F7E2
:106E400065FE294607464046F9F7B4FE31468146BD
:106E50003846F9F7AFFE01464846F9F7A1FD124959
:106E6000F9F75CFFFAF76CF8104C31462080404689
:106E7000F9F7A0FE294606463846F9F79BFE01467B
:106E80003046F9F78FFD0849F9F748FFFAF758F847
:106E90006080BDE8F08700BF9215002035FA8E3C77
:106EA0003A1600203416002000002041FA0D002080
:106EB0006416002038B5254CE37A2246002B3ED0DC
:106EC0002348017804293AD92248817A79B1E179B5
:106ED000002939D12048214B012221721970011D4E
:106EE000E271FFF74DF91E490220087038BDC37AE0
:106EF000E171C3B11B4A1068408900F073F890B18A
:106F0000237A002B20D115481749037017480A68C7
:106F10004B680125011D026043602572FFF730F9BF
:106F20000F48057038BD0D48084B027800211972D2
:106F300052B901210170BDE83840FFF72DB8002398
:106F4000D3711372064A137038BD00BFB316002008
:106F5000A0160020C41600206C1600206800002037
:106F6000900C002064160020881600204016002097
:106F7000094B1A68811A00290DDB084A1178042987
:106F800009D900F5123000F5F8721A60044BD9687F
:106F900081F40040D86070470C0E0020A01600203D
:106FA00000080140034B196808420CBF0020012073
:106FB000704700BFA80E0020024B1A6810431860EB
:106FC000704700BFA80E0020024B1A6822EA00009A
:106FD00018607047A80E0020014B1868704700BF6A
:106FE000A80E0020094BB3F90020002AB8BF524276
:106FF000824209DAB3F902100029B8BF494281423E
:10700000ACBF00200120704700207047DA16002036
:1070100010B544780078002303FB03F1193961436C
:1070200001F6C4115943414340F6C41291FBF2F1F9
:10703000034A22F813100133072BEDD110BD00BF16
:10704000FA1600202DE9F04384780A276743C678B2
:10705000C4F1640C1A4D5FFA8CFCC6F1640800237D
:107060001A1B12B2002A04DCB8BF204602DB012042
:1070700000E0604602FB02F9404309FB06F999FB78
:10708000F0F0404442434FF00A0992FBF9F2B8187D
:1070900082B26A800888B1F8029012B2C0EB090986
:1070A00002FB09F20A334FF47A7992FBF9F29BB2B0
:1070B0008018782B25F8020FD2D1BDE8F08300BFED
:1070C000E0160020037A0A46042B14D8DFE803F008
:1070D0000303070B0F000849084B00F0C7BA064925
:1070E000064B00F01BB90449044B00F0E5B9024916
:1070F000024B00F0C3B8704708170020BC0E0020F8
:1071000038B504460D46002361890B4A9952023373
:10711000242BF9D10820FBF761FC28B12046294631
:10712000BDE83840FFF7CEBF0448054A2946BDE810
:10713000384000F0B1B800BF0A170020081700203F
:10714000BC0E0020037A042B0CD8DFE803F0030305
:107150000507090000F0C4BA00F00EB900F0CAB982
:1071600000F07AB8002070472DE9F8430746082060
:107170008846FBF733FC70B10024224A414613686D
:107180003846E2B29847204921F814000134082C0F
:10719000F3D1BDE8F8831D4A1D4D1378591CCCB2BC
:1071A00004F00306147005EB46090446064615482C
:1071B0004146036832463846984729F824002A8811
:1071C0006988AB885018EA88C118881803B2991CDE
:1071D000042291FBF2F00C4A0E4BA15EE052CB1E52
:1071E000984201DA811CA152135FD91C884201DD4B
:1071F000023810530136F6B202340835082ED6D1C3
:10720000BDE8F883BC0E00200A170020C00E002045
:10721000C20E0020AC0E0020F8B505460F46441EF5
:1072200014F8011F49B1054E304605F0EBFD00286A
:10723000F6D0861B631BBB55F2E7F8BD14E40008CB
:10724000014B33F8120070470A170020014B01224E
:107250001A707047020F002010B5064C207838B124
:10726000054B186801680A689047002323700120C5
:1072700010BD00BF020F0020C810002002490A60A4
:107280000BB1024A1A607047C81000204172000812
:10729000805CFAF717BA0000024B082113600170F6
:1072A000704700BF91720008825C044B53F82200C3
:1072B000410801F5777290B2704700BF0C0F0020B3
:1072C00038B50446FDF7C6F8104B40F6C4111A68ED
:1072D000821A8A421A460E4B01D9002119701B7876
:1072E00010600BB90F2C10D10A4800210170084A18
:1072F0004BB1094D182B1D4405F8014C03D1012356
:107300000370117038BD0133137038BD040F0020B5
:10731000080F0020090F00202C0F002038B54089ED
:107320001C460E4B0D461A60A0F577710C4A4B00B7
:10733000136053609360D360136153619361D361B1
:1073400008490948094A0523FAF74AFD0849C8606F
:107350000CB10848206008232B7038BDC8100020ED
:107360000C0F0020C172000800440040A0860100FC
:1073700044170020A972000870B5294D287800280C
:107380004CD0284CA67DC6F3C006002E44D1264B17
:10739000186801680A68904761782278234B01F0E9
:1073A000070042EA00221A60A2782E7002F03F0025
:1073B000400140EAD1015960E078810041EA921130
:1073C000227902F0010041EA80219960617901F09F
:1073D0000F00C00140EA5202DA60A27902F07F0099
:1073E000000140EA11111961E079410041EAD2122D
:1073F000217A01F0030042EA40225A61627A02F0E7
:107400001F00800140EA91019961A07AC10041EA20
:107410005212DA61012070BD0020287070BD00BFDB
:10742000090F00202C0F0020C81000200C0F002096
:10743000825C034B53F82200C0F3CF00704700BFBB
:10744000640F002010B50446FDF704F8154B1A68C8
:10745000811AB1F57A6F1A46134B01D900211970C0
:107460001060187820B9A82C1AD1104B187006E0BB
:10747000022802D10E4A147001E0142801D80D49E7
:107480000C540B490130C3B20878074A4100481D2B
:107490008342137004D100230449137001220A703F
:1074A00010BD00BF480F0020840F0020610F002096
:1074B000620F00204C0F002038B51C46084B0D46CB
:1074C0001A60084908484FF4E1320123FAF788FCB2
:1074D0000649C8600CB10648206008222A7038BDF1
:1074E000C8100020457400080044004044170020E4
:1074F00031740008154B10B51A780AB9002010BD78
:107500001349002018704B78012BF7D1114A1068ED
:1075100001680B68984710480278082A01D90821A9
:10752000017001780D4A0023D8B2023288420AD293
:1075300012F8010C12F8024C40EA0424084840F802
:1075400023400133F0E7012010BD00BF610F002090
:107550004C0F0020C8100020620F00204F0F0020A9
:10756000640F00201F4B2DE9F0431B7823B31E4C02
:107570001E4D277891F800C095F8008002231C4C1E
:1075800003F10109E65C46FA07F606F00F05EEB2D4
:1075900066450BD20B2E09D8E65C14F8094006EAC2
:1075A000080604EB0626134C44F825600233102B22
:1075B000E5D10C4B00241C700978914202D90E4B86
:1075C000197811B94089BDE8F0830C4B825C1978B9
:1075D000084B53F8220001B1400800F5777188B2DA
:1075E000BDE8F0838C0F0020850F0020C80F00201D
:1075F0002E170020980F0020950F0020960F0020D6
:10760000134B012210B51A700446FCF723FF114AF0
:107610000146106811600B1A0F4841F288318B4205
:1076200003600E4B01D900221A7018780C49E4B29D
:107630000F280C5408D10B4B0B491A680120087015
:1076400010680168884710BD044A431C137010BDC0
:10765000950F0020880F0020900F0020940F00202D
:107660002E170020C81000208C0F002010B51C46DB
:10767000134B1A60027A5AB1012A13D1114B03201D
:107680001870114B07201870104802700C2208E087
:107690000C4B022018700C4B032018700B48027022
:1076A00007220A700A490B484FF4E1320123FAF726
:1076B00097FB0949C8600CB1084B236010BD00BF9F
:1076C000C8100020850F0020C80F0020960F002052
:1076D000017600080044004044170020657500084A
:1076E000014B1878704700BF8C0F0020014B1860C9
:1076F000704700BF40170020034B18680178D1F194
:10770000010038BF0020704740170020034B186865
:1077100001784A1E534253EB020070474017002085
:1077200008B54FF40060FBF759F908B9002008BD0F
:107730004020FBF753F928B9074B186841784A1ED7
:10774000012AF3D9FFF7E2FF20B1034B1868417813
:107750000029EBD0012008BD40170020084B186815
:10776000427852B9817811B9064A507801E0064B47
:10777000187D003018BF012070470120704700BFFE
:1077800040170020B3160020C416002008B5FFF7EC
:10779000B3FF08B100F094F8FFF7B8FF18B1BDE8E7
:1077A000084000F04BBA08BD0D4B10B51878B0B1C9
:1077B000FFF7D4FF0B4904460A7882420FD050B13C
:1077C000FFF79AFF08B100F085F8FFF79FFF20B19F
:1077D00000F02CFA01E0FFF7D9FF024B1C7010BD3E
:1077E000CA0F0020C90F002010B50446FBF792FA1B
:1077F000084B10B11A6800215170186800234370BB
:107800002268A260FFF78CFF03490870BDE81040B2
:10781000FFF7CABF40170020CA0F002008B5094B68
:10782000187870B1FFF79AFF58B1FFF765FF08B1FC
:1078300000F068F8FFF76AFF18B1BDE8084000F0F3
:1078400005BA08BDCA0F002038B5064C05465E21B2
:10785000A068FCF7CDFDA0682946BDE83840FCF7DC
:10786000C7BD00BF44170020024B5E219868FCF79B
:10787000BFBD00BF4417002010B50A4C5E2801466A
:10788000A06805D15D21FCF7B3FDA0683E2105E0AD
:107890005D2903D1FCF7ACFDA0683D21BDE8104097
:1078A000FCF7A6BD4417002010B50446C0B2FFF790
:1078B000E3FFC4F30720BDE81040FFF7DDBF000081
:1078C000034B1868417809B900F092BA704700BFBD
:1078D00040170020044B1868417819B94FF416502E
:1078E00000F078BA704700BF4017002008B5044B7D
:1078F0009868FCF78DFDD0F1010038BF002008BD6D
:10790000441700202DE9F041FFF7F0FF002800F0B8
:107910004081FCF7B9FDA04B1A68811A7C2940F21E
:10792000388118609D480478651C0570002404F1B6
:107930002406F0B2FFF788FF994B33F91400F9F7EA
:10794000E5F8984A05461088F9F7E0F80146284618
:10795000F9F7E4F99449F9F72DF9F9F7F1FA013457
:1079600000B2FFF7A1FF032CE1D13020FFF76CFF3D
:107970008E49B1F90000FFF797FFFFF775FF8748C1
:10798000067816F0030629D1894D1020FFF75CFF19
:107990002B68642493FBF4F210B2FFF785FF2120DB
:1079A000FFF752FF296891FBF4F004FB101484EAFE
:1079B000E473A3EBE47318B2FFF776FF1420FFF72C
:1079C00043FF7C4AB2F90000FFF76EFF1C20FFF76F
:1079D0003BFF3046FFF768FFFFF746FF6F49087827
:1079E000430740F0B080744D0220FFF72DFFB5F93A
:1079F00000300A2593FBF5F0FFF756FF0220FAF757
:107A0000EDFF002847D06D4F6D4E3878347840F642
:107A10003401B4FBF0F26B4C4A4321882A2391FBDA
:107A2000F0F800FB1810B2FBF3F24FEA001399B222
:107A300041EA022C1FFA8CFEC2F303224EEA02082E
:107A40000620FFF701FF0FFA88F0FFF72DFF2088CF
:107A50003F78431C9AB292FBF7F107FB112036786E
:107A600020806E247443152394FBF3F43A2064279A
:107A7000FFF7EAFEB4FBF7F63046FFF715FF3B20B1
:107A8000FFF7E2FE07FB164291B24C1D94FBF5F0A6
:107A900000B2FFF709FF2020FFF784FA002850D03A
:107AA000494C1320FFF7D0FE2568484F002DB8BF82
:107AB0006D4295FBF7F630B2FFF7F6FE1B20FFF79D
:107AC000C3FE23680A26002BB8BF5B4293FBF6F186
:107AD00042F2107591FBF5F205FB121000B2FFF7B0
:107AE000E3FE2320FFF7B0FE2368002BACBF4E203F
:107AF0005320FFF7D9FE1220FFF7A6FE6168002988
:107B0000B8BF494291FBF7F210B2FFF7CDFE1A2041
:107B1000FFF79AFE60680028B8BF404290FBF6F677
:107B200096FBF5F305FB136108B2FFF7BDFE2220BB
:107B3000FFF78AFE6268002AACBF45205720FFF796
:107B4000B3FEFFF791FE15480378282B21D10024BE
:107B50000470FCF799FC4FF47A753C24B0FBF5F601
:107B60001720FFF771FEB6FBF4F5B5FBF4F104FB4B
:107B70001152100200B2FFF797FE1820FFF764FEC3
:107B800004FB156318B2FFF78FFEBDE8F041FFF765
:107B90006BBEBDE8F08100BFCC0F0020CB0F0020F2
:107BA000BC1500204200002000007A446C0B00202D
:107BB000900A0020921500204A1500204000002065
:107BC000CC100020D00F002088160020A0860100D5
:107BD000154B2DE9F04180460F4698680221FCF7CD
:107BE0002BFC00242646781E84420F4D0DDA18F82F
:107BF0000410A8688E190134FCF7FAFB4FF47A7070
:107C0000B6B2FCF747FCE4B2EDE7F1B2A868FCF7C6
:107C1000EFFB4FF47A70FCF73DFCA8680121BDE84A
:107C2000F041FCF709BC00BF44170020024B0121C2
:107C30009868FCF701BC00BF44170020024B0321E9
:107C40009868FCF7F9BB00BF44170020F8B5544C06
:107C5000A068FCF7DDFB002800F0A080A068FCF71E
:107C6000DCFB05460520FCF720FC8A2D21D08E2D5B
:107C7000EDD14C4C00212E22204605F007F84A4A4F
:107C80007C2323701378E0207D21E07084F82C1091
:107C900014204FF4FA71A3772375482278232076B5
:107CA000607661836570628484F8243020462E21DA
:107CB00071E02020FFF776F90028C8D03B4C002166
:107CC0002C22204604F0E2FFA021E170384B394914
:107CD0007C207D22207084F82B201878CA7A657069
:107CE000A076002A52D0344934480F686625FE0F2A
:107CF00097FBF0FC6672324E5FFA8CFC06FB0C724E
:107D000084F8295006256A4342F21073B2FBF3FE51
:107D100003FB1E274968277391FBF0F03F0AC0B2AE
:107D20006773CF0F06FB00116943B1FBF3F56422C3
:107D300003FB1513E9B202FB0010010AE0732148AE
:107D4000217401885FFA8EFE63741B0A02FB0CEC3F
:107D5000A374B1FBF2F224235A4390B21A4A010AE7
:107D60001388E0712172180A1849207518480A888A
:107D700001884FEA1C2EE374130A84F80AC084F8C1
:107D80000BE0A7736275A375217702E0202384F8C6
:107D9000293006482C21FFF71BFF58E7F8BD00BF2C
:107DA00044170020FE0F0020CC100020D20F00202E
:107DB000A0160020B316002088160020A08601001F
:107DC0006079FEFF3E160020681600203216002063
:107DD0007416002008B50246032303480021F9F772
:107DE000FFFF024B186008BD003801404417002017
:107DF000024B18680068FFF7EDBF00BF2C10002091
:107E000008B5044B1860FFF7F3FFBDE8084000F029
:107E1000CFBF00BF2C100020034B187808B100F032
:107E2000D1BD01F03FB800BF30100020232801D1A0
:107E300000F0C8BD044B19688A7A824202D1012041
:107E4000FCF7F8BB704700BF2C10002010B5441E93
:107E500014F8011F21B1034B1868FCF7C9FAF7E7C2
:107E600010BD00BF441700200148FFF7EFBF00BF5F
:107E7000A0E5000810B50748FFF7E8FF0024064B0F
:107E800006481A19E15852680C34FBF77FF8C02CE9
:107E9000F5D110BDDEE50008BCE40008F4E50008FB
:107EA00070B5FCF7F1FA244C244B4FF47A71B0FB17
:107EB000F1F11A7822482378FBF768F8FFF78CF87D
:107EC00005462048204902682048B2FBF1F1FBF743
:107ED0005DF800241E4B53F8241051B1012000FA24
:107EE00004F0284202D01B48FBF750F80134E4B2FA
:107EF000F0E70220FFF756F868B1174A174B1178E0
:107F0000174853F82110FBF741F81648017A11B1D0
:107F10001548FBF73BF8154C1548FFF797FF2488E9
:107F2000F9F75CFE0246134821464FF46973BDE839
:107F30007040FBF72BB800BF40000020CC100020A1
:107F4000FCE500088801002040420F003AE60008E6
:107F5000E0F3000858E60008760A00207CE50008F7
:107F60005CE600085815002066E60008560A002066
:107F7000EAE800086AE6000838B50C6805462046BD
:107F800005F01CF8024628682146BDE8384005F097
:107F900045B8000037B5037904460D46052B34D8A3
:107FA000DFE803F003060A0D1114816809782DE05B
:107FB000806890F9001029E08368198826E08268BB
:107FC000B2F9001022E0816809681FE08068694604
:107FD0000068FBF7ADF801461148FAF7D7FFF5B195
:107FE000E068F8F793FD6946FBF7A2F801460D48F3
:107FF000FAF7CCFF2069F8F789FD6946FBF798F896
:1080000001460848FAF7C2FF09E000210648FAF7DE
:10801000BDFF25B10548E1682269FAF7B7FF3EBD0B
:1080200063E6000862E60008A0E600089CE6000897
:1080300008B50548FFF70AFF0A20FCF736FA0020CA
:10804000BDE80840FCF7F6BAA3E6000808B5074803
:10805000FFF7FCFE064B93F8A003FAF743FCFAF790
:1080600051FCBDE80840FFF7E3BF00BFB2E60008DF
:10807000D01000207FB5044604F0A0FF082825D1C9
:1080800000231F49E25C086885186E7806F003013A
:10809000022908BF203AE2540133082BF1D1002510
:1080A000665D1848314604F0ADFE28B1013560190F
:1080B000314604F0A7FE18B11348FFF7C7FE1DE0D4
:1080C000082DEDD120461149FFF7A6F81048FFF71B
:1080D000BDFE00230F4A04A9981890F808218818BB
:1080E000084A995C0133082B00F80C1CF2D10020DF
:1080F0008DF80C0001A90848FAF748FF7FBD00BFC2
:10810000A401002014E40008BCE60008D8110020F7
:10811000DCE60008D0100020F7E5000808B5FDF700
:10812000EFFF01300CBF03480348BDE80840FFF7EC
:108130008DBE00BFF1E6000817E700082DE9F04109
:10814000054604F03BFF0446FAF7DEFD064694B907
:108150002A48FFF77BFE2A4951F8241049B1012231
:1081600002FA04F2324202D02648FAF70FFF013435
:10817000F1E7254821E028462449224604F04EFF35
:1081800058B92348FFF762FE224C54F8041F002917
:10819000EFD01C48FAF7FAFEF7E72B782D2B04D125
:1081A0000135013C4FF0010801E04FF000080026C6
:1081B000134850F8267027B91748BDE8F041FFF77B
:1081C00045BE28463946224604F028FFA0B90120C2
:1081D00000FA06F0B8F1000F03D0FAF78DFD0F4852
:1081E00002E0FAF705FC0E48FFF730FE0D4839466D
:1081F000BDE8F041FAF7CABE0136D9E735E7000815
:1082000020E4000858E60008EAE80008DBF100086E
:1082100048E700081CE400085DE7000877E700086D
:1082200081E70008F7E5000810B504460848FFF7A5
:108230000DFE084A084809490023036013700B70BB
:10824000FDF7BCF82046BDE81040FFF7FFBE00BFB9
:108250008AE7000831100020641000203010002050
:1082600008B50448FFF7F2FDFAF7CAFBBDE808407D
:10827000FFF7DEBEA2E700082DE9F04389B004460F
:1082800004F09CFEC6B2002E6AD17A48FFF7DEFDEC
:10829000794C20690021F8F721FE38BB0136774878
:1082A0003146FAF773FE206904A9FAF741FF014647
:1082B0007348FAF76BFE606904A9FAF739FF0146C3
:1082C0006F48FAF763FEA06904A9FAF731FF014687
:1082D0006B48FAF75BFEE06904A9FAF729FF01464B
:1082E0006848FAF753FE10340C2ED2D10025664CA4
:1082F0002F46A8464FF000091034B14514DA404625
:1083000054F8101CF8F74EFB54F80C1C8046284615
:10831000F8F748FB54F8081C05463846F8F742FBC6
:1083200009F101090746E7E75848CDF804800295AE
:108330000397FFF78BFD002401A82358544923F02D
:108340000040F8F7F3FD5349534A0434002814BFA2
:1083500010460846FFF77AFD0C2CEDD14F4871E02E
:1083600020464F49052204F059FE38B9424B0022FD
:10837000C1181030C0280A61F8D177E02046494979
:10838000042204F04BFE054620460DBB202104F0DC
:1083900039FD00286AD0461C304604F00FFE2C46FA
:1083A0000746414850F824500DB940484AE030464D
:1083B0002946FAB204F032FE40B920463C49FDF7A6
:1083C00099F83C482946FAF7E1FD47E00134E8E72F
:1083D00004F012FB461E0B2E074643DC20462021EC
:1083E00004F010FD054640B1451C2846FAF708FF89
:1083F000214B3F01D851012400E0044628462021AA
:1084000004F000FD054640B1451C2846FAF7F8FE89
:108410001949013401EB061250612846202104F06D
:10842000F1FC054640B1451C2846FAF7E9FE124B1F
:10843000013403EB061188612846202104F0E2FC98
:1084400018B91D48FFF702FD10E00130FAF7D8FE19
:10845000094A032C02EB0616F061F2D11748FFF728
:108460000BFF03E016480C21FAF790FD09B0BDE8B8
:10847000F08300BFC3E70008D0100020EEE700083B
:10848000F4E70008F7E50008E4100020F8E700082A
:108490000AD7233CBFE70008BBE70008EAE800086A
:1084A00007E800080DE8000860E4000812E800088A
:1084B000E01000202AE800083DE8000829EB000849
:1084C00077E80008F8B5074604F078FD044638B9A7
:1084D0001A491B4B4A791B48511E53F8211028E0BA
:1084E00038461949224604F099FD60B91748FFF74C
:1084F000ADFC174C54F8041F19B11648FAF746FDA5
:10850000F8E7154805E000250D4B53F8256026B91E
:108510001248BDE8F840FFF799BC3846314622467C
:1085200004F07CFD01350028EED104483146457148
:108530000B48BDE8F840FAF729BD00BFD010002075
:1085400060E400089FE80008DBF10008B3E80008D9
:108550005CE4000858E60008EAE8000812E80008B1
:10856000C6E800082DE9F047064604F027FD054659
:1085700020B1012819D133782A2B16D14748FFF7AB
:1085800065FC002414266643454F4648F159FAF726
:10859000FDFCB8192946FFF7FDFC01344248FFF7FE
:1085A00055FC6F2CEED1BDE8F08730463D2104F03C
:1085B00029FC002857D0441C204604F01DFA8246AE
:1085C0002046FAF71DFE0027054614247C43DFF8F9
:1085D000D09054F80980404604F0F0FC4146024631
:1085E000304604F01BFD002835D14C44E068F8F714
:1085F0008DFA01462846F8F78FFC002829D020691B
:10860000F8F784FA01462846F8F77CFC002820D0C9
:1086100020792279052818BF5546052A0FD8DFE8AA
:1086200002F003030606090CA1680D7007E0A268BA
:10863000158004E0A068056001E0A1680D60414676
:108640001A48FAF7A3FC20460021BDE8F047FFF7DF
:10865000A1BC174803E001376F2FB6D11548BDE81C
:10866000F047FFF7F3BB0446142565430C4F314632
:1086700055F80780404604F0A3FF50B10948414631
:10868000FAF784FC78190021FFF784FC0648FAF712
:108690007DFC01346F2CE7D1BDE8F087D8E80008F5
:1086A00000F40008B2EA0008EAE80008EDE8000873
:1086B000F8E800081DE9000810B50446204604F05B
:1086C0007DFC10F0FF0F07D10B490C4891F8A01367
:1086D000BDE81040FAF75ABC204604F08DF9022894
:1086E00008D8054B064C83F8A003FAF70BF9FAF704
:1086F000C5F8E3E710BD00BFD01000203AE900083C
:1087000029EB000870B5044604F058FC08B920486D
:1087100030E020461F4905F0C9F8002426462546CA
:1087200078B12CB1012C06D104F066F9064602E0BE
:1087300004F062F9054600201649013405F0B6F848
:10874000EEE70B2D05D914480C21BDE87040FAF76F
:108750001DBC012C08DC114A114832F915202946AC
:10876000BDE87040FAF712BCA6F57A73B3F57A7FCC
:1087700004D90C48BDE87040FAF708BC0A482946FD
:108780003246FAF703FC054820F8156070BD00BFBB
:1087900050E90008F3EA00088AE9000808160020FA
:1087A000B0E90008C8E90008EAE9000838B505465C
:1087B00004F004FCC0B268B904461249124801EB47
:1087C0004402B2F8462021460134FAF7DFFB152CAB
:1087D000F3D138BD284604F00FF9142804460BDC09
:1087E0002021284604F00EFB04F006F9054B03EBAC
:1087F0004404A4F8460038BD04481521BDE83840BB
:10880000FAF7C4BB7814002003EA00080FEA000856
:108810002DE9F043584885B0584CFAF7B7FB584853
:10882000FFF7C4FF6279574B511E574853F8211088
:10883000FAF7ACFB20690021F8F750FB002858D16B
:108840000025266900213046F8F748FB00284CD166
:1088500001354E482946D4F81490D4F81880E769B9
:10886000FAF794FB30460021F8F742FB10B1484874
:10887000FAF78CFB69463046FAF75AFC0146454840
:10888000FAF784FB48460021F8F732FB10B1404864
:10889000FAF77CFB69464846FAF74AFC01463D4830
:1088A000FAF774FB40460021F8F722FB10B1384874
:1088B000FAF76CFB69464046FAF73AFC0146354840
:1088C000FAF764FB38460021F8F712FB10B1304884
:1088D000FAF75CFB69463846FAF72AFC01462E484F
:1088E000FAF754FB10340C2DABD12C48691CFAF765
:1088F0004DFBFAF709FA2A4C064654F8041F19B141
:108900002848FAF743FBF8E70D46274850F82510AA
:1089100049B1012202FA05F2324202D02348FAF7A5
:1089200035FB0135F1E7154B214ACE1896F8084181
:108930008B5C04A801310519082905F8103CF2D117
:1089400000241C4869468DF80840FAF71FFB1425DF
:108950006543194E1948A959FAF718FB00217019F7
:10896000FFF718FB01341648FFF770FA6F2CEED1B1
:1089700005B0BDE8F08300BF35EA0008D010002044
:1089800029EB000860E4000865EA000870EA0008C6
:10899000F3EA000863E60008F7E5000878EA000853
:1089A0001CE400088AEA000820E4000898EA0008AD
:1089B00014E40008A5EA000800F40008AEEA000884
:1089C000EAE80008F0B5694B87B01A783AB9012097
:1089D00018706748FFF73AFA6648FFF737FA664CAF
:1089E0002068FBF715FD002800F0BD802068FBF72C
:1089F00014FD09280146614A01D03F2851D10025C4
:108A000017685F4C2E462FB15E4821683A4604F045
:108A100005FB10B9254606B926465B490C348C4245
:108A2000F1D3C6B13468D5F800E03B46E05C1EF8EF
:108A3000031081420DD1534A41B92D2B06D8202471
:108A40004E48D45401330360D15404E0D054013370
:108A5000ECE74A490B60494A14681CB1AE4201D1A7
:108A60003C4612E04948FFF7F1F9AE4209D856F802
:108A70000C0BFFF7EBF9404B09211868FBF7B8FC2A
:108A8000F3E73C48FFF7E2F900243C4B18688442C6
:108A9000A5D239493B4A0868115DFBF7A9FC0134AE
:108AA000F3E713682BB9042838D13648FFF7BCFB2D
:108AB00059E00C2801D136488CE70A2901D00D294C
:108AC00048D12E4D3348FFF7C1F92E4C2A68324960
:108AD0000023A3540493009103A8294910220C23D6
:108AE000039403F08DFF054638B1006804F066FA80
:108AF0000130AA682018904702E02848FFF7A6F93D
:108B0000002130221F4804F0C1F818481B4B02789E
:108B100000211960002A7FF45FAF24E00C28CAD03E
:108B20007F2903D15BE72F2B3FF659AF1F297FF633
:108B300056AF7E293FF653AF13B920293FF44FAF0C
:108B4000104C0E480C4AE154013303601068FBF7E7
:108B50004FFC44E77F29E6D10A485C1E00210155FD
:108B600014600F4839E707B0F0BD00BF3010002097
:108B7000B8EA0008F0EA000844170020641000205A
:108B8000BCE40008311000207CE50008F5EA00088C
:108B9000FAEA0008EAE80008797F000805EB000817
:108BA00026EB0008F8B5174E174C184D0746C1B212
:108BB00030682170FBF71CFC22782B78C7F3072163
:108BC00082EA0300287030682170FBF711FC2178DD
:108BD0002A78306881EA0203C7F307412B702170BD
:108BE000FBF706FC2078297880EA0102390E30680C
:108BF00021702A70FBF7FCFB2B78207880EA0301B8
:108C00002970F8BD441700206B1000206810002068
:108C1000F8B50D4E0D4D0E4CC1B2074630682970A7
:108C2000FBF7E6FB2A782378391282EA03002070EA
:108C300029703068C9B2FBF7DBFB23782A7882EA17
:108C400003002070F8BD00BF441700206E10002004
:108C500068100020054B10B5044621461868FBF744
:108C6000C7FB034802785440047010BD441700202D
:108C700068100020034B04491A78885C01321A708E
:108C8000704700BF6A1000208510002010B5FFF764
:108C9000F1FF0446FFF7EEFF04EB002080B210BDA9
:108CA00010B5FFF7F3FF0446FFF7F0FF04EB0040B9
:108CB00010BD000038B5044624200D46FFF7CAFF5A
:108CC0004D20FFF7C7FF002C0CBF3E202120FFF7EF
:108CD000C1FF064B002228461A70FFF7BBFF04486D
:108CE0000078BDE83840FFF7B5BF00BF681000202E
:108CF0006F10002001460020FFF7DCBF0146012075
:108D0000FFF7D8BF014B1878FFF7A4BF6810002009
:108D100070B5054608460E46FFF7ECFF2C46721963
:108D2000D0B2E3B2984204D014F8010BFFF792FFDF
:108D3000F5E770BD10B5441E14F8010F10B1FFF730
:108D400089FFF9E710BD00002DE9F8430027012451
:108D50000025144B187885421CDA1349134B15F87B
:108D600001800C2202FB0830406804F027F981469C
:108D70000CB13F180CE026464E4509DA0B4A0C218F
:108D800001FB08235868805DFFF764FF0136F3E7B5
:108D90000135DEE724B1F8B2FFF7ACFF0024D7E7D6
:108DA000BDE8F8836C100020701000206C000020DB
:108DB00070B5394DFF211522284603F067FF0023C7
:108DC00002202B70FEF7EEF8012418B102206C701F
:108DD000A87003240420FEF7E5F868B12E4E0321A5
:108DE0004FF400503155651CF9F7F8FD18B1042215
:108DF0007255023400E02C460220FEF7D3F848B149
:108E0000254B05201E190621072518557170B570D0
:108E1000033404E00820FEF7C5F80028F0D1202034
:108E2000F9F7DCFD18B11C4B08221A5501344FF438
:108E30008070F9F7D3FD30B117480A2601190B25C8
:108E400006554D700234154A134B5079082801D04D
:108E50000E2802D10C261E5501340D21042019556F
:108E6000651CF9F7BBFD18B10B4811224255A51C32
:108E70000A49132391F82E21074E6C1C101C18BFB1
:108E800001207355F9F7AAFD10B114203055AC1C20
:108E9000034B1C7070BD00BF70100020D01000206C
:108EA0006C100020F8B5B54C2068FBF7B1FA00282B
:108EB00000F033852068FBF7B0FAB14A0346117819
:108EC00071B9B0F12404634253EB0401117000291D
:108ED000E9D1AC4A5478002CE5D1FEF7A7FFE2E7D0
:108EE000012904D14D280CBF0223002321E00229CF
:108EF00004D13C280CBF032300231AE003290FD11F
:108F000040284FF0000101D91170CCE79E489F4CDA
:108F100003709F48217001709E490B70042308E084
:108F2000042908D19B499C480C78037063400B705E
:108F300005231370B7E70529B5D19448924C017801
:108F400022788A42934A07D914785C401470934A75
:108F500053544B1C0370A6E71078984240F0D88415
:108F60008D4B19787B2900F01F8300F2C5806E2994
:108F700000F0698360D8682900F0328325D865291C
:108F800000F0068219D8642940F0BD840720844C83
:108F9000FFF7B0FEE620FFF75DFE6079FFF75AFEAF
:108FA0000020FFF757FE94F819017E4B7E4A0028F7
:108FB0000CBF1046184600F059BC662900F06682C6
:108FC000672940F0A08479480BE36B2900F01983EE
:108FD00023D8692900F009836A2940F0948410207D
:108FE000FFF788FE6748724CC07AFFF733FE71497D
:108FF0000878FFF72FFE2068FFF7D4FD6068FFF7C1
:10900000D1FD6D4AB2F90000FFF702FE6B4BB3F9D8
:109010000000FFF7FDFD6A4A12E36C2900F00383AC
:109020006D2940F070840620FFF764FE65490868EA
:10903000FFF7B8FD644A03E3732900F071833CD85D
:10904000702900F02F83C0F00F83712900F03D8359
:10905000722940F05884524C1620FFF74BFE002036
:10906000FFF7D6FDB4F9D000FFF7D2FD574DB4F9A4
:10907000D200FFF7CDFDB4F9D400FFF7C9FDB5F973
:10908000BA00FFF7C5FD0020FFF7C2FD0020FFF783
:1090900089FDB5F928000A2390FBF3F0FFF7B8FD2E
:1090A00094F80401FFF7D6FD94F80601FFF7D2FD0E
:1090B00094F80501FFF7CEFD61E3762900F03B83CC
:1090C0000DD8742900F01983752940F01C842F20D5
:1090D000FFF710FE3E48FFF72DFE00F017BC772982
:1090E00000F00E83782940F00E84384C3820FFF7CA
:1090F00001FE04F1400507E2D02900F0758300F27B
:10910000CA80CA2900F005816CD8A42900F0DA834E
:1091100010D8A02940F0F7830C20FFF7EBFD2D4974
:109120002D4C0868FFF73EFD2C4A1068FFF73AFD0A
:1091300020689BE3C82900F0DE80C92940F0E38362
:10914000FFF798FD0F4B1A4CD872FFF793FD1949A2
:109150000870FFF7A5FD2060FFF7A2FD6060FFF734
:1091600095FD154A1080FFF791FD144B18801C489F
:10917000017841F002040470DAE000BF44170020D7
:10918000C5100020B3160020691000206D100020CB
:109190006A100020681000206F1000208510002049
:1091A000D01000201C00008014000080540000201B
:1091B00088160020A0160020321600203E1600203F
:1091C000680E0020B41500206C0B002078140020DD
:1091D000ACFC0008E8F7FF1FF0F7FF1FECF7FF1FDC
:1091E000880E0020CD2900F0098322D8CB2900F079
:1091F000A180CC2940F08783FFF73CFDCC4CE07781
:10920000FFF738FD84F82000FFF734FD84F82300D1
:10921000FFF730FD84F82400FFF72CFD84F82500CB
:10922000FFF728FD84F82100FFF724FD84F82200D1
:109230007EE0CE2900F0EC82CF2940F06483FFF776
:1092400025FDFFF723FDBB4CB94DA4F8D000FFF777
:109250001DFDA4F8D200FFF719FDA4F8D400FFF714
:1092600015FDA5F8BA00FFF711FDFFF719FDFFF78F
:109270000DFD0A2358432885FFF7FCFC84F8040100
:10928000FFF7F8FC84F80601FFF7F4FC84F8050109
:10929000FFF7F0FC4CE0D52900F094810FD8D229DB
:1092A00061D0C0F07082D3296DD0D42940F02B83D7
:1092B0009F4C0020FFF71EFD04F1400556E1F02908
:1092C00000F0C7820CD8D62944D0EF2940F01B8388
:1092D000FFF7DCFC964CA085FFF7D8FC608527E003
:1092E000FA2900F09D82FE2940F00D830820FFF747
:1092F00001FD0024A5E20024FFF7C8FC8E4A1053AC
:109300000234102CF8D10020FFF7F4FCFDF79EFF8B
:10931000FCE28A4C04F10A05FFF7ACFC01346070F2
:10932000FFF7A8FCE072FFF7A5FCAC426075F3D133
:10933000002083E20024824801788C42F8D2814DDB
:10934000655DFFF7A3FC7A4A013402EB4505A5F8F9
:109350004600F0E70024FFF799FC7B4A10530234E3
:10936000102CF8D1E4E7794C6478002CE0D1FFF7B9
:1093700081FC7049022881F8A00388BF81F8A043CE
:10938000F9F7C0FA37E2FFF781FC714B1880CFE79D
:10939000704D0B20FFF7AEFCB5F90000FFF738FC6D
:1093A000F8F71CFC00B2FFF733FC0220FDF7FAFDD2
:1093B00005460420FDF7F6FD04460820FDF7F2FD02
:1093C000820042EA4401294320208CB2FDF7EAFDE5
:1093D00044EAC00084B21020FDF7E4FD44EA001323
:1093E00018B2FFF715FC594A1079D17884005378E8
:1093F000907944EA4101194341EAC0045179537A12
:1094000044EA411040EA83145348C17944EAC11345
:10941000047A417A43EA042343EA4124D379117A56
:1094200044EA8324927A44EAC123417B43EA02342A
:10943000827B44EA4133017C43EA8234027944EA84
:109440000143417C43EA0214827C44EA4143C17CEB
:1094500043EA8244007D44EAC142394B42EA005467
:109460000020197803468B420AD2364D01225D5DF9
:1094700002FA05F525421CBF9A4010430133F2E77A
:109480002C4CFFF78FFB94F8A00379E11220FFF733
:1094900031FC32490C88B4F5806F314CB4F90000CE
:1094A00008D8FFF7B5FBB4F90200FFF7B1FBB4F938
:1094B00004000EE0082590FBF5F0FFF7A9FBB4F9D6
:1094C000020090FBF5F0FFF7A3FBB4F9043093FB27
:1094D000F5F0244CFFF79CFBB4F90000FFF798FB74
:1094E000B4F90200FFF794FBB4F904001E4CFFF737
:1094F0008FFBB4F90000FFF78BFBB4F90200FFF714
:1095000087FBB4F90400AEE1B4F97800FFF780FB03
:10951000B4F97A00FFF77CFBB4F97C00FFF778FB25
:1095200094F87E000834FFF795FBAC42ECD1EDE1F6
:1095300078140020D01000200A1700207714002093
:109540006C1000207010002008160020B3160020B8
:1095500080150020560A0020C4160020420000207A
:10956000BC150020600B002068150020FFF78EFB63
:10957000A4F87800FFF78AFBA4F87A00FFF786FBCF
:10958000A0F57A7107288AB298BF84F87F00B2F5F7
:109590007A7F98BFA4F87C00FFF76CFB84F87E000C
:1095A0000834AC42E2D1B1E10820FFF7A3FB00246C
:1095B000B04AA31893F87F000834FFF74BFB402C08
:1095C000F6D1A3E10020FFF795FB0024FFF752FB43
:1095D000A84AA3180834402C83F87F00F6D195E1FF
:1095E000A5481021FFF794FB90E11020FFF782FBC4
:1095F0000024A248005F0234FFF70AFB102CF8D1C8
:1096000084E10520FFF776FB9D4BB3F90000FFF7DF
:10961000FFFA9C48B0F90000FFF7FAFA9A490A7875
:1096200002F00100ACE0994C0620FFF763FBB4F9AF
:109630000000FFF7EDFAB4F90200FFF7E9FA944AE7
:10964000B2F900000FE10720FFF754FB91480078C2
:10965000FFF700FB0020FFF7DBFA8F4BB3F90000A8
:10966000FFF7D6FA0020FEE0824C0720FFF742FB0E
:10967000E07FFFF7EFFA94F82000FFF7EBFA94F899
:109680002300FFF7E7FA94F82400FFF7E3FA94F8D1
:109690002500FFF7DFFA94F82100FFF7DBFA94F8D2
:1096A00022006DE01E20FFF725FB7C4C04F10A052B
:1096B00001346078FFF7CEFAE07AFFF7CBFA607DED
:1096C000FFF7C8FAAC42F3D120E175490A7854009B
:1096D00004F0FE00FFF70EFB0024714803789C4263
:1096E00080F014816F496348625C013400EB4203EF
:1096F000B3F94600FFF78CFAEFE7FFF725FB05E12A
:10970000674900240878FFF7F5FA654A1078844223
:1097100080F0FC80634B185DFFF79CFA0134F4E79E
:109720000820FFF7E7FA0124E0B20134FFF792FACC
:10973000092CF9D1EAE0FFF79DFA06461220FFF75F
:10974000D9FA0EB9584902E0102E03D157490D68D5
:109750004C6801E0002425463046FFF77BFA284696
:10976000FFF720FA2046FFF71DFA514A1068FFF76D
:1097700019FA0020FFF74CFA0020FFF749FA002001
:10978000FFF768FAC2E0FFF775FA0546FFF788FAB7
:109790000746FFF785FA0646FFF782FA0446FFF709
:1097A00075FAFFF773FAFFF765FA65B93E48414964
:1097B000012207604660CD710A73002C3FF4B8ADFA
:1097C0003B4B1C60B4E5102D7FF4B2AD3748076009
:1097D00046600CB136490C603448374B0222011DFB
:1097E0001A70FCF7CDFCA3E53248417800297FF4DC
:1097F0009FADF9F705F9F9F741F899E52D4C637834
:10980000002B7FF495AD4FF4C870FAF72BFC8FE571
:109810002848417800297FF48BAD0122827387E5C7
:10982000244B5C78002C6ED1244991F8A003F9F701
:1098300059F8F9F767F8F9F721F82046FFF75AFACF
:1098400064E01F48005F0234FFF7E2F9082CF8D10A
:109850005CE0084C0420FFF74DFAB4F92C00FFF748
:10986000D7F9B4F92A00FFF7D3F94FE0FFF79AF9D7
:109870004CE000BF78140020F01500200A170020EB
:109880006816002074160020880E0020800B00202F
:1098900092150020CC1000205415002077140020D1
:1098A0006C100020701000206C1600204016002064
:1098B000B8150020B3160020900C0020D010002016
:1098C0004C150020154C23789800411CC8B2FFF7B6
:1098D00011FA2078FFF7BEF90024104A13789C4251
:1098E00014D20F48005DFFF7B5F90E49085DFFF788
:1098F000B1F90D4A105DFFF7ADF90C4B185DFFF79C
:10990000A9F90134E9E70020FFF7F8F9FFF7FAF9C0
:10991000074900200870FFF7C6BAF8BDA11600205D
:10992000211600207616002090160020A216002096
:10993000C51000202DE9F041074688461646002450
:10994000B44213D00025BD420AD0094B0135DA6874
:10995000EDB282F48050D8604046FAF7A6FDF2E7F7
:109960003C200134FAF7A1FDE4B2E9E7BDE8F0815B
:10997000001001400F4B1A6842F00100186059684E
:109980000D4A0A405A60186820F0847121F4803230
:109990001A60186820F4802119605A684FF41F017A
:1099A00022F4FE0058609960044B4FF000629A6008
:1099B000704700BF001002400000FFF800ED00E01B
:1099C000164A174B516801F00C00042803D00828F0
:1099D00005D0144801E014490868186011E0516886
:1099E0005068C1F383410231C00301D40F4A06E03D
:1099F00052680D4812F4003F026818BF52085143E4
:109A00001960064B0A485A68054BC2F30311415CC2
:109A10001A6822FA01F21A60704700BF0010024073
:109A20008801002000127A008401002000093D0016
:109A3000740100201FB50023574C4FF4E011009330
:109A4000019302930391226842F480332360A16959
:109A500041F01002A261504C236803F400310191DF
:109A6000009A531C0093019919B9009AB2F5A06F9E
:109A7000F1D12168484B11F4003401D0022416E0E2
:109A80001A6842F0010119600094434B1C6804F00D
:109A90000202019200994C1C0094019A1AB9009993
:109AA000B1F5A06FF1D11B6899073BD501243B4963
:109AB00002940A6842F010030B600C6824F0030261
:109AC0000A600B6843F002040C60A1F580535968EA
:109AD00059605A685A605C68314A44F48061596040
:109AE000146824F0704111602E4C2F490C605C68A2
:109AF00024F47C145C60146844F00044146094689E
:109B000024F400449460043A9268120449BF274A3E
:109B10004FF4E0120A604FF4801203920299012977
:109B200001D119E0FEE702291AD168B10398B0F516
:109B3000801F02D14FF4A01205E0039BB3F5E01F94
:109B400002D14FF400120392134B5968039841EA73
:109B5000000242F4803002E0596841F4601058601D
:109B60000D4B1A68184642F08071196002680A4B62
:109B70009201FBD5596821F0030058605A6842F001
:109B800002015960044B586800F00C02082AF9D110
:109B9000FFF716FF1FBD00BF00100240002002406B
:109BA0000410014000127A0084010020001BB7005D
:109BB000CB78F0B5DA0648BF8A78098803F00F053C
:109BC00048BF154311F0FF0F1ED004680022012783
:109BD00007FA02F707EA0106BE4211D197004FF0DB
:109BE0000F0C0CFA07FC05FA07F724EA0C04282BE3
:109BF00044EA070401D1466102E0482B08BF066130
:109C00000132082AE3D10460FF2920D944680022E8
:109C100002F10806012707FA06F707EA0106BE4225
:109C200011D197004FF00F0C0CFA07FC05FA07F75B
:109C300024EA0C04282B44EA070401D1466102E01F
:109C4000482B08BF06610132082AE1D14460F0BD0B
:109C500008B5154B98420BD101214FF4805000F00C
:109C6000B5FD4FF480500021BDE8084000F0AEBDC6
:109C70000E49884207D14FF48040012100F0B2FD27
:109C80004FF4804009E00A4A90420BD14FF4004063
:109C9000012100F0A7FD4FF400400021BDE808407D
:109CA00000F0A0BD08BD00BF0030014000380040FA
:109CB000003C00400B8810B54C88028823438C88F8
:109CC00002F441522343CC8823430C8923434C891B
:109CD00023438C892343CC89098A23431A4393B2B3
:109CE0000380828B22F400631A04130C83830182A5
:109CF00010BD038819B199B241F0400303E023F08D
:109D000040010A04130C03807047818170478089E9
:109D100080B27047038919420CBF002001207047B0
:109D2000426810B522F470230A6823F4807444EA70
:109D300002030C7943EA04224260CB688A68846893
:109D40001A43084B234013434A7943EA4203836092
:109D5000097CC26A4B1E22F47002D9B242EA015257
:109D6000C26210BDFDF7F1FF836811B143F001013C
:109D700001E023F0010181607047836811B143F471
:109D8000807101E023F4807181607047836843F043
:109D90000801816070478068C0F3C0007047836825
:109DA00043F00401816070478068C0F38000704711
:109DB000836811B143F4A00101E023F4A0018160A4
:109DC0007047092970B54FF003040CD94C4307259F
:109DD0001E3C05FA04F503FA04F3C66826EA0505F5
:109DE0002B43C3600BE04C43072505FA04F503FA47
:109DF00004F3066926EA050545EA03040461062A18
:109E00004FF005030DD8013A53431F2202FA03F223
:109E100001FA03F1446B24EA020242EA01034363BC
:109E200070BD0C2A0DD853431F22233B02FA03F2C4
:109E300001FA03F1046B24EA020242EA010303631C
:109E400070BD53431F22413B02FA03F201FA03F1B2
:109E5000C46A24EA02021143C16270BD40F0BF60CF
:109E6000024B40F40031D960704700BF00ED00E0C4
:109E7000C37810B503B3164CE168CB43C3F3022497
:109E80004178C4F1040201FA02F10F2222FA04F22D
:109E90008478037822400A43110103F16043CAB277
:109EA00003F5614181F800230078012200F01F03CF
:109EB000410902FA03F007E00078012200F01F03D5
:109EC000410902FA03F02031024B43F8210010BD92
:109ED00000ED00E000E100E030B5048C24F0010565
:109EE0002C04250C0584048BA5B225F0F3052A4328
:109EF00042EA0313114A048C9042A4B29DB215D0D9
:109F000002F50063984211D0B0F1804F0ED0A3F556
:109F1000983290420AD002F58063984206D003F549
:109F20008062904218BF24F00A0401D124F0020498
:109F300044F0010421430583018430BD002C01401D
:109F400030B5048C24F010052C04250C0584048BFA
:109F5000058C24F440742405240D44EA022242EACC
:109F60000333144AADB290429BB212D002F50062A4
:109F700090420ED0B0F1804F0BD0A2F598329042B3
:109F800007D002F58062904203D002F580629042D1
:109F900007D125F0200242F0100545EA011189B2EF
:109FA00004E025F0A00545F0100529430383018452
:109FB00030BD00BF002C0140224A038890429BB272
:109FC00012D002F5006290420ED0B0F1804F0BD05B
:109FD000A2F59832904207D002F58062904203D0F9
:109FE00002F58062904203D14A8823F07003134344
:109FF000154A904208D002F58062904204D023F4C2
:10A000004073CA889BB2134303808B880A88838578
:10A010000C4B028598420FD003F5006290420BD0A2
:10A0200002F54063984207D003F58062904203D066
:10A0300002F58063984201D1097A01860122828269
:10A04000704700BF002C014000100040038C70B529
:10A0500023F001021404250C0584068C8388028BEE
:10A060009CB222F073052B040D881A0C26F0020610
:10A0700033042A434E880D891B0C3543ADB22B4364
:10A08000134DA8420FD005F50065A8420BD005F589
:10A090004065A84207D005F58065A84203D005F5C4
:10A0A0008065A8420ED123F008064B898D881E4397
:10A0B00026F004032B43CE898D8924F44074354364
:10A0C000ADB22C43C988848002838186038470BD2D
:10A0D000002C0140038C30B523F010021404250C31
:10A0E0000584038C8288048B23F0200324F4E64546
:10A0F0002C040D88240C44EA05241D042B0C0D8926
:10A1000092B243EA05134D88A4B243EA0513124DF7
:10A110009BB2A84203D005F50065A84215D14D8930
:10A1200023F080039BB243EA05134FF6BF751D4031
:10A130008B8822F4406245EA0315ABB28D8942EA6E
:10A140008502CD8942EA850292B2C9888280048361
:10A150000187038430BD00BF002C0140038C30B563
:10A1600023F480721404250C0584038C8288848B6C
:10A1700023F4007324F073052C040D88240C2C4365
:10A180001D042B0C0D8992B243EA05234D8843EA46
:10A190000523124D9BB2A84203D005F50065A842E5
:10A1A00015D14D8923F400639BB243EA05234FF692
:10A1B000FF351D408B8822F4405245EA0325ABB29F
:10A1C0008D8942EA0512CD8942EA051292B2C98808
:10A1D000828084838187038430BD00BF002C0140CE
:10A1E000038C30B523F480521404250C0584038CB1
:10A1F0008288858B94B225F4E64215042A0C0D88DA
:10A2000023F4005342EA05221D042B0C0D8992B25F
:10A2100043EA05334D8843EA05330A4D9BB2A84211
:10A2200003D005F50065A84205D18D8924F480444A
:10A2300044EA8514A4B2C98884808283A0F84010BF
:10A24000038430BD002C014000214FF6FF73838052
:10A250000180C180418001727047038819B199B2B1
:10A2600041F0010303E023F001010A04130C038011
:10A270007047B0F8443029B16FEA43436FEA534165
:10A280008AB201E059044A0CA0F84420704783893F
:10A290009BB20AB1194301E023EA010181817047B1
:10A2A000038B23F0080213041A0C11430183704737
:10A2B000038B23F4006213041A0C42EA01218BB2CF
:10A2C00003837047838B23F0080213041A0C114395
:10A2D00081837047838B23F4006213041A0C42EAD3
:10A2E00001218BB283837047038B23F00C0213048C
:10A2F0001A0C0283038B9AB2114301837047038BBC
:10A3000023F4406213041A0C0283038B9AB242EACC
:10A3100001218BB203837047838B23F00C0213045B
:10A320001A0C8283838B9AB2114381837047838B8B
:10A3300023F4406213041A0C8283838B9AB242EA9C
:10A3400001218BB283837047F8B50B880D46044614
:10A350004988AA8843B92B89FFF7BEFDE9882046C2
:10A36000BDE8F840FFF7C0BF042B08D12B89FFF7E9
:10A37000E7FDE9882046BDE8F840FFF7C0BF082B9D
:10A380000E462F89008C3BD120F480731804030CF7
:10A390002384A08B83B223F0F30343EA0717374BE0
:10A3A000208CBFB29C4280B247EA020212D003F571
:10A3B00000639C420ED0B4F1804F0BD0A3F59833CC
:10A3C0009C4207D003F580639C4203D003F5806371
:10A3D0009C4207D120F4007040EA06218BB243F47E
:10A3E000807305E020F4206041F4807140EA0103AD
:10A3F000E9882046A2832384BDE8F840FFF78CBF9C
:10A4000020F480531804030C2384A38B208C23F4A2
:10A4100040731B051B0D43EA022242EA0733174A29
:10A4200080B294429BB212D002F5006294420ED0E8
:10A43000B4F1804F0BD0A2F59832944207D002F5C8
:10A440008062944203D002F58062944207D120F4E6
:10A45000005040EA063291B241F4805205E047F6DE
:10A46000FF52024041F480510A43E9882046A38309
:10A470002284BDE8F840FFF75ABF00BF002C01401E
:10A48000808E80B27047008F80B27047808F80B21C
:10A490007047B0F8400080B27047038A828911EAA1
:10A4A000030092B203D011420CBF0020012070477C
:10A4B000C9438AB202827047038A30B50D4604460A
:10A4C000EA8898B220F4405111432182A389288957
:10A4D000A98823F4B05340EA0102688923F00C01F3
:10A4E00002430804030C1A4391B2A181A08AAA89ED
:10A4F00083B223F4407187B01143A18201A800F018
:10A50000F3F81848A38984420CBF0498039819B241
:10A5100000294FF019032A6803FB00F001DA51000B
:10A5200000E09100B0FBF1F16423B1FBF3F2120102
:10A53000100903FB1011A08900B2002806DAC90037
:10A540003231B1FBF3F303F0070005E009013231CA
:10A55000B1FBF3F303F00F00024390B2208107B088
:10A5600030BD00BF00380140838919B199B241F470
:10A57000005303E023F400510A04130C8381704755
:10A58000C1F3421310B5012401F01F01A34204FAE4
:10A5900001F101D10C3004E0022B01D1103000E0B8
:10A5A0001430036812B143EA010201E023EA010218
:10A5B000026010BD838A9BB20AB1194301E023EA0D
:10A5C000010181827047090A012303FA01F3DA438A
:10A5D00091B2018070470000034A044B02F18830B9
:10A5E0005A605860704700BF230167450020024051
:10A5F000024B1A6942F08000186170470020024047
:10A60000014BD860704700BF00200240084BDA6859
:10A61000D20709D4D868400708D4D96811F0100FC0
:10A620000CBF0420032070470120704702207047B0
:10A630000020024010B50446FFF7E8FF012806D1CC
:10A640001CB1FFF7E3FF013CF8E7052010BD002C2B
:10A6500008BF052010BD000073B5002306464FF467
:10A6600000500D460193FFF7E5FF04281AD10E4C68
:10A67000AAB2206940F0010121614FF400503280FC
:10A68000FFF7D8FF042808D102360196019B2D0C54
:10A690001D804FF40050FFF7CDFF216941F6FE7297
:10A6A0000A4022617CBD00BF0020024038B505464B
:10A6B0004FF43020FFF7BEFF042812D1094C236964
:10A6C00043F002002061656121694FF4302041F0C0
:10A6D00040022261FFF7AEFF216941F6FD730B4096
:10A6E000236138BD00200240204B10B55A6802F0AB
:10A6F0000C01042903D0082905D01D4B01E01D4C95
:10A700002368036011E05C685968C4F38342941CB9
:10A71000C90301D4184A06E016495B680A6813F4B5
:10A72000003F18BF520854430460104B5968C1F3EE
:10A73000031212498C5C026822FA04F242605C68DF
:10A74000C4F302240C5D22FA04F484605C68C4F350
:10A75000C224095D22FA01F2C2605B680849C3F3B2
:10A760008133CB5CB2FBF3F2026110BD00100240FA
:10A7700000127A008401002000093D0090010020B1
:10A780008C010020044B5A6909B1104301E022EA10
:10A7900000005861704700BF00100240044B9A69E6
:10A7A00009B1104301E022EA00009861704700BF40
:10A7B00000100240044BDA6909B1104301E022EABB
:10A7C0000000D861704700BF00100240044BDA68F7
:10A7D00009B1104301E022EA0000D860704700BFD1
:10A7E00000100240044B1A6909B1104301E022EA4B
:10A7F00000001861704700BF00100240024B5A6A07
:10A8000042F08070586270470010024008B50B4B50
:10A81000984207D14FF400100121FFF7E3FF4FF4F6
:10A82000001006E04FF480000121FFF7DBFF4FF43A
:10A8300080000021BDE80840FFF7D4BF005400406D
:10A84000F0B58688044687B026F03F000D46010427
:10A8500001A80E0CFFF748FF2C4A0399B1FBF2F058
:10A8600087B23E43A680238823F0010213041A0C0A
:10A8700022802B68264A93420AD85B00B1FBF3F092
:10A88000013783B2BFB22784032B98BF042320E093
:10A89000EE884BF6FF72964204D103225343B1FB7C
:10A8A000F3F305E019225343B1FBF3F141F4804384
:10A8B00099B20A054FF4967208BF41F00101504366
:10A8C00041F400434FF47A7190FBF1F0421C91B2D5
:10A8D0002184A383228891B241F001032380208840
:10A8E00020F4816222F002010B04AA886989180C05
:10A8F00041EA02032989AA89184380B241EA020386
:10A90000208098B2208107B0F0BD00BF40420F0008
:10A91000A086010041F28833002103604BF6FF72EC
:10A920004FF480438180C2800181418183817047DF
:10A93000038819B199B241F0010303E023F001014A
:10A940000A04130C03807047038819B199B241F4CB
:10A95000807303E023F480710A04130C03807047B2
:10A96000038819B199B241F4007303E023F4007134
:10A970000A04130C03807047038819B199B241F49B
:10A98000806303E023F480610A04130C03807047A2
:10A9900083889BB20AB1194301E023EA0101818057
:10A9A000704701827047008AC0B2704712B141F00F
:10A9B000010101E001F0FE010182704702684FF6DB
:10A9C000FE73134003602D4B0021984201604160EB
:10A9D0008160C16022D02A49884229D0294B9842FF
:10A9E00030D02949884237D0284B98423ED0284B56
:10A9F000984206D153F8681C41F4700043F8680C83
:10AA000070472449884206D151F87C0C40F07062AE
:10AA100041F87C2C7047204B984206D153F8042C07
:10AA200042F00F0143F8041C70471C49884206D1CC
:10AA300051F8183C43F0F00041F8180C7047184BDF
:10AA4000984206D153F82C2C42F4706143F82C1C28
:10AA500070471449884206D151F8403C43F4704095
:10AA600041F8400C7047104B984205D153F8542CD4
:10AA700042F4702143F8541C704700BF08000240A4
:10AA80001C000240300002404400024058000240D6
:10AA90006C00024080000240080402401C04024096
:10AAA00030040240440402405804024070B5066875
:10AAB0008C680D6A26F4FF4222F070060A6945EAA6
:10AAC00004034C6913438A692343CC6913431C4331
:10AAD0004B6A44EA03028B6A1A4332430260CB6832
:10AAE0000A68496843608260C16070BD00230360EA
:10AAF00043608360C360036143618361C361036238
:10AB000043628362704719B1016841F0010303E0B9
:10AB100002684FF6FE7313400360704703680AB182
:10AB2000194301E023EA0101016070474160704769
:10AB3000406880B270470000C3004CBF014B024B1D
:10AB400058607047000402400000024000B540F623
:10AB5000D87320F00042C3F649739A4283B001468D
:10AB600015DDB2F1FF4F03DBF5F71AFF03B000BDAF
:10AB7000694600F095FB00F00302012A0098019954
:10AB80000ED0022A07D082B900F0A0FDEEE7002126
:10AB900000F09CFDEAE700F099FD00F10040E5E7D8
:10ABA00001F040FC00F10040E0E7012201F03AFC36
:10ABB000DCE700BF30B5C0F3C754A4F17F031E2B00
:10ABC00083B0014621DC581C1DDBCD0F162B0CDD9C
:10ABD00021F07F4323F4000040F40000963C00FA8B
:10ABE00004F005B1404203B030BD114850F8254093
:10ABF0002046F5F7D7FE019021460198F5F7D0FEE3
:10AC000020F0004121B90020EDE7F6F799F9EAE7D5
:10AC100020F07F4222F40003C0F3C75043F4000148
:10AC2000C0F1960221FA02F0002DDCD0DAE700BF75
:10AC30008CFD000800B540F6D87320F00042C3F642
:10AC400049739A4283B0014616DDB2F1FF4F03DB30
:10AC5000F5F7A6FE03B000BD694600F021FB00F049
:10AC60000300012815D002280BD0B8B9009801992B
:10AC7000012201F0D7FBEDE70021002201F0D2FB19
:10AC8000E8E700980199012201F0CCFB00F10040B7
:10AC9000E0E70098019900F019FDDBE700980199C1
:10ACA00000F014FD00F10040D4E700BF70B58AB099
:10ACB000064600F09BF8224C054694F9003001331B
:10ACC00003D0304601F0B0FD10B928460AB070BD7F
:10ACD000304601F05BFD4FF07E51F6F727F9002872
:10ACE000F3D0184A012100253046019200910895C1
:10ACF000F5F79CFB02460B461348CDE90423CDE94A
:10AD0000022301F011FC94F90030CDE90601022B79
:10AD10000BD0684601F006FC38B1089850B9DDE95F
:10AD20000601F5F7E9FD0546CFE701F089FE21218F
:10AD30000160F2E701F084FE089A0260EFE700BFCD
:10AD4000A001002094FD00089CFD000800F002BA5C
:10AD500070B58AB0054600F04FFC224C064694F9C7
:10AD60000030013308D0284601F05EFD20B12846AE
:10AD70000021F6F7BDF810B930460AB070BD1A4A86
:10AD8000012128460026009101920896F5F74EFB16
:10AD90002478CDE90401CDE902017CB90022002329
:10ADA000CDE90623684601F0BDFB88B10898A0B93B
:10ADB000DDE90601F5F7A0FD0646DDE700200021EC
:10ADC00002460B46F5F7B0FC022CCDE90601E9D1AD
:10ADD00001F036FE21230360E8E701F031FE089917
:10ADE0000160E5E7A0010020A0FD0008F8B520F013
:10ADF0000043B3F17E5F044613D00BDCB3F17C5FFC
:10AE000014DAB3F10C5F00F3A48040F6DB70C3F6F4
:10AE1000C970F8BD0146F5F7C3FD0146F5F77EFFA1
:10AE2000F8BD002840F30E810020F8BD0028C0F2D4
:10AE30000E8101464FF07E50F5F7B2FD4FF07C5188
:10AE4000F5F7B8FE044600F0D7FB4EF6087106464B
:10AE500020F47F65C3F611012046F5F7ABFE47F6F7
:10AE60000471C3F64F21F5F79DFD2146F5F7A2FECB
:10AE700041F24611C3F62451F5F792FD2146F5F74C
:10AE800099FE40F6A821C3F64E61F5F78BFD2146E9
:10AE9000F5F790FE4BF29001C3F6A661F5F780FD41
:10AEA0002146F5F787FE4AF6AB21C3F62A61F5F78E
:10AEB00079FD2146F5F77EFE4CF22E610746C3F67A
:10AEC0009D512046F5F776FE43F26131C3F63071AD
:10AED000F5F766FD2146F5F76DFE45F22D71C4F2DA
:10AEE0000101F5F75FFD2146F5F764FE4DF23911DA
:10AEF000C4F21901F5F754FD2146F5F75BFE4FF05A
:10AF00007E51F5F74FFD01463846F5F707FF31460C
:10AF1000F5F750FE25F00F05074629462846F5F7B8
:10AF200049FE01462046F5F73BFD294604463046DA
:10AF3000F5F738FD01462046F5F7F0FE01463846A4
:10AF4000F5F730FD2946F5F72DFD0146F5F72AFD09
:10AF5000F8BD0146F5F72EFE4EF60871C3F6110155
:10AF60000546F5F727FE47F60471C3F64F21F5F7BE
:10AF700019FD2946F5F71EFE41F24611C3F624518C
:10AF8000F5F70EFD2946F5F715FE40F6A821C3F6A4
:10AF90004E61F5F707FD2946F5F70CFE4BF29001DF
:10AFA000C3F6A661F5F7FCFC2946F5F703FE4AF661
:10AFB000AB21C3F62A61F5F7F5FC2946F5F7FAFD52
:10AFC0004CF22E610646C3F69D512846F5F7F2FD78
:10AFD00043F26131C3F63071F5F7E2FC2946F5F72B
:10AFE000E9FD45F22D71C4F20101F5F7DBFC2946BC
:10AFF000F5F7E0FD4DF23911C4F21901F5F7D0FC77
:10B000002946F5F7D7FD4FF07E51F5F7CBFC014609
:10B010003046F5F783FE01462046F5F7CBFD0146A5
:10B0200042F26810C3F2A230F5F7BAFC014620469E
:10B03000F5F7B6FC014640F6DA70C3F6C970F5F7CD
:10B04000AFFCF8BD40F6DB70C4F24900F8BD4FF02C
:10B050007E51F5F7A7FC4FF07C51F5F7ABFD4EF6AE
:10B060000871C3F611010446F5F7A4FD47F6047113
:10B07000C3F64F21F5F796FC2146F5F79BFD41F20B
:10B080004611C3F62451F5F78BFC2146F5F792FDE6
:10B0900040F6A821C3F64E61F5F784FC2146F5F78A
:10B0A00089FD4BF29001C3F6A661F5F779FC2146C4
:10B0B000F5F780FD4AF6AB21C3F62A61F5F772FC7D
:10B0C0002146F5F777FD0646204600F095FA4CF24A
:10B0D0002E610546C3F69D512046F5F76BFD43F200
:10B0E0006131C3F63071F5F75BFC2146F5F762FD7F
:10B0F00045F22D71C4F20101F5F754FC2146F5F734
:10B1000059FD4DF23911C4F21901F5F749FC2146F8
:10B11000F5F750FD4FF07E51F5F744FC01463046FF
:10B12000F5F7FCFD2946F5F745FD42F26811C3F23B
:10B13000A231F5F735FC01462846F5F733FC014608
:10B14000F5F730FC014640F6DA70C4F24900F5F735
:10B1500027FCF8BDF8B521F00044B4F1FF4F0346D9
:10B1600017DC20F00045B5F1FF4F064611DCB1F1C8
:10B170007E5F42D08F1707F0020040EAD37775B99F
:10B18000022F35D0032F08D140F6DB73CCF24903F0
:10B1900003E01846F5F706FC03461846F8BDD4B19F
:10B1A000B4F1FF4F2DD0B5F1FF4F14D02C1BE41597
:10B1B0003C2C18DC002952DB1846F5F7AFFD01F0F6
:10B1C000E5FA01F0B7F9012F46D0022F35D0002F54
:10B1D00025D10346E1E7002E40F6DB731CDBC3F606
:10B1E000C9731846F8BD40F6DB70C3F6C970EAE7CC
:10B1F00040F6DB73C4F24903CFE7BDE8F84001F045
:10B2000099B9B5F1FF4F2FD0022FF1D0032FBBD04A
:10B21000012F34D00023C0E7CBF6C973BDE74BF64E
:10B220002E51C3F2BB31F5F7BDFB40F6DB71C4F222
:10B230004901F5F7B5FB0346AFE74BF62E51C3F2D4
:10B24000BB31F5F7AFFB014640F6DB70C4F24900B5
:10B25000F5F7A6FB0346A0E700F100439DE714F1D4
:10B260003C0FA9DA0020AEE7022F13D0032F0CD039
:10B27000012F40F6DB7305D0C3F649738DE74FF01D
:10B2800000438AE7CBF6497387E74CF6E433CCF208
:10B29000160382E74CF6E433C4F216037DE700BFE1
:10B2A0002DE9F04F40F6D87320F00044C3F64973FF
:10B2B0009C4289B006460D4640F38B804CF6E33144
:10B2C000C4F216018C4226DC4FF478610028C3F6E4
:10B2D000C97140F32B81F5F763FB4FF47D6224F0D5
:10B2E0000F04C3F6C9729442064600F0818044F20E
:10B2F0004341C3F23571F5F753FB014628603046F0
:10B30000F5F74EFB44F24341C3F23571F5F748FBC4
:10B310000127686061E04FF47867C4F24937BC42A6
:10B3200040F38180B4F1FF4F5BDA4FEAE459A9F1B1
:10B330008609A4EBC9542046F5F702FEF5F7E6FBB3
:10B340000246014620460592F5F72AFB4FF0874159
:10B35000F5F730FC0746F5F7F3FDF5F7D7FB0146A7
:10B36000044638460694F5F71BFB4FF08741F5F786
:10B3700021FC00210790F5F7B1FD002800F0F680D0
:10B380000327204600210DF11808013FF5F7A6FD1F
:10B3900040B158F8044D00212046013FF5F79EFDCD
:10B3A0000028F6D1924B02200090019305A83B465D
:10B3B00029464A4600F066FA002E07460DDA95E85F
:10B3C0000C0002F1004103F1004229606A6047422B
:10B3D00003E00023286000274B60384609B0BDE831
:10B3E000F08F0146F5F7DCFA002768602860F4E783
:10B3F0004FF48841C3F23571F5F7D2FA4AF20831B9
:10B40000C2F685610446F5F7CBFA0146286020466E
:10B41000F5F7C6FA4AF20831C2F68561F5F7C0FAC7
:10B4200001276860D9E701F0B1F94FF68411C3F63E
:10B4300022718046F5F7BEFB4FF07C51F5F7B2FA6A
:10B44000F5F77EFD0746F5F761FB4FF47861C3F62B
:10B45000C9718346F5F7AEFB01464046F5F7A0FA01
:10B4600044F243418146C3F235715846F5F7A2FBD9
:10B470001F2F8246514648461FDC5E4B7A1E53F80A
:10B48000223024F0FF029A4217D0F5F789FA80465D
:10B49000C5F8008041464846F5F782FA5146F5F76F
:10B4A0007FFA002E686098DA08F1004800F1004148
:10B4B000C5F8008069607F428FE7F5F771FAE31500
:10B4C0008046C0F3C750191A0829E1DD4FF48841BE
:10B4D000C3F2357158460393F5F76CFB824651462B
:10B4E0004846F5F75DFA044621464846F5F758FA0E
:10B4F0005146F5F755FA4AF208318146C2F68561A0
:10B500005846F5F757FB4946F5F74AFA8246514641
:10B510002046F5F745FA039BC0F3C7528046981AB8
:10B52000192841DCC5F80080A146B3E7F5F73AFADF
:10B530004FF47D6724F00F04C3F6C977BC4206467A
:10B5400016D044F24341C3F23571F5F72BFA0146A8
:10B5500028603046F5F724FA44F24341C3F23571CE
:10B56000F5F720FA4FF0FF37686036E7032719E751
:10B570004FF48841C3F23571F5F714FA4AF20831F5
:10B58000C2F685610446F5F70DFA014628602046AB
:10B59000F5F706FA4AF20831C2F68561F5F702FAC4
:10B5A0004FF0FF37686018E74FF42341C2F685611A
:10B5B0005846F5F7FFFA804641462046F5F7F0F980
:10B5C000814649462046F5F7EBF94146F5F7E8F99B
:10B5D00043F232110446C2F28D415846F5F7EAFAB9
:10B5E0002146F5F7DDF98246514648464DE700BF52
:10B5F00028FE0008A8FD000820F00042B2F1FF4F2D
:10B60000F8B50446034646D2002A42D0002852DB51
:10B61000C415B2F5000F09D210F4000553D15B0038
:10B6200001351902FBD5C5F10100241823F07F4133
:10B630007F3C21F40006E20746F4000048BF4000CA
:10B6400043004FF08072002760109A423C462CDD88
:10B650005B004FF400021825A61851089E4205F120
:10B66000FF3502DCB4189B1BBF185B0062189A42BE
:10B6700002DC9B1A54187F185B004A08013DEBD18D
:10B6800013B107F001017F187C1004F17C5303EB28
:10B69000C0542046F8BD0146F5F78CFA0146204615
:10B6A000F5F780F904462046F8BD4FF0007403F129
:10B6B0007F431746CCE70146F5F772F90146F5F7E7
:10B6C0002DFB0446E5E70120AFE700BF2DE9F84375
:10B6D00020F00046B6F1485F05460F465BDAF5F705
:10B6E0002FFC002800F0CA8029462846F5F762FAA8
:10B6F0004DF24E71CAF647510446F5F75BFA47F230
:10B70000F641C3F20F11F5F74DF92146F5F752FA5C
:10B710004FF27C21C3F29341F5F742F92146F5F748
:10B7200049FA40F60151C3F2D071F5F73BF92146D1
:10B73000F5F740FA40F66131C3F6B621F5F730F976
:10B740002146F5F737FA4AF6AB21C3F62A51F5F749
:10B7500029F92146F5F72EFA804620464FF07C5114
:10B76000F5F728FA414606462046F5F723FA39460A
:10B7700004462846F5F71EFA01462046F5F710F96B
:10B7800001463046F5F70CF901464FF07E50F5F7CB
:10B7900007F9BDE8F8830146F5F70CFA4DF24E7152
:10B7A000CAF647510446F5F705FA47F2F641C3F2E7
:10B7B0000F11F5F7F7F82146F5F7FCF94FF27C2168
:10B7C000C3F29341F5F7ECF82146F5F7F3F940F6AB
:10B7D0000151C3F2D071F5F7E5F82146F5F7EAF922
:10B7E00040F66131C3F6B621F5F7DAF82146F5F7F0
:10B7F000E1F94AF6AB21C3F62A51F5F7D3F8214611
:10B80000F5F7D8F949F69913C3F699639E42804635
:10B81000A3DD0020C3F64870864227DC06F17F4690
:10B820004FF07E503146F5F7BBF8814620464FF089
:10B830007C51F5F7BFF93146F5F7B2F841460646B7
:10B840002046F5F7B7F9394604462846F5F7B2F928
:10B8500001462046F5F7A4F801463046F5F7A0F872
:10B8600001464846F5F79CF8BDE8F8834FF000091B
:10B870000026C3F63879C3F69066D7E74FF07E50BE
:10B88000BDE8F8832DE9F04FDFB00C930C9D224BFF
:10B89000689C0A91691ED61E48BF161D834653F840
:10B8A0002400F71027EAE7730890049104980D9399
:10B8B000089DDC43DDF834C002EBC4024119079255
:10B8C000C0EB0C0750D47E18699BC7EB0609013604
:10B8D000002F03EB870522AC09F0010AC0F2FE82BB
:10B8E0002868F5F713F90137B74220604FF00408D4
:10B8F0003AD0BAF1000F26D0002FC0F2F18255F8ED
:10B900000800F5F703F90137B74244F8080008F1D9
:10B91000040818D128E000BF4001010855F80800CC
:10B92000F5F7F4F8013708F1040944F8080013D4D6
:10B9300055F80900F5F7EAF80137B74244F809006D
:10B9400009F1040810D0002FE8DA0020013708F1CF
:10B95000040944F80800EBD501370020B74244F849
:10B96000090009F10408EED1089A002AC0F24585C1
:10B9700008990C9E8D004AAB5C19039549AF02945F
:10B980004FEA860A049A002AC0F296820DF18808CE
:10B9900008EB860555F8041CAAF10403DBF8000047
:10B9A000C3F38009F5F706F901460020F4F7FAFF22
:10B9B0000424043D544580462BD0B9F1000F0DD02E
:10B9C00055F8041DDBF80400F5F7F4F8014640468D
:10B9D000F4F7E8FF0824544580461AD055F8041CB3
:10B9E0005BF80400F5F7E6F801464046F4F7DAFFA5
:10B9F0000434804655F8081C5BF80400F5F7DAF8C3
:10BA000001464046F4F7CEFF0434083D54458046D5
:10BA1000E4D1029847F8048F01368742B2D1039FE0
:10BA20000EA9CE190996089EB2005EAB9D18002E95
:10BA3000029255F8509C7DDD0DF5947C4FF06E51CF
:10BA400048460DACA7180CEB0205F5F7B3F8F5F76F
:10BA500077FAF5F75BF84FF087410190F5F7AAF810
:10BA600001464846F4F79CFFF5F76AFA0EAC2060F1
:10BA70000198014655F8040DF4F794FFBC42814645
:10BA8000C7F3800156D0E9B14FF06E51F5F792F847
:10BA9000F5F756FAF5F73AF84FF087410190F5F7C8
:10BAA00089F801464846F4F77BFFF5F749FA019A11
:10BAB0000FAC2060114655F8040DF4F773FFBC423B
:10BAC000814637D04FF06E514846F5F773F8F5F7D9
:10BAD00037FAF5F71BF84FF087418046F5F76AF81B
:10BAE00001464846F4F75CFFF5F72AFA41466060E4
:10BAF00055F8040DF4F756FF4FF06E518146F5F7F7
:10BB000059F8F5F71DFAF5F701F84FF0874180462F
:10BB1000F5F750F801464846F4F742FFF5F710FAFA
:10BB20004146A06055F8040DF4F73CFF0834BC42D0
:10BB30008146C7D10799484600F0A2FE4FF07851E0
:10BB40000546F5F737F800F025FE4FF08241F5F78E
:10BB500031F801462846F4F723FF0746F5F7F0F9D8
:10BB60008146F4F7D3FF01463846F4F719FF0799E9
:10BB70000746002940F33981721E0EAC079D54F828
:10BB80002230C5F1080043FA00F101FA00F0C5F1D6
:10BB900007041B1A43FA04F40DF1380C89444CF8DD
:10BBA0002230002C55DD002E09F1010940F394816B
:10BBB000029D0EABDDF808C053F8042B281F0DF1D1
:10BBC000380E00250EEB0C01C0F3800022B1C2F547
:10BBD000807243F8042C01258B4226D060B10F9A65
:10BBE0000433002D40F0F38022B1C2F5807543F894
:10BBF000045C01258B4218D053F8042B002D40F033
:10BC0000EC80C2F5807012B143F8040C012553F8A2
:10BC1000042B002D40F0DB80C2F58070002AE9D0B3
:10BC200001258B4243F8040CE6D1079900290DDD6C
:10BC3000012900F0E280022908D1701E0DF1380EB2
:10BC40005EF8202002F03F034EF82030022C00F076
:10BC5000E08038460021F5F741F9002800F0F38034
:10BC60000898751EA84225DC029B0DF1380E0EEBDC
:10BC700003010B46DDF824C053F8042DCCEB010082
:10BC8000011F6345C1F3800011D030B153F8041D8A
:10BC9000DDF824E00A43734509D0099F53F8040DE9
:10BCA00053F8041D0243BB4242EA0102F6D1002AC6
:10BCB00040F01A81089F0EAD781E55F82020002A0A
:10BCC00040F0108105EB8004012354F8041D01337A
:10BCD0000029FAD0F018771C87420B9075DCDDF84C
:10BCE00010E00D9D0B9B0C9C0EEB0702DDF808C0CD
:10BCF000699F991B06EB05094AA8A61922AB07EB19
:10BD0000890900EB0C05571C8A0003EB860102959C
:10BD100006920591002659F8040FF4F7F7FE059CEA
:10BD2000A051049800285EDB22AD05EB8702AAF142
:10BD30000403C3F3800452F8041CDBF800000394EE
:10BD4000141FF4F737FF01460020F4F72BFE4FF0E5
:10BD50000408D04505462DD0039971B154F8041D4F
:10BD6000DBF80400F4F726FF01462846F4F71AFE34
:10BD70004FF00808D04505461CD054F8041C5BF869
:10BD80000800F4F717FF01462846F4F70BFE08F108
:10BD90000408054654F8081C5BF80800F4F70AFF8D
:10BDA00001462846F4F7FEFD08F10408083CD0459A
:10BDB0000546E2D1DDF808E0069804364EF8045F47
:10BDC00001378642CDF808E0A5D10B9E2CE6C2F1E2
:10BDD000FF0243F8042C01250CE7C2F1FF0543F8EC
:10BDE000045C012513E70025E4E75ED1701E0DF128
:10BDF000380E5EF820301C12D3E6711E0DF1380C9F
:10BE00005CF82100022C00F07F024CF821207FF426
:10BE100020AF39464FF07E50F4F7C2FD0746002DA3
:10BE20003FF417AF07994FF07E5000F029FD01460F
:10BE30003846F4F7B5FD074638460021F5F74EF8C9
:10BE400000287FF40DAF0294079C38466142CDF87C
:10BE5000109000F015FD4FF087410546F5F75CF8AE
:10BE6000002800F0D2824FF06E512846F4F7A2FE6F
:10BE7000F5F766F8F4F74AFE4FF087410746F4F706
:10BE800099FE01462846F4F78BFDF5F759F80EA9FF
:10BE900041F826003846F5F753F8079A013608327C
:10BEA0000EAC079244F8260034E04FF07C51F5F7D1
:10BEB00033F858B90024CCE64FF00008029847F850
:10BEC000048F013687427FF45DADA8E50224002E81
:10BED00009F101093FF76CAE0025A6E6002002E556
:10BEE000002010E50123F5E6079A0EAE56F825303E
:10BEF000083ACDF8109002940792002B40F08E8201
:10BF000006EB85042E4654F8045D013E083A002DE8
:10BF1000F9D007924FF07E50079900F0B1FC002E47
:10BF20000446C0F2AC804FEA860AC6EB867B0EAFB1
:10BF30004FEA8B095744C9F100034AA9386801EB5D
:10BF40000A08C3F3800BF4F7E1FD2146F4F732FE53
:10BF50004FF06E51C8F800002046F4F72BFEA9F10F
:10BF600004096FF0030ACA45054631D0BBF1000F42
:10BF70000BD057F8040CF4F7C9FD2946F4F71AFE64
:10BF80006FF0070A48F8040C1AE057F80A00F4F7B3
:10BF9000BDFD2946F4F70EFE4FF06E5148F80A0039
:10BFA0002846F4F707FEAAF1040405463859F4F7C9
:10BFB000ADFD2946F4F7FEFDAAF1080A48F8040091
:10BFC00028464FF06E51F4F7F5FDCA450546DCD121
:10BFD000701CDFF84C94DDF820A003900027059634
:10BFE000BAF1000FC0F20582002FC0F202820026D3
:10BFF00000241AF0010F354620D0D8F80010D9F8E7
:10C000000000F4F7D7FD01462046F4F7CBFC0125EC
:10C01000AA45044626DB0426BD420FDD22E0BB45CF
:10C0200020DC58F8021059F80200F4F7C3FD01466D
:10C030002046F4F7B7FCBD42044613DC58F806105E
:10C0400059F80600F4F7B6FD01462046F4F7AAFCBD
:10C0500005F1010B06F104020235DA45044602F14E
:10C060000406DCDA5EABDDF80CC003EB87010137B8
:10C07000674541F8A04CA8F10408B1D1059E689C21
:10C08000032C16D8DFE814F085011F011F011B00E7
:10C0900000230299002900F00B81379C369804F1A7
:10C0A00000420A9C00F1004503F1004325606260F4
:10C0B000A360049D05F007005FB0BDE8F08F002E7F
:10C0C000E6DD06F1FF3836AF07EB88094D4655F837
:10C0D00004290DF1D40AD5F808B01046594601924A
:10C0E000F4F760FC804641460198F4F759FC01469C
:10C0F0005846F4F757FC5545C9F38003A860C5F8C6
:10C10000048044D0BBB155F80429D5F808B01046D6
:10C1100059460192F4F746FC01998046084641468B
:10C12000F4F73EFC01465846F4F73CFC5545C5F88B
:10C130000480A8602BD02C4654F80439D4F808B0F9
:10C14000184659460193F4F72DFC80464146019864
:10C15000F4F726FC01465846F4F724FCC4F80480A2
:10C16000A06055F804BC251FD5F808805846414604
:10C17000F4F718FC044621465846F4F711FC014632
:10C180004046F4F70FFC55456C60A860D3D1012EF2
:10C190007FF77EAF4D4655F804B9C7EB090ED5F8C9
:10C1A00008A058465146AEF10409F4F7FBFB80465F
:10C1B00041465846F4F7F4FB01465046F4F7F2FBCB
:10C1C000BD42C9F38009C5F80480A86043D0B9F125
:10C1D000000F15D055F804A9D5F8089050464946E7
:10C1E000F4F7E0FB804641465046F4F7D9FB0146A0
:10C1F0004846F4F7D7FBBD42C5F80480A8602AD0B2
:10C200002C4654F804A9D4F8089050464946F4F74F
:10C21000C9FB804641465046F4F7C2FB01464846FA
:10C22000F4F7C0FBC4F80480A06055F8049C251FF7
:10C23000D5F8088048464146F4F7B4FB0446214649
:10C240004846F4F7ADFB01464046F4F7ABFBBD4270
:10C250006C60A860D4D1013607EB860708353E46EE
:10C260007A1B131F56F8041D0020C3F38007F4F750
:10C2700099FBAE4203463FF40CAF3FB156F8041DA4
:10C28000F4F790FBAE4203463FF403AF184656F86E
:10C29000041C341FF4F786FB083E54F8041CF4F722
:10C2A00081FBAE42F3D10299034600297FF4F5AE3B
:10C2B000DDF828C036993798CCF80010CCF8040087
:10C2C000CCF80830F5E60023002E29DB36AF751CCC
:10C2D00007EB85042546E21B55F8041DA2F1040E68
:10C2E0000020CEF38008F4F75DFBBD42034617D073
:10C2F000B8F1000F06D055F8041DF4F753FBBD420A
:10C3000003460DD0184655F8041C2C1FF4F74AFBC1
:10C31000083D54F8041CF4F745FBBD42F3D1034635
:10C320000299002967D003F10040DDF828C01946C2
:10C33000CCF800003698F4F733FB002E034621DDDD
:10C3400036AF07EB8606F51B2A1F3799C2F3800725
:10C35000F4F728FB37ACB442034613D037B1616819
:10C36000F4F720FB38ACB44203460BD0184654F81F
:10C37000041FF4F717FB54F8041FF4F713FBB4423F
:10C38000F5D10346029909B103F100430A9C6360A9
:10C390008FE6002E40DB36AF013607EB8600054600
:10C3A000C21B55F8041D0020141FF4F7FBFABD4210
:10C3B000C4F38006034615D036B155F8041DF4F7D2
:10C3C000F1FABD4203460DD0184655F8041C2C1F47
:10C3D000F4F7E8FA083D54F8041CF4F7E3FABD4218
:10C3E000F3D10346029909B103F100430A9C23608B
:10C3F0005FE6002436E6184697E7DDF830E0900067
:10C4000003904FEA8E0AFFF70ABB2846F4F798FD1F
:10C410000EAB43F826007DE50023E3E72E4679E5E1
:10C420004C0101082DE9F84320F00043B3F1485FC7
:10C4300004460F46904603DAF4F782FD002859D0EF
:10C4400021462046F4F7B6FB21460546F4F7B2FB39
:10C450004CF6D311C2F62E7106462846F4F7AAFB15
:10C4600042F63471C3F2D721F4F79AFA2946F4F769
:10C47000A1FB4EF61B71C3F23861F4F793FA29461B
:10C48000F4F798FB40F60151C3F65011F4F788FA1F
:10C490002946F4F78FFB48F68901C3F60841F4F703
:10C4A00081FA8146B8F1000F27D04FF07C51384611
:10C4B000F4F780FB494680463046F4F77BFB0146A3
:10C4C0004046F4F76DFA2946F4F774FB3946F4F761
:10C4D00067FA4AF6AB210546C3F62A613046F4F7FF
:10C4E00069FB01462846F4F75DFA01462046F4F759
:10C4F00057FA04462046BDE8F88301462846F4F77B
:10C5000059FB4AF6AB21C3F62A61F4F749FA3146E2
:10C51000F4F750FB01462046F4F744FA044620465F
:10C52000BDE8F8830020704700210020C7F6F871AD
:10C53000704700BF2DE9F04120F00045B5F1A14F53
:10C54000044606460DDBB5F1FF4F00F39C80002842
:10C5500040F6DB7440F3D480C3F6C9742046BDE8CE
:10C56000F0814FF6FF73C3F6DF639D4200F3A280B4
:10C57000B5F1445FC0F28E804FF0FF372146204670
:10C58000F4F718FB01468046F4F714FB46F6D71182
:10C59000C3F685410546F4F70DFB4DF65921C3F668
:10C5A0004B51F4F7FFF92946F4F704FB46F6353111
:10C5B000C3F68851F4F7F6F92946F4F7FBFA42F688
:10C5C0006E61C3F6BA51F4F7EDF92946F4F7F2FAC1
:10C5D00044F62511C3F61261F4F7E4F92946F4F79D
:10C5E000E9FA4AF6AB21C3F6AA61F4F7DBF9414652
:10C5F000F4F7E0FA4AF221218046CBF6155128469D
:10C60000F4F7D8FA4FF26B11C3F66E51F4F7C8F98C
:10C610002946F4F7CFFA48F29571C3F69D51F4F725
:10C62000BFF92946F4F7C6FA48F63861C3F6E35174
:10C63000F4F7B6F92946F4F7BDFA4CF6CD41C3F646
:10C640004C61F4F7ADF92946F4F7B4FA7B1C0146C6
:10C65000404658D0F4F7A6F92146F4F7ABFA494B17
:10C6600053F82710F4F79CF92146F4F799F901469D
:10C67000454850F82700F4F793F9002E3DDB0446B7
:10C680002046BDE8F0810146F4F78CF904462046C7
:10C69000BDE8F0814FF2CA21C7F24911F4F782F9DF
:10C6A0004FF07E51F4F742FC00283FF465AF20467E
:10C6B000BDE8F08100F06AF84FF6FF71C3F697719C
:10C6C0008D4204464FF6FF7228DCC3F62F72954266
:10C6D00046DC0146F4F766F94FF07E51F4F760F955
:10C6E0004FF0804105462046F4F75CF901462846A4
:10C6F000F4F714FB0027044640E700F100442DE75F
:10C70000CBF6C9742AE7F4F74DF92146F4F752FA4B
:10C7100001462046F4F744F904461FE7C4F21B0221
:10C72000954214DC4FF07F51F4F73AF94FF07F5106
:10C7300005462046F4F73EFA4FF07E51F4F732F901
:10C7400001462846F4F7EAFA0227044616E70020D5
:10C750002146CBF68070F4F7E1FA032704460DE793
:10C760004FF07E51F4F71CF94FF07E5107462046FA
:10C77000F4F718F901463846F4F7D0FA01270446D1
:10C78000FCE600BF780101088801010820F00040A4
:10C79000704700BFF8B520F00046F50D7F3D162D1F
:10C7A000014604461BDC002D074620DB4FF6FF73D5
:10C7B000C0F27F0343FA05F606420ED04FF2CA21BB
:10C7C000C7F24911F4F7EEF80021F4F7AFFB18B106
:10C7D000002C1BDB27EA060421460846F8BDB6F10B
:10C7E000FF4FFAD3F4F7DEF801460846F8BD4FF2E2
:10C7F000CA21C7F24911F4F7D5F80021F4F796FBE6
:10C800000028E9D0002C07DB0024E5E74FF4000006
:10C8100040FA05F56719DDE70021CBF68071002E9F
:10C8200018BF0C46D8E700BF08B902207047B0F126
:10C83000004FFAD0A0F500026FF001439A4201D8F0
:10C840000420704700F1FF419942F9D94FF6FE7379
:10C85000421EC0F27F039A4201D80320704700F1C4
:10C8600000414A1E9A42F8D9B0F1FF4F05D010F5A9
:10C87000000F14BF0020012070470120704700BF47
:10C8800038B530F00044034602460D460FD0B4F1EF
:10C89000FF4F0ED2B4F5000F11D3E40D6419FE2C36
:10C8A00033DC002C1BDD22F0FF4141EAC453184663
:10C8B00038BD0146F4F776F80346184638BD4FF008
:10C8C0009841F4F777F943F6B041CFF6FF718D4206
:10C8D000034612DBC0F3C7540246193CDEE714F1ED
:10C8E000160F21DA4CF25032954219460EDC44F212
:10C8F0006020C0F6A25000F023F844F26021C0F698
:10C90000A251F4F757F90346D1E719464FF2CA206E
:10C91000C7F2491000F014F84FF2CA21C7F24911CA
:10C92000F4F748F90346C2E722F0FF4304F1190087
:10C9300043EAC0504FF04C51F4F73CF90346B6E7D8
:10C9400001F0004120F00040084370472DE9F0411C
:10C95000274C84B025680746D5F84841002C41D0C3
:10C9600066681F2E1CDD234810B94FF0FF301FE012
:10C970004FF4C870039102920193AFF300800399C2
:10C980000446029A019B0028EFD0D5F848610020A8
:10C9900060602660C5F84841C4F88801C4F88C017D
:10C9A000656847B9A81C013544F82010656000206F
:10C9B00004B0BDE8F081012000FA05F0D4F88861E8
:10C9C00004EB85080643022FC8F88820C4F8886164
:10C9D000C8F80831E6D1D4F88C3143EA0002C4F833
:10C9E0008C21DFE705F5A674C5F84841B8E700BF1C
:10C9F000A00201080000000000210A2201F028B86E
:10CA00002DE9F84FDDF828B081468A4698469AB15C
:10CA100093B11646002503E00FD0651CAE420BD93A
:10CA20007419640808FB04A748463946D84700280B
:10CA3000F2DA2646AE42F3D800273846BDE8F88F32
:10CA400040F2D053C2F2000318687047114B124AEB
:10CA500070B5981A831018D0591E02EB83040D4646
:10CA600054F8042D01F00106904775B126B154F831
:10CA7000040D8047013D08D054F8043D9847013D1E
:10CA800054F8041D8847013DF6D1BDE8704003F01D
:10CA90000FBC00BFC8020108C4020108F8B5204F4E
:10CAA000204C381B871017D07A1E2368012502F00E
:10CAB00001069847AF420FD02EB154F8041F02254B
:10CAC0008847AF4208D0606880470235A268261DBB
:10CAD00090470834AF42F6D1134F144C03F0E2FBF9
:10CAE0003B1B9F1018D07D1E216805F00106012513
:10CAF0008847AF4211D02EB154F8040F0225804769
:10CB0000AF420BD0626890470235A368261D984754
:10CB10000834AF42F6D1F8BDF8BDF8BDF8BD00BF8E
:10CB2000BC020108BC020108C4020108BC020108E1
:10CB30000F2A2DE9F00340F2A18041EA00039B0790
:10CB400040F09E800C68A2F1100504604B68AC4672
:10CB500043608C68BCF10F0F8460CC68C5F300158E
:10CB6000C46000F1100301F110042BD975B12568E0
:10CB7000ACF1100C1D6065685D60A5689D60E5689E
:10CB80001034DD601033BCF10F0F1BD9276804F19E
:10CB900010061F60676803F110055F60A768ACF1BD
:10CBA000200C9F60E768DF6024691C61776806F1EC
:10CBB00010046F60B7682033AF60F668BCF10F0FE8
:10CBC000EE60E3D8A2F1100828F00F0302F00F0482
:10CBD00003F1100C032C00EB0C0301EB0C0851D9F2
:10CBE000211F4FEA9109444608EB890C54F8046B65
:10CBF000C8EB0C010CF1040C1D46644545F8046BB0
:10CC0000C1F3800112D029B154F8041B644545F8E2
:10CC1000041B0BD0274657F8041B2E4646F8041B6E
:10CC200064686C603C1D351D6445F3D109F1010C4D
:10CC30004FEA8C0902F0030208EB09014B44D2B120
:10CC40000D789A18DC4303F8015B1419934204F041
:10CC5000010410D02CB111F8014F03F8014B93429D
:10CC600009D04D781C4604F8015B8D7802315D7067
:10CC7000631C9342F5D1BDE8F00370470346DEE73D
:10CC80000346DDE741462246D9E700BFF0B48407FA
:10CC9000034600F08D80541E002A00F08780E507CF
:10CCA000CEB211D41A4602F8016B1346154692070C
:10CCB00010D0621E002C79D003F8016B14469A073D
:10CCC0001D4607D0013CEDE7034603F8016B9A07C8
:10CCD0001D46F7D1032C52D9CEB246EA06270F2CB7
:10CCE00047EA07432DD9A4F1100217460F2FC2F3CC
:10CCF00000162B606B60AB60EB6005F1100216D97B
:10CD00003EB1103F136053609360D36010320F2F19
:10CD10000DD9203F02F11006136053609360D36079
:10CD2000136153619361D36120320F2FF1D8A4F1C5
:10CD3000100222F00F0204F00F041032032C1544ED
:10CD40001DD9271F3E462A46032E42F8043BC7F34F
:10CD500080070DD927B1043E032E42F8043B07D9C2
:10CD6000174647F8043B083E53603A1D032EF7D898
:10CD7000231F23F00302131D04F00304ED18ACB1CC
:10CD8000C9B2EA432C1905F8011BA318A54203F008
:10CD900001020BD01AB105F8011BA54206D02B46A3
:10CDA00003F8011B69705D1CA542F8D1F0BC704707
:10CDB000054614468EE700BF830770B5064614D1BA
:10CDC0000368A3F1013222EA030010F0803F0CD186
:10CDD000331D1A4653F8044BA4F1013525EA040427
:10CDE00014F0803FF5D0104600E0304603782BB1B8
:10CDF000421C147810460132002CFAD100F080F861
:10CE0000304670BDC9B2F0B400294BD082070FD0B4
:10CE10000278002A71D0914242D0431C05E013F8F9
:10CE2000012B002A3BD091423AD09A071846F6D1FE
:10CE3000036841EA0127A3F1013222EA030212F05A
:10CE4000803F47EA07471CD17B40A3F1013222EA29
:10CE5000030313F0803F14D1021D02E014F0803F61
:10CE60000FD1104652F8043BA3F1013687EA0304C0
:10CE700026EA0303A4F1013513F0803F25EA0404F8
:10CE8000ECD00278002A38D0914209D0431C01E04E
:10CE9000914205D0184613F8012B002AF8D110460C
:10CEA000F0BC704783070BD00278002AF8D0431CEF
:10CEB00003E0017801330029F2D099071846F8D130
:10CEC0000168A1F1013323EA010212F0803F0AD187
:10CED000031D184653F8041BA1F1013424EA010292
:10CEE00012F0803FF5D00378002BD9D0421C117886
:10CEF000104601320029FAD1D2E71046D0E700BF30
:10CF000080EA0102844612F0030F4FD111F0030FA3
:10CF100032D14DF8044D11F0040F51F8043B0BD001
:10CF2000A3F101329A4312F0803F04BF4CF8043B56
:10CF300051F8043B16D100BF51F8044BA3F1013264
:10CF40009A4312F0803FA4F101320BD14CF8043B1C
:10CF5000A24312F0803F04BF51F8043B4CF8044B4D
:10CF6000EAD023460CF8013B13F0FF0F4FEA3323BE
:10CF7000F8D15DF8044B704711F0010F06D011F89D
:10CF8000012B0CF8012B002A08BF704711F0020F8B
:10CF9000BFD031F8022B12F0FF0F16BF2CF8022B76
:10CFA0008CF8002012F47F4FB3D1704711F8012B99
:10CFB0000CF8012B002AF9D1704700BF20F00301C3
:10CFC00010F00300C0F1000051F8043B00F1040C24
:10CFD0004FEACC0C6FF000021CBF22FA0CF2134394
:10CFE0004FF0010C4CEA0C2C4CEA0C4CA3EB0C025D
:10CFF00022EA030212EACC1204BF51F8043B0430C7
:10D00000F4D013F0FF0F1FBF013013F47F4F013036
:10D0100013F47F0F18BF0130704700BFF0B4002A2F
:10D0200063D0344B04461B6814F8010B571E1D18BF
:10D030006E7807F0010706F00305012D58D011F8AE
:10D04000015B5E19767806F00306012E08BF2035D5
:10D05000401B4BD1002D49D0013A47D02FB314F8D3
:10D06000010B1D186E7806F00305012D11F8015B08
:10D0700008BF20305E19767806F00306012E08BF3F
:10D080002035401B32D18DB3013A0ED12EE011F87C
:10D09000012B9E18767806F00306012E08BF203279
:10D0A000801A23D112B36A1E20D014F8010B1D1868
:10D0B0006E7806F00305012D11F8015B08BF2030E2
:10D0C0005E19767806F00306012E08BF2035401B56
:10D0D0000CD15DB114F8010B551E1A18567806F0E4
:10D0E0000302012AD3D12030D1E71046F0BC7047AB
:10D0F0002030A4E7A401002041EA00039B07F0B41C
:10D1000074D1032A72D90C4654F8045B161FA5F19A
:10D11000013727EA050717F0803F0346C6F3800C66
:10D1200031D10346032E324643F8045B2AD9BCF1C1
:10D13000000F0AD0214654F8045BA5F1013626EA17
:10D14000050616F0803F18D01DE0264656F8045B11
:10D150002146A5F1013727EA050717F0803F12D1D4
:10D1600043F8045B65683146A5F1013626EA0506F9
:10D17000043A0C1D16F0803F05D1043A032A43F807
:10D18000045BE2D821467AB30D78013A03F8015BDB
:10D190009DB112F0010F1C462AD1234622B311F88B
:10D1A000015F013A03F8015B3DB111F8015F013AFB
:10D1B00065705C1C2346002DEFD1AAB100219C189C
:10D1C000DA4303F8011BA218A34202F001020BD0BC
:10D1D0001AB103F8011BA34206D01A4602F8011B3C
:10D1E0005970531CA342F8D1F0BC70470346CAE7FC
:10D1F00011F8015F1C4604F8015B013A2346002D3B
:10D20000CBD1DAE72DE9F00701273C4600254FF0A6
:10D21000FF3663198B4200EB060C0DD21CF804A0FC
:10D2200010F80380D0452ED201241D469F1B6319A0
:10D230008B4200EB060CF1D34FF0010A1760544605
:10D2400000254FF0FF3C6319994200EB0C080ED902
:10D2500018F8048010F80390C1451AD901241D461E
:10D26000CCEB030A6319994200EB0C08F0D80CF1DF
:10D2700001000136B0423CBFBA463046C2F800A0B9
:10D28000BDE8F00770470BD001272E463C46ED194C
:10D29000BFE709D04FF0010AAC4654465544D2E7E7
:10D2A000BC4205D00134B4E7544505D00134CAE787
:10D2B00027461D460124ACE7A2461D460124C2E7CD
:10D2C0002DE9F04FADF2244D15460646894610462D
:10D2D000194607AA1C46FFF795FF07AB82460DF2D9
:10D2E0001C411A1D5C6008338B425460F9D114B3A1
:10D2F00001232F78611E08A8A34240F8271001EAF5
:10D30000030218D032B16A7802234F1EA34240F8BC
:10D31000227010D0B046A4465C1C15F803E0CE1A6B
:10D320002A5D02330F1B634540F82E6040F82270DF
:10D33000F2D146466446079928466918524600F0DD
:10D3400045FC002840F0B6800AF1FF3E05EB0E0CCC
:10D35000CDF808E0CAF1010E834604F1FF38CDF89C
:10D360000CC0CDF814E00746CDF810A04A46009551
:10D37000019408E027B1079FBB4201D20199CB1B62
:10D380009B4400272246019CB0185C440021A21A4D
:10D3900000F07CFB002840F08780002C00F08480A7
:10D3A000301910F8013C08A951F82330002BE1D1C5
:10D3B000049B9F4228BF3B46434527D2DDF800909F
:10D3C00006EB0B0119F80350CA5C09EB0300954208
:10D3D00066D1DD43454415F0010F024613D00133F9
:10D3E000434513D24078CD5C013285420BD057E0E3
:10D3F00012F8010FCD5C854252D1013312F8010FB2
:10D40000CD5C85424CD101334345F1D3DDF810901A
:10D41000029B4F4528BF4B4639D2DDF808C0DDF8E6
:10D42000009006EB0B0519F80C1015F80C00814262
:10D4300040F0C080DDF80CE009EB070ACAEB0E01F2
:10D44000C80772461ED5DDF8089009F1FF31DDF8F6
:10D450000C90685C19F801CC09F1FF32844516D1B3
:10D460000B460FE012F8019C15F800E04A1EF1454A
:10D470000DD10346013815F800C011F8011C6145B3
:10D4800005D10346581E524502F1FF31EAD101375A
:10D490009F4200F29180079F019ABB44D71B71E71E
:10D4A000DDF814E0F3446BE7002009B00DF5806D62
:10D4B000BDE8F08FCAEB0400504538BF5046CAF1B2
:10D4C0000102431C0AF1FF3C05EB0A0704F1FF3B94
:10D4D000019200944A460793B1464FF00008644613
:10D4E0003E46009909EB020008EB0107BA1A002139
:10D4F00000F0CCFA0028D7D1002FD5D009EB0700D7
:10D5000010F8013C08AA52F8230000284AD1DA4555
:10D5100009EB08002AD210F80A303178994218BF76
:10D52000534642D16FEA0A0303EB0B01C9073246A7
:10D53000534618D50AF101035B4517D2324612F85B
:10D54000011F10F803E08E450DD02EE012F8011FE8
:10D5500010F803C08C4528D1013312F8011F10F8D0
:10D5600003E08E4521D101335B45EFD3621C234696
:10D570009BD0295D025D914213D1E10709D5631E5D
:10D58000E95CC25C914204D00BE0E95CC25C914270
:10D5900007D15A1E002B88D0A95C825C023B9142C5
:10D5A000F3D0079880443A469BE7DDF804C0E04496
:10D5B0009844F8E7049B6AE706EB0B0075E700BFA9
:10D5C0002DE9F04F037889B080460D46002B00F01E
:10D5D00065810A789AB184460131012602E011F88A
:10D5E000012B5AB1934214BF002606F001061CF825
:10D5F000013F0C46002BF2D1207820B936B14046CD
:10D6000009B0BDE8F08F4FF00008F8E708F101001D
:10D610002978FFF7F7FB641B06460028F3D0012C9E
:10D6200000F0B580A044404594BFC0EB0807012737
:10D630001F2C06D939462A462346FFF741FE80466D
:10D64000DDE7214607AA2846FFF7DCFD079903908E
:10D6500069182846039A00F0B9FA002840F099802A
:10D66000DDF80CC0DDF80C900CF1FF3E05EB0E016F
:10D67000C9F1010C8346CDF808E080460491CDF84D
:10D6800014C03A46B146019508EB040609EB0200C6
:10D690000021B21A00F0FAF90028B4D1002EB2D05D
:10D6A000039B9B4528BF5B469C4227D9019D09EB04
:10D6B000030010F80820E95CE81891425FD1DD43CF
:10D6C0002D1915F0010F024609EB080113D00133A3
:10D6D0009C4213D94078CD5C013285420BD04EE09C
:10D6E00012F8010FCD5C854249D1013312F8010FC8
:10D6F000CD5C854243D101339C42F1D8DDF80CE08A
:10D70000029ADE4540F2CD80019B09EB0805995C49
:10D71000A85C814240F0C580DDF804A0049BDA4497
:10D72000CAEB0301C8071AD5029FDDF810C0791EA5
:10D73000685C1CF8017C0CF1FF33874214D10A4667
:10D740000DE013F801EC2F5C4B1EBE450CD10246D8
:10D7500001382F5C11F8011CB94205D10246501E58
:10D76000534503F1FF31ECD10BF1010B934500F26E
:10D770009A80079A9044C2EB040B324684E7059DD9
:10D7800005EB080B0BEB03084FF0000BF5E78046A9
:10D7900035E7DDF80CA00399CAEB0403534538BF05
:10D7A0005346CAF1010B581C06EB0A0205EB0A08A6
:10D7B000CDF808B03B4607904FF00009019201F107
:10D7C000FF3B37468A4609EB0406F8180021F21A97
:10D7D00000F05CF900287FF416AF002E3FF413AF81
:10D7E000544598BF07EB09002CD9DDF804E098F800
:10D7F00000001EF8093098424AD16FEA0A02111956
:10D80000C9074246534607EB090018D50AF1010340
:10D810009C4217D9424612F8011F10F803C08C45EC
:10D820000DD036E012F8011F10F803E08E4530D11C
:10D83000013312F8011F10F803C08C4529D10133C0
:10D840009C42EFD8BBF1FF3F5B463FF4F8AE15F8C2
:10D850000B1010F80B20914216D11BF0010F0AD0CB
:10D860000BF1FF33E95CC25C914204D00CE0E95C4F
:10D87000C25C914208D15A1E002B3FF4E0AEA95C75
:10D88000825C023B9142F2D00798814433469AE78A
:10D890005346DDF808E0F1449944F7E70C460126C9
:10D8A000AAE6039A60E74E46C844A8E640F2D05381
:10D8B000C2F200031A6801235C3200F001B800BF15
:10D8C000F0B4002825D0074638463E780D4601378B
:10D8D00015F8014B3CB1A642FAD1002BF4D11760E8
:10D8E00007F8013C11E0C6B13D4600E01BB915F850
:10D8F000016B0C46284614F8013B9E42F6D136B126
:10D90000002105F8011C1060781EF0BC70473046FD
:10D91000F9E710680028D6D1F7E716603046F4E73B
:10D920002DE9F00F494C82B0D4F800C001900F46A9
:10D930003C4614F8015B0CEB05004678274606F0E0
:10D940000800C6B2002EF3D12D2D61D02B2D04BFBF
:10D95000244614F8015BB346002B41D1302D43D04F
:10D960000A239A46BBF1000F0CBF6FF000474FF03F
:10D970000047B7FBFAF90AFB1970009000208046B7
:10D980000CE0303DAB421BDD461C05D0C84539D804
:10D9900035D00AFB0858012014F8015B0CEB050692
:10D9A000767806F00407FFB2002FEAD116F00306DE
:10D9B00006D0012E14BF57263726AD1BAB42E3DC41
:10D9C000431C2AD0BBF1000F01D0C8F10008002A87
:10D9D00031D0D0B94046116002B0BDE8F00F7047B9
:10D9E000102BBED1302DBCD12578782D25D0582DC7
:10D9F00023D043BB4FF0080A30255346B2E70098C6
:10DA00008542C6DD4FF0FF30C6E74046611EE2E7C3
:10DA100014F8015B4FF0010B9EE7BBF1000F019979
:10DA20000CBF6FF000404FF0004022230B60002A33
:10DA3000D2D0611ECFE74046CEE74FF0100A65789E
:10DA4000534602348EE79A4630258BE7A401002026
:10DA500070B440F2D054C2F2000406460D4620686D
:10DA6000134631462A4670BCFFF75ABF024B13B12A
:10DA7000024800F005B87047000000004DCA0008D9
:10DA80000146002002460346FEF760BF8307F0B45C
:10DA9000C9B200F09680531E002A00F094800278EC
:10DAA0008A420BD0421CD8071AD512F0030F104639
:10DAB0001CD01478013B01328C4211D1F0BC70476C
:10DAC000002B7CD01278013B8A42F7D014F0030F70
:10DAD000204604F1010209D02478013B8C42EDD0AC
:10DAE00012F0030F104602F10104E9D1032B3FD9D4
:10DAF000046841EA012545EA054585EA0407A7F1DE
:10DB0000013222EA07021E1F041D12F0803FC6F3F5
:10DB100080072DD1032E334629D967B126682046C8
:10DB200085EA0602A2F1013626EA0202043412F066
:10DB3000803F19D01CE020462468061D85EA0402B7
:10DB4000A2F1013424EA020212F0803F10D13468BD
:10DB5000043B85EA0402A2F1013424EA0202341DE6
:10DB600012F0803F304603D1043B032BE3D820461C
:10DB70005D1E23B303788B42A0D0431C0022E8072C
:10DB800014D51C781846012201338C4296D0954258
:10DB9000184603F1010402F102020ED01B788B42F9
:10DBA0008CD020462478431C8C4287D0954218465E
:10DBB00003F1010402F10202F0D100207EE71846D1
:10DBC0007CE7134692E7104678E700BF032AF0B4DB
:10DBD00031D941EA00039C072ED106680F68151F52
:10DBE000031D0C1DBE42C5F3800C24D1032D2A4613
:10DBF0001FD9BCF1000F08D01E68256821461846C1
:10DC000004340433AE4211D015E0214618461C6896
:10DC10000B68051D0E1D9C420DD1314628462E680D
:10DC20000D68043A031D0C1DAE4204D1043A032AC8
:10DC3000EBD8214618461AB303780C78A3420AD1D0
:10DC4000551E0022EB0714D510F8013F11F8014FC3
:10DC50000122A3420DD0181B10E010F8013F11F86B
:10DC6000014FA342F7D110F8013F11F8014FA34231
:10DC7000F1D1AA4202F10202EFD10020F0BC7047BC
:10DC80001046FBE71E1E6464646464640010014077
:10DC9000001010020008014000801002340800400B
:10DCA000380800403C080040400800403404004070
:10DCB000380400403C040040400400409D1F000820
:10DCC000371D0008AF1D0008651D00084D1D000828
:10DCD000351D0008D0073200320032003200320019
:10DCE00032003200C8006400000041455452313215
:10DCF00033340030313233343536373839414243EA
:10DD00004445464748494A4B4C4D4E4F505152535B
:10DD10005455565758595A002D330008B13300084E
:10DD2000713300084D330008893300080D340008B2
:10DD3000393300080000803F00000000A8AAAA3F75
:10DD40000000803F0000803F000080BFB0AA2ABFD3
:10DD5000000080BF0000803F0000803FB0AA2ABFC3
:10DD6000000080BF0000803F00000000A8AAAA3F7A
:10DD7000000080BF0000803F000080BFB0AA2ABF23
:10DD80000000803F0000803F0000803FB0AA2ABF13
:10DD90000000803F0000803F00000000A8AAAA3FCA
:10DDA000000000000000803F000080BFB0AA2ABF32
:10DDB000000000000000803F0000803FB0AA2ABFA2
:10DDC000000000000000803F000080BF0000803F96
:10DDD000000080BF0000803F000080BF000080BFC7
:10DDE0000000803F0000803F0000803F0000803F37
:10DDF0000000803F0000803F0000803F000080BFA7
:10DE0000000080BF0000803F000000000000000014
:10DE1000000000000000803F000000000000000043
:10DE2000000000000000803F000000000000803F74
:10DE30000000803F0000803F000080BF000080BFE6
:10DE4000000000000000803F000000000000803F54
:10DE5000000080BF0000803F0000803F000080BFC6
:10DE6000000000800000803F000000000000803FB4
:10DE7000000080BF0000803F000080BF0000000065
:10DE80000000803F0000803F0000803F0000000055
:10DE90000000803F0000803F00000000000080BFC5
:10DEA000000080BF0000000000000000030100002F
:10DEB00094DD00080400000064DE00080400000097
:10DEC0009CE00008020100003CE0000800010000A6
:10DED000000000000600000034DD0008060000001D
:10DEE000DCDF000801010000000000000400000069
:10DEF0005CE00008060000005CE10008080000008B
:10DF0000BCE10008080000005CDF00080800000019
:10DF1000DCE000080101000000000000000100003A
:10DF200000000000000100000000000004000000EC
:10DF300024DE000806000000C4DD00080001000027
:10DF400000000000020100003CE2000801010000A6
:10DF50000000000000000000000000000000803F02
:10DF6000F704353FF70435BF0000803F0000803FD5
:10DF7000F70435BFF70435BF0000803F0000803F45
:10DF8000F70435BFF704353F0000803F0000803FB5
:10DF9000F704353FF704353F0000803F0000803F25
:10DFA00000000000000080BF000080BF0000803F34
:10DFB000000080BF00000000000080BF0000803F24
:10DFC000000000000000803F000080BF0000803F94
:10DFD0000000803F00000000000080BF0000803F84
:10DFE000D0B35DBF0000003F0000803F0000803FD5
:10DFF000D0B35DBF000000BF000080BF0000803FC5
:10E00000D0B35D3F0000003F0000803F0000803F34
:10E01000D0B35D3F000000BF000080BF0000803F24
:10E0200000000000000080BF0000803F0000803F33
:10E03000000000000000803F000080BF0000803F23
:10E040000000803F00000000000000000000803F52
:10E05000000080BF00000000000000000000803FC2
:10E06000000000000000803F000080BF0000803FF3
:10E07000000080BF000080BF000000000000803F63
:10E08000000000000000803F0000803F0000803F53
:10E090000000803F000080BF000000000000803FC3
:10E0A000000080BF0000803F000080BF0000803F74
:10E0B000000080BF000080BF0000803F0000803F64
:10E0C0000000803F0000803F0000803F0000803F54
:10E0D0000000803F000080BF000080BF0000803F44
:10E0E0000000803F000000BF0000803F0000803F34
:10E0F000000000BF000080BF0000803F0000803FA4
:10E10000000080BF0000003F0000803F0000803F13
:10E110000000003F0000803F0000803F0000803F83
:10E120000000003F000080BF000080BF0000803F73
:10E13000000080BF000000BF000080BF0000803FE3
:10E14000000000BF0000803F000080BF0000803F53
:10E150000000803F0000003F000080BF0000803FC3
:10E16000000000BFD0B35D3F0000803F0000803F53
:10E17000000000BFD0B35DBF0000803F0000803FC3
:10E180000000003FD0B35D3F000080BF0000803F33
:10E190000000003FD0B35DBF000080BF0000803FA3
:10E1A000000080BF00000000000080BF0000803F32
:10E1B0000000803F000000000000803F0000803F22
:10E1C000000080BF0000803F000080BF0000803F53
:10E1D000000080BF000080BF0000803F0000803F43
:10E1E0000000803F0000803F0000803F0000803F33
:10E1F0000000803F000080BF000080BF0000803F23
:10E20000000080BF0000803F0000803F0000803F92
:10E21000000080BF000080BF000080BF0000803F82
:10E220000000803F0000803F000080BF0000803F72
:10E230000000803F000080BF0000803F0000803F62
:10E240000000000000000000000080BF0000803FD0
:10E2500000000000000000000000803F24505542F4
:10E26000582C34312C312C303030332C303030318C
:10E270002C3131353230302C302A31450D0A002412
:10E28000504D544B3235312C3131353230302A310A
:10E29000460D0A0024505542582C34312C312C3074
:10E2A0003030332C303030312C35373630302C3064
:10E2B0002A32440D0A0024504D544B3235312C354E
:10E2C000373630302A32430D0A0024505542582C3C
:10E2D00034312C312C303030332C303030312C3341
:10E2E000383430302C302A32360D0A0024504D5448
:10E2F0004B3235312C33383430302A32370D0A0066
:10E3000024505542582C34312C312C303030332CA1
:10E31000303030312C31393230302C302A32330D1C
:10E320000A0024504D544B3235312C3139323030C3
:10E330002A32320D0A00B56206010300F00500FF23
:10E3400019B56206010300F00300FD15B562060170
:10E350000300F00100FB11B56206010300F00000AC
:10E36000FA0FB56206010300F00200FC13B5620665
:10E37000010300F00400FE17B5620601030001026C
:10E38000010E47B562060103000103010F49B562A2
:10E3900006010300010601124FB5620601030001E8
:10E3A00012011E67B562061608000307030000008D
:10E3B000000031E5B56206080600C8000100010052
:10E3C000DE6A00000000000000C201005CE20008FC
:10E3D0007FE200080100000000E1000094E2000874
:10E3E000B6E200080200000000960000CAE2000841
:10E3F000ECE2000803000000004B000000E300080E
:10E4000022E30008040000008025000029EB00083A
:10E4100029EB0008414552543132333400000000EA
:10E420006CF3000870F3000875F3000886F3000829
:10E430008FF300089AF30008A5F30008B0F3000872
:10E440007EF20008B9F3000878F20008C2F3000871
:10E45000CCF30008D7F30008DDF30008000000004B
:10E46000BEF20008C2F20008C8F20008CEF20008AE
:10E47000D1F20008D8F20008DBF20008E0F2000850
:10E48000ECF20008EFF20008F5F20008FCF20008D8
:10E4900006F3000810F3000819F3000827F300083A
:10E4A00033F300083AF3000840F300084DF3000886
:10E4B00058F3000865F3000800000000C0F00008F1
:10E4C000C4F00008AD870008EBF00008F0F0000889
:10E4D0007982000804F100080DF10008618200084B
:10E4E0002AF100082FF10008118800085EF10008E9
:10E4F00029EB00082982000863F100086BF100088D
:10E500003D8100087FF100088EF100081D810008A0
:10E51000A8F1000829EB0008757E0008ADF100089D
:10E52000B1F1000875800008FEF00008CDF1000888
:10E53000C5840008E0F10008E6F10008058700083E
:10E5400001F2000809F20008B986000818F2000874
:10E550001DF200084D80000809E800082DF20008AF
:10E56000658500085BF200084FF20008A17E0008F4
:10E5700062F2000829EB0008697E000829EB000818
:10E580008AF2000892F200089AF20008A2F200084B
:10E59000A9F20008B4F20008B9F200080000000077
:10E5A0004166726F333220434C492076657273693D
:10E5B0006F6E20322E32204D617920203320323090
:10E5C0003134202F2032323A35303A3335202D2065
:10E5D00028636C65616E666C6967687429004176B2
:10E5E00061696C61626C6520636F6D6D616E6473EF
:10E5F0003A0D0A0025730925730D0A0053797374C7
:10E60000656D20557074696D653A202564207365C9
:10E61000636F6E64732C20566F6C746167653A206B
:10E620002564202A20302E3156202825645320626C
:10E63000617474657279290D0A0043505520256470
:10E640004D487A2C20646574656374656420736535
:10E650006E736F72733A2000257320004143434864
:10E66000573A202573002E2563004379636C65209B
:10E6700054696D653A2025642C2049324320457247
:10E68000726F72733A2025642C20636F6E6669671F
:10E690002073697A653A2025640D0A0020256420DC
:10E6A0002564000D0A5265626F6F74696E672E2EC5
:10E6B0002E00536176696E672E2E2E004D75737491
:10E6C00020626520616E79206F72646572206F66CA
:10E6D0002041455452313233340D0A004375727271
:10E6E000656E742061737369676E6D656E743A2030
:10E6F000004572726F723A20456E61626C652061EE
:10E700006E6420706C756720696E204750532066D8
:10E71000697273740D0A00456E61626C696E6720E0
:10E7200047505320706173737468726F7567682EF9
:10E730002E2E0D0A00456E61626C6564206665616F
:10E7400074757265733A2000417661696C61626C20
:10E75000652066656174757265733A2000496E764E
:10E76000616C69642066656174757265206E616DA7
:10E77000652E2E2E0D0A0044697361626C6564205B
:10E7800000456E61626C656420000D0A4C6561761F
:10E79000696E6720434C49206D6F64652E2E2E0DE7
:10E7A0000A00526573657474696E6720746F206423
:10E7B000656661756C74732E2E2E004E4709004FEE
:10E7C0004B0900437573746F6D206D697865723AFB
:10E7D000200D0A4D6F746F720954687209526F6C84
:10E7E0006C095069746368095961770D0A00232523
:10E7F000643A09002573090053616E6974792063D6
:10E800006865636B3A09007265736574006C6F61CB
:10E810006400496E76616C6964206D697865722068
:10E82000747970652E2E2E0D0A004C6F616465643C
:10E83000202573206D69782E2E2E0D0A0057726FD9
:10E840006E67206E756D626572206F6620617267FB
:10E85000756D656E74732C206E65656473206964D4
:10E86000782074687220726F6C6C207069746368B1
:10E87000207961770D0A004D6F746F72206E756D8F
:10E88000626572206D7573742062652062657477AD
:10E8900065656E203120616E642025640D0A004399
:10E8A000757272656E74206D697865723A20257391
:10E8B0000D0A00417661696C61626C65206D697852
:10E8C0006572733A20004D69786572207365742013
:10E8D000746F2025730D0A0043757272656E742083
:10E8E00073657474696E67733A200D0A002573208E
:10E8F00073657420746F20004552523A2056616C43
:10E9000075652061737369676E6D656E74206F75D0
:10E9100074206F662072616E67650D0A0045525261
:10E920003A20556E6B6E6F776E2076617269616208
:10E930006C65206E616D650D0A0043757272656EBF
:10E94000742070726F66696C653A2025640D0A0048
:10E9500055736167653A0D0A6D6F746F7220696E49
:10E96000646578205B76616C75655D202D20736829
:10E970006F77205B6F72207365745D206D6F746FAD
:10E98000722076616C75650D0A004E6F2073756399
:10E9900068206D6F746F722C207573652061206E16
:10E9A000756D626572205B302C2025645D0D0A0058
:10E9B0004D6F746F72202564206973207365742015
:10E9C00061742025640D0A00496E76616C696420CB
:10E9D0006D6F746F722076616C75652C20313030EC
:10E9E000302E2E323030300D0A0053657474696E4B
:10E9F00067206D6F746F7220256420746F2025640A
:10EA00000D0A006175782025752025750D0A0049CD
:10EA10006E76616C69642046656174757265206903
:10EA20006E6465783A206D757374206265203C20B1
:10EA300025750D0A0043757272656E7420436F6E02
:10EA40006669673A20436F707920657665727974DC
:10EA500068696E672062656C6F7720686572652EE5
:10EA60002E2E0D0A006D697865722025730D0A003F
:10EA7000636D697820256400636D697820256420C2
:10EA8000302030203020300D0A00666561747572C8
:10EA900065202D25730D0A00666561747572652009
:10EAA00025730D0A006D61702025730D0A007365D2
:10EAB00074202573203D20000D0A456E746572692F
:10EAC0006E6720434C49204D6F64652C207479702B
:10EAD000652027657869742720746F2072657475C6
:10EAE000726E2C206F72202768656C70270D0A00EB
:10EAF0000D0A2320000D1B5B4B001B5B324A1B5B86
:10EB0000313B3148004552523A20556E6B6E6F775B
:10EB10006E20636F6D6D616E642C20747279202796
:10EB200068656C702700082008006C6F6F7074694E
:10EB30006D6500656D665F61766F6964616E6365C2
:10EB4000006D69647263006D696E636865636B0074
:10EB50006D6178636865636B006D696E7468726F70
:10EB600074746C65006D61787468726F74746C6530
:10EB7000006D696E636F6D6D616E640064656164E4
:10EB800062616E6433645F6C6F77006465616462B8
:10EB9000616E6433645F68696768006E657574727E
:10EBA000616C3364006465616462616E6433645FE8
:10EBB0007468726F74746C65006D6F746F725F70DF
:10EBC000776D5F7261746500736572766F5F7077E1
:10EBD0006D5F726174650072657461726465645F13
:10EBE00061726D00666C6170735F7370656564005F
:10EBF000666978656477696E675F616C74686F6C6D
:10EC0000645F646972007265626F6F745F636861EC
:10EC100072616374657200736F66747365726961A3
:10EC20006C5F626175647261746500736F667473A2
:10EC3000657269616C5F315F696E76657274656477
:10EC400000736F667473657269616C5F325F696EC1
:10EC5000766572746564006770735F7479706500BF
:10EC60006770735F62617564726174650073657269
:10EC700069616C72785F747970650074656C656D3C
:10EC8000657472795F70726F76696465720074651D
:10EC90006C656D657472795F706F72740074656C09
:10ECA000656D657472795F73776974636800766205
:10ECB00061747363616C6500766261746D61786321
:10ECC000656C6C766F6C7461676500766261746DFB
:10ECD000696E63656C6C766F6C7461676500706FEC
:10ECE0007765725F6164635F6368616E6E656C0017
:10ECF000616C69676E5F6779726F00616C69676EDE
:10ED00005F61636300616C69676E5F6D616700617D
:10ED10006C69676E5F626F6172645F726F6C6C00CA
:10ED2000616C69676E5F626F6172645F7069746362
:10ED30006800616C69676E5F626F6172645F7961C0
:10ED400077006D61785F616E676C655F696E636C9B
:10ED5000696E6174696F6E006779726F5F6C70665F
:10ED6000006D6F726F6E5F7468726573686F6C644C
:10ED7000006779726F5F636D70665F666163746F61
:10ED800072006779726F5F636D70666D5F66616355
:10ED9000746F7200616C745F686F6C645F7468722A
:10EDA0006F74746C655F6E65757472616C00616C14
:10EDB000745F686F6C645F666173745F6368616ED3
:10EDC0006765007468726F74746C655F636F7272EC
:10EDD000656374696F6E5F76616C756500746872E7
:10EDE0006F74746C655F636F7272656374696F6E64
:10EDF0005F616E676C65007961776465616462610B
:10EE00006E64007961775F636F6E74726F6C5F64BC
:10EE10006972656374696F6E007961775F646972A6
:10EE2000656374696F6E007472695F756E61726D8F
:10EE300065645F736572766F0072635F726174659B
:10EE40000072635F6578706F007468725F6D6964EB
:10EE5000007468725F6578706F00726F6C6C5F70C1
:10EE6000697463685F72617465007961775F72616C
:10EE70007465007470615F72617465007470615FC5
:10EE8000627265616B706F696E74006661696C7344
:10EE90006166655F64656C6179006661696C736168
:10EEA00066655F6F66665F64656C6179006661695F
:10EEB0006C736166655F7468726F74746C6500660C
:10EEC00061696C736166655F6465746563745F74C2
:10EED00068726573686F6C6400727373695F6175E3
:10EEE000785F6368616E6E656C0067696D62616C06
:10EEF0005F666C616773006163635F68617264770A
:10EF0000617265006163635F6C70665F6661637404
:10EF10006F720061636378795F6465616462616EDA
:10EF200064006163637A5F6465616462616E64005A
:10EF30006163635F756E61726D656463616C0061CE
:10EF400063635F7472696D5F7069746368006163A5
:10EF5000635F7472696D5F726F6C6C006261726F77
:10EF60005F7461625F73697A65006261726F5F6E80
:10EF70006F6973655F6C7066006261726F5F636674
:10EF80005F76656C006261726F5F63665F616C746F
:10EF9000006D61675F6465636C696E6174696F6E53
:10EFA000006770735F706F735F70006770735F707E
:10EFB0006F735F69006770735F706F735F64006782
:10EFC00070735F706F73725F70006770735F706FE4
:10EFD00073725F69006770735F706F73725F640054
:10EFE0006770735F6E61765F70006770735F6E61EC
:10EFF000765F69006770735F6E61765F640067704B
:10F00000735F77705F726164697573006E61765FBC
:10F01000636F6E74726F6C735F68656164696E674D
:10F02000006E61765F73706565645F6D696E006E1A
:10F0300061765F73706565645F6D6178006E61769F
:10F040005F736C65775F72617465007069645F639C
:10F050006F6E74726F6C6C657200705F7069746350
:10F060006800695F706974636800705F726F6C6CD0
:10F0700000695F726F6C6C00705F79617700695F27
:10F0800079617700705F616C7400695F616C740016
:10F09000645F616C7400705F6C6576656C00695FBD
:10F0A0006C6576656C00645F6C6576656C00705F9E
:10F0B00076656C00695F76656C00645F76656C00F0
:10F0C00061757800666561747572655F6E616D6506
:10F0D00020617578666C6167206F7220626C616E6A
:10F0E0006B20666F72206C69737400636D697800C1
:10F0F00064657369676E20637573746F6D206D69E5
:10F100007865720064656661756C7473007265730E
:10F11000657420746F2064656661756C747320611A
:10F120006E64207265626F6F740064756D7000703C
:10F1300072696E7420636F6E666967757261626C66
:10F14000652073657474696E677320696E20612031
:10F150007061737461626C6520666F726D006578B2
:10F1600069740066656174757265006C69737420FA
:10F170006F72202D76616C206F722076616C006753
:10F180007073706173737468726F75676800706113
:10F1900073737468726F7567682067707320746F1B
:10F1A0002073657269616C0068656C70006D6170D8
:10F1B000006D617070696E67206F662072632063F6
:10F1C00068616E6E656C206F72646572006D69783F
:10F1D0006572206E616D65206F72206C69737400BA
:10F1E0006D6F746F72006765742F736574206D6F37
:10F1F000746F72206F75747075742076616C7565AC
:10F200000070726F66696C6500696E6465782028AD
:10F210003020746F20322900736176650073617647
:10F220006520616E64207265626F6F74006E616D3F
:10F23000653D76616C7565206F7220626C616E6BE6
:10F24000206F72202A20666F72206C6973740073BD
:10F25000686F772073797374656D2073746174754A
:10F26000730076657273696F6E004759524F0041A3
:10F270004343004241524F00534F4E4152004750CA
:10F2800053004750532B4D4147004144584C3334B1
:10F2900035004D505536303530004D4D4138343500
:10F2A0007800424D41323830004C534D33303344B6
:10F2B0004C48430046414B45004E6F6E650054522A
:10F2C000490051554144500051554144580042496C
:10F2D0000047494D42414C005936004845583600D8
:10F2E000464C59494E475F57494E470059340048EC
:10F2F00045583658004F43544F5838004F43544FE9
:10F30000464C415450004F43544F464C41545800D2
:10F31000414952504C414E450048454C495F3132BD
:10F32000305F4343504D0048454C495F39305F449E
:10F33000454700565441494C34004845583648002A
:10F3400050504D5F544F5F534552564F0044554106
:10F350004C434F505445520053494E474C45434F40
:10F360005054455200435553544F4D0050504D009A
:10F370005642415400494E464C494748545F414328
:10F38000435F43414C0053455249414C5258004D54
:10F390004F544F525F53544F5000534552564F5F96
:10F3A00054494C5400534F465453455249414C0024
:10F3B0004C45445F52494E47004641494C534146F3
:10F3C000450054454C454D4554525900504F574502
:10F3D000524D4554455200564152494F0033440066
:10F3E0006AF200086FF2000873F2000886F2000863
:10F3F00078F200087EF2000882F2000800000000A7
:10F400002AEB000802000000DC10002000000000D1
:10F410002823000033EB000800000000DE1000206D
:10F42000000000000100000041EB000802000000A5
:10F43000E2110020B0040000A406000047EB000821
:10F4400002000000E411002000000000D0070000CE
:10F4500050EB000802000000E61100200000000050
:10F46000D007000059EB000802000000A0110020A6
:10F4700000000000D007000065EB0008020000005B
:10F48000A211002000000000D007000071EB00086E
:10F4900002000000A411002000000000D0070000BE
:10F4A0007CEB000802000000A61100200000000014
:10F4B000D00700008BEB000802000000A81100201C
:10F4C00000000000D00700009BEB000802000000D5
:10F4D000AA11002000000000D0070000A5EB0008E2
:10F4E00002000000AC11002000000000D007000066
:10F4F000B9EB000802000000AE110020320000004D
:10F50000007D0000C8EB000802000000B0110020E0
:10F5100032000000F2010000D7EB000800000000FC
:10F52000E81100200000000001000000E4EB0008EA
:10F5300000000000E911002000000000640000004D
:10F54000F0EB000801000000EA110020FFFFFFFFC0
:10F550000100000006EC000800000000FA11002085
:10F56000300000007E0000001BEC000804000000DA
:10F57000F0110020B004000000C2010017EC0008E8
:10F5800004000000F4110020B0040000004B000053
:10F590002BEC000800000000F81100200000000023
:10F5A0000100000041EC000800000000F9110020FB
:10F5B000000000000100000057EC000800000000FF
:10F5C000EC110020000000000400000060EC0008C6
:10F5D00001000000ED110020000000000400000008
:10F5E0006DEC000800000000E011002000000000A9
:10F5F000040000007BEC000800000000FC1100206B
:10F6000000000000010000008EEC00080000000077
:10F61000FD11002000000000020000009DEC000829
:10F6200000000000FE1100200000000001000000AA
:10F63000AEEC000800000000D41100200A00000019
:10F64000C8000000B8EC000800000000D511002040
:10F650000A00000032000000CBEC000800000000AF
:10F66000D61100200A00000032000000DEEC000885
:10F6700000000000D7110020000000000900000079
:10F68000F0EC000800000000B211002000000000B3
:10F6900008000000FBEC000800000000B31100208F
:10F6A000000000000800000005ED00080000000058
:10F6B000B411002000000000080000000FED000859
:10F6C00003000000B61100204CFFFFFF680100009E
:10F6D00020ED000803000000B81100204CFFFFFFE0
:10F6E0006801000032ED000803000000BA1100209C
:10F6F0004CFFFFFF6801000042ED0008020000001F
:10F70000C6110020640000008403000058ED0008CA
:10F7100002000000BE1100200000000000010000F7
:10F7200061ED000800000000C4110020000000008E
:10F730008000000071ED000802000000C0110020F0
:10F7400064000000E803000082ED000802000000F1
:10F75000C211002064000000E803000094ED0008DE
:10F7600000000000EA14002001000000FA00000080
:10F77000AEED000800000000EB14002000000000C7
:10F7800001000000C3ED000800000000EE1400209E
:10F790000000000096000000DDED000802000000FF
:10F7A000EC140020010000008403000019EF0008A1
:10F7B00000000000E814002000000000200000000D
:10F7C000F7ED000800000000E91400200000000030
:10F7D0006400000003EE000801000000BC110020DE
:10F7E000FFFFFFFF0100000019EE0008010000000C
:10F7F00036150020FFFFFFFF0100000027EE000884
:10F80000010000003715002000000000010000008A
:10F8100039EE0008000000009714002000000000EE
:10F82000FA00000041EE00080000000098140020DB
:10F83000000000006400000049EE00080000000025
:10F8400099140020000000006400000051EE000840
:10F85000000000009A140020000000006400000076
:10F860005AEE0008000000009B1400200000000079
:10F87000640000006AEE0008000000009C140020F4
:10F88000000000006400000073EE000800000000AB
:10F890009D14002000000000640000007CEE0008C1
:10F8A000020000009E140020E8030000D0070000C2
:10F8B0008BEE000800000000301500200000000062
:10F8C000C80000009AEE000800000000311500207A
:10F8D00000000000C8000000ADEE000802000000BB
:10F8E00032150020E8030000D0070000BFEE00083A
:10F8F000020000003415002064000000D007000062
:10F90000D9EE000801000000EB110020000000000B
:10F9100004000000EAEE0008000000003815002096
:10F9200000000000FF000000F7EE000800000000EB
:10F93000BD110020000000000500000004EF0008D9
:10F9400000000000A614002000000000FA000000E3
:10F9500013EF000800000000A814002000000000C1
:10F960006400000022EF000800000000A71400203F
:10F97000000000006400000030EF000800000000FC
:10F98000BC14002000000000010000003FEF000850
:10F9900003000000A4140020D4FEFFFF2C0100008F
:10F9A0004EEF000803000000A2140020D4FEFFFF69
:10F9B0002C0100005CEF000800000000AC140020E7
:10F9C00000000000300000006AEF000805000000A1
:10F9D000B0140020000000000100000079EF0008D2
:10F9E00005000000B4140020000000000100000029
:10F9F00085EF000805000000B8140020000000009A
:10FA00000100000091EF000803000000A014002096
:10FA1000B0B9FFFF50460000A1EF00080000000051
:10FA20007D14002000000000C8000000ABEF0008BB
:10FA3000000000008714002000000000C800000043
:10FA4000B5EF000800000000911400200000000045
:10FA5000C8000000BFEF0008000000007E14002076
:10FA600000000000C8000000CAEF0008000000000D
:10FA70008814002000000000C8000000D5EF000836
:10FA8000000000009214002000000000C8000000E8
:10FA9000E0EF0008000000007F14002000000000DC
:10FAA000C8000000EAEF00080000000089140020F0
:10FAB00000000000C8000000F4EF00080000000093
:10FAC0009314002000000000C8000000FEEF0008B2
:10FAD000020000003A15002000000000D0070000DE
:10FAE0000CF00008000000003E150020000000009F
:10FAF0000100000021F00008020000004015002075
:10FB00000A000000D00700002FF0000802000000EB
:10FB1000421500200A000000D00700003DF0000858
:10FB2000000000003D1500200000000064000000FF
:10FB30004BF00008000000007814002000000000D6
:10FB4000010000005AF00008000000007A140020B4
:10FB500000000000C800000062F000080000000083
:10FB60008414002000000000C80000002AED0008F6
:10FB7000000000008E14002000000000C8000000FB
:10FB80006AF0000800000000791400200000000066
:10FB9000C800000071F0000800000000831400207D
:10FBA00000000000C800000019ED0008000000007F
:10FBB0008D14002000000000C800000078F000084C
:10FBC000000000007B14002000000000C8000000BE
:10FBD0007EF00008000000008514002000000000F6
:10FBE000C80000003CED0008000000008F14002059
:10FBF00000000000C800000084F0000800000000C1
:10FC00007C14002000000000C80000008AF00008FA
:10FC1000000000008614002000000000C800000062
:10FC200090F0000800000000901400200000000088
:10FC3000C800000096F000080000000080140020BA
:10FC400000000000C80000009EF000080000000056
:10FC50008A14002000000000C8000000A6F0000880
:10FC6000000000009414002000000000C800000004
:10FC7000AEF0000800000000821400200000000028
:10FC8000C8000000B4F00008000000008C14002040
:10FC900000000000C8000000BAF0000800000000EA
:10FCA0009614002000000000C8000000524F4C4C89
:10FCB0003B50495443483B5941573B414C543B50BE
:10FCC0006F733B506F73523B4E6176523B4C4556BF
:10FCD000454C3B4D41473B56454C3B0041524D3B0B
:10FCE00000414E474C453B00484F52495A4F4E3B0E
:10FCF000004241524F3B00564152494F3B004D415B
:10FD0000473B0048454144465245453B0048454134
:10FD10004441444A3B0043414D535441423B00431C
:10FD2000414D545249473B0047505320484F4D45A1
:10FD30003B0047505320484F4C443B0050415353E5
:10FD4000544852553B004245455045523B004C45B6
:10FD5000444D41583B004C45444C4F573B004C4CA4
:10FD600049474854533B0043414C49423B00474FAD
:10FD70005645524E4F523B004F53442053573B0081
:10FD800054454C454D455452593B00000000004B32
:10FD9000000000CB61636F7366000000000000008C
:10FDA0007371727466000000000FC93F000F494074
:10FDB00000CB9640000FC9400053FB4000CB1641DA
:10FDC00000ED2F41000F49410031624100537B415A
:10FDD000003A8A4100CB9641005CA34100EDAF415F
:10FDE000007EBC41000FC94100A0D5410031E24175
:10FDF00000C2EE410053FB4100F20342003A0A42C6
:10FE00000083104200CB164200141D42005C2342C6
:10FE100000A5294200ED2F4200363642007E3C42CA
:10FE200000C74242000F4942A2000000F900000052
:10FE3000830000006E0000004E000000440000003F
:10FE40001500000029000000FC0000002700000051
:10FE500057000000D1000000F50000003400000051
:10FE6000DD000000C0000000DB00000062000000B8
:10FE700095000000990000003C00000043000000D5
:10FE80009000000041000000FE0000005100000052
:10FE900063000000AB000000DE000000BB000000BB
:10FEA000C500000061000000B70000002400000051
:10FEB0006E0000003A000000420000004D0000000B
:10FEC000D2000000E0000000060000004900000031
:10FED0002E000000EA00000009000000D100000030
:10FEE000920000001C000000FE0000001D00000049
:10FEF000EB0000001C000000B10000002900000021
:10FF0000A70000003E000000E800000082000000A2
:10FF100035000000F50000002E000000BB000000CE
:10FF20004400000084000000E90000009C00000084
:10FF30007000000026000000B40000005F00000018
:10FF40007E00000041000000390000009100000028
:10FF5000D6000000390000008300000053000000BC
:10FF600039000000F40000009C0000008400000044
:10FF70005F0000008B000000BD000000F9000000E1
:10FF8000280000003B0000001F000000F8000000F7
:10FF900097000000FF000000DE00000005000000E8
:10FFA000980000000F000000EF0000002F0000008C
:10FFB000110000008B0000005A0000000A00000041
:10FFC0006D0000001F0000006D0000003600000002
:10FFD0007E000000CF00000027000000CB000000E2
:10FFE00009000000B70000004F00000046000000BC
:10FFF0003F000000660000009E0000005F0000005F
:020000040801F1
:10000000EA0000002D00000075000000270000003D
:10001000BA000000C7000000EB000000E50000008F
:10002000F10000007B0000003D0000000700000020
:1000300039000000F70000008A00000052000000B4
:1000400092000000EA0000006B000000FB000000CE
:100050005F000000B10000001F0000008D000000E4
:100060005D000000080000005600000003000000D2
:100070003000000046000000FC0000007B00000093
:100080006B000000AB000000F0000000CF0000009B
:10009000BC000000200000009A000000F4000000F6
:1000A000360000001D000000A9000000E300000071
:1000B00091000000610000005E000000E60000000A
:1000C0001B0000000800000065000000990000000F
:1000D000850000005F00000014000000A000000088
:1000E00068000000400000008D000000FF000000DC
:1000F000D8000000800000004D00000073000000E8
:10010000270000003100000006000000060000008B
:100110001500000056000000CA0000007300000037
:10012000A8000000C900000060000000E20000001C
:100130007B000000C00000008C0000006B0000008D
:100140000400000007000000090000000000C93F93
:100150000000F0390000DA370000A2330000842EDE
:100160000000502B0000C2270000D0220000C41F56
:100170000000C61B000044176937AC3168212233E8
:10018000B40F14336821A2333863ED3EDA0F493FD0
:100190005E987B3FDA0FC93F0020202020202020DE
:1001A0002020282828282820202020202020202027
:1001B0002020202020202020208810101010101037
:1001C0001010101010101010100404040404040483
:1001D000040404101010101010104141414141411D
:1001E00001010101010101010101010101010101FF
:1001F000010101011010101010104242424242420F
:1002000002020202020202020202020202020202CE
:100210000202020210101010200000000000000076
:1002200000000000000000000000000000000000CE
:1002300000000000000000000000000000000000BE
:1002400000000000000000000000000000000000AE
:10025000000000000000000000000000000000009E
:10026000000000000000000000000000000000008E
:10027000000000000000000000000000000000007E
:10028000000000000000000000000000000000006E
:10029000000000000000000000000000430000001B
:1002A000A8010020F8B500BFF8BC08BC9E46704706
:0C02B000F8B500BFF8BC08BC9E467047C3
:0802BC006DDA000835010008AD
:0402C400110100081C
:1002C800000000400000020000000040040004009C
:1002D8000000004008000800000000400C0010006A
:1002E8000004004000000200000400400400040074
:1002F8000004004008000800000400400C00100042
:1003080003010001554600080000803F000000007E
:1003180000000000DC05DC05DC05DC05DC05DC058F
:10032800DC05DC050000803F010000000000000043
:10033800DCFC00080000000001000000E1FC0008EF
:100348000100000002000000E8FC000802000000B4
:1003580003000000F1FC0008030000000400000096
:10036800F7FC00080400000005000000FEFC00087F
:10037800050000000600000003FD0008060000005C
:10038800070000000DFD000807000000080000003D
:1003980016FD000808000000090000001FFD000805
:1003A800090000000A00000028FD00080A000000FB
:1003B8000B00000032FD00080B0000000C000000DC
:1003C8003CFD00080C0000000D00000046FD000880
:1003D8000D0000000E0000004EFD00080E00000099
:1003E8000F00000056FD00080F000000100000007C
:1003F8005EFD0008100000001100000067FD000805
:1004080011000000120000006EFD0008120000003C
:100418001300000078FD000813000000140000001D
:1004280080FD000814000000150000000000000016
:10043800FF000000000000000000000001020304AB
:100448000607080900127A0000A24A0402040608F6
:100458000000000001020304010203040607080962
:100468000100000098010108000000009404002029
:10047800FC040020640500200000000000000000CB
:100488000000000000000000000000000000000064
:100498000000000000000000000000009C020108AD
:1004A8000000000000000000000000000000000044
:1004B8000000000000000000000000000000000034
:1004C8000000000000000000000000000000000024
:1004D8000000000000000000000000000000000014
:1004E8000000000000000000000000000000000004
:1004F80000000000000000000000000000000000F4
:1005080000000000000000000000000000000000E3
:1005180001000000000000000E33CDAB34126DE680
:10052800ECDE05000B0000000000000000000000E9
:1005380000000000000000000000000000000000B3
:1005480000000000000000000000000000000000A3
:100558000000000000000000000000000000000093
:100568000000000000000000000000000000000083
:04089800A801002093
:0400000508000000EF
:00000001FF
